:020000040800F2
:1000000000000120D5450008512C0008532C0008A1
:10001000552C0008572C0008592C0008000000003F
:100020000000000000000000000000005B2C000841
:100030005D2C0008000000005F2C0008612C000807
:100040002546000825460008652C000825460008BE
:100050002546000825460008712C000825460008A2
:1000600025460008A52C0008AB2C000825460008F2
:10007000772C0008792C00087D2C0008892C0008BA
:10008000952C0008992C00082546000825460008F4
:100090000000000025460008AD2C00082546000899
:1000A0002546000825460008254600082546000884
:1000B0002546000825460008254600082546000874
:1000C0002546000825460008254600082546000864
:1000D00025460008B12C00082546000825460008E2
:1000E00025460008AF2C0008BD2C00082546000856
:1000F000254600080000000000000000254600081A
:100100002546000825460008C92C00082546000899
:100110002546000825460008254600082546000813
:100120002546000825460008254600082546000803
:080130002546000825460008E1
:1001400010B5054C237833B9044B13B10448AFF311
:1001500000800123237010BD840A002000000000ED
:10016000A86C010808B5034B1BB103490348AFF362
:10017000008008BD00000000880A0020A86C01086B
:1001800014214160704714207047406A7047000096
:1001900081010008870100088B010008A101000807
:1001A00010B5044604F1100000F05CFCC4F8F8003F
:1001B0000148C4F87C0110BD90010008F8B5E6B014
:1001C00004460D4616461F460A4906A800F0CAFE18
:1001D00070996F9A05910492009733466E996D9AC3
:1001E000039102922A466C990191214600F060F831
:1001F00067B0F0BD9C010008F8B5E6B004460D46B6
:1002000016461F46094906A800F0ACFE6F996E9A83
:100210000491039200976D996C9A02910192334672
:100220002A46214600F087F867B0F0BD9C0100081F
:1002300038B500281CBF01680029184A23D1184B83
:100240001C684FF6F0710C404CF24025AC421FBFC9
:100250001B6819404CF27024A14212D1114D29683B
:1002600079B911490B68C3F30B03B3F58A6F1FBF4C
:100270000968C1F30B0140F28343994204BF012195
:10028000117028B905E0094B994204BF0121117092
:100290004068BDE8324002F015B900BFA00A002056
:1002A00000ED00E0002004E00010005C0000374892
:1002B0002DE9F04104460D46216816464A681F465E
:1002C00090478046B8F5403F2ED122680A9993683E
:1002D000204698478046B8F5403F25D12368089AC4
:1002E0000799D3F80CC02046E0478046B8F5403F58
:1002F0001AD12368069A39461F692046B8478046B6
:10030000B8F5403F10D1236829465D693246204642
:10031000A8478046B8F5403F06D123680B9A099953
:100320009D692046A847804621680A682046904774
:100330004046BDE8F0812DE9F04104460D462168B4
:1003400016464A681F4690478046B8F5403F2ED172
:1003500022680A999368204698478046B8F5403F3E
:1003600025D12368089A0799D3F80CC02046E047A6
:100370008046B8F5403F1AD12368069A39461F696E
:100380002046B8478046B8F5403F10D1236829463B
:100390005D6932462046A8478046B8F5403F06D101
:1003A00023680999DD6900222046A8478046216814
:1003B0000A68204690474046BDE8F0814FF440303F
:1003C00070470000F0B50C4685B0114600281A466B
:1003D0001CBF0568002D0B4B11D082B104B971B957
:1003E0000D9860B10F9E0E9F0A9B02900496039792
:1003F0000B980C9E009001962046A847034618468D
:1004000005B0F0BD020003002DE9F04F0646D0B064
:100410000868F56DD6F860E0726EB76EF36E00BADC
:1004200000906C46486800BA60600DF1400888682A
:1004300000BAA060C86800BAE060086900BA20612C
:10044000486900BA6061886900BAA061C86900BAE9
:10045000E061086A00BA2062486A00BA6062886A8D
:1004600000BAA062C86A00BAE062086B00BA2063F2
:10047000486B00BA6063886B00BAA063C86B00BAAF
:10048000E063402058F80C1C58F820CC58F838ACE1
:100490008CEA010158F840CC8AEA01018CEA010992
:1004A0004FEAF979401E48F8049BEBD187EA020035
:1004B00000EA0E00784010EBF5610098DFF824C4E4
:1004C00041186144C81882EABE032B404FEAF0612C
:1004D00053405918636859186144CF194FEAB5035E
:1004E00083EABE01014081EABE0111EBF765A16814
:1004F0004D196544A91883EAB0023A404FEAF16504
:100500005A405519E26855194FEAB70282EAB00716
:1005100065440F4005EBBE0E97EAB00717EBFE658A
:1005200027697D194FEAB10782EA0701654401EAAC
:100530000E01EB18514011EBF36561694D194FEA5B
:10054000BE0187EA010E65440EEA030E15EBB0000A
:100550008EEA070E0EEBF065D4F818E0754465449A
:10056000AA1881EAB30505404FEAF26E4D40AE4449
:10057000E569AE44E64477444FEAB00080EAB30E42
:100580000EEA020E8EEAB30E0EEBF765D4F820E009
:1005900075446544691880EAB2053D404FEAF16E42
:1005A0004540AE44656AAE44E6440EEBB3034FEA01
:1005B000B70787EAB20E0EEA010E8EEAB20E0EEB14
:1005C000F365D4F828E075446544281887EAB10536
:1005D0001D404FEAF06E7D40AE44E56AAE44E6440D
:1005E0000EEBB2024FEAB30383EAB10E0EEA000E3D
:1005F0008EEAB10E0EEBF265D4F830E07544654436
:10060000EF1983EAB00515404FEAF76E5D40AE443E
:10061000656BAE44E6440EEBB1014FEAB20282EAEA
:10062000B00E0EEA070E8EEAB00E0EEBF165D4F8AE
:1006300038E075446544EB1882EAB7050D404FEA8F
:10064000F36E5540AE44E56BAE44E6440EEBB000AD
:100650004FEAB10181EAB70E0EEA030E8EEAB70E39
:100660000EEBF065D4F840E07544654481EAB30EC2
:10067000AA180EEA000E4FEAF2658EEA010E7544E2
:10068000DDF844E04FEAB000754480EAB30E6544FB
:100690000EEA020E15EBB7078EEAB30E0EEBF76506
:1006A000DDF848E04FEAB202754480EA020E654484
:1006B0000EEA070E69188EEA000E0EEBF165DDF802
:1006C0004CE07544654405EBB3034FEAB70E1427BD
:1006D0000DF1500CDFF810528EEA010B82EA0B0B81
:1006E0000BEBF36A5CF804BBDA44AA44504483EA97
:1006F000B10B4FEAF06A8EEA0B0BDA445CF804BBEC
:10070000DA44AA44524480EAB30B4FEAF26A8BEA15
:10071000B10BDA445CF804BBDA444FEAB000AA44F7
:1007200080EA020BD6448BEAB30B0BEBFE6A5CF853
:1007300004BBDA444FEAB202AA4482EA0E0B0AEB87
:10074000B10180EA0B0B0BEBF16A5CF804BBDA44F5
:100750007F1DAA44282F0AEBB3034FEABE0EBBD37A
:100760003C2F61D3502F4DD204EB870CC7F15407B7
:100770005E4CA7FB04A504465D4FA8088EEA010A5B
:1007800082EA0A0A5CF804BB0AEBF3655D447D1952
:100790002C1983EAB10A4FEAF4658EEA0A0A554435
:1007A0005CF804AB5CF804BB55447D19AA1884EAD4
:1007B000B30A4FEAF2658AEAB10A55445D444FEA4A
:1007C000B4047D1984EA020AAE448AEAB30A0AEB49
:1007D000FE655CF804AB55444FEAB2027D1982EA2B
:1007E0000E0A15EBB10184EA0A0A5CF804BB0AEBB5
:1007F000F1655D447D1915EBB303401E4FEABE0E53
:10080000BCD12046F46D1B19F365336EC9183166EF
:10081000716E71447166B36ED218B266F16E401893
:10082000F06650B0BDE8F08F4EEA010B0EEA010A07
:100830000BEA020B4BEA0A0A0AEBF36554F827A00D
:10084000DFF8B0C0554443EAB10B654403EAB10A8E
:100850000BEA0E0B28184BEA0A0A7F1C0AEBF0651C
:1008600054F827A0554440EAB30B654400EAB30AA4
:100870000BEAB10BAA184BEA0A0A7F1C0AEBF265D5
:1008800054F827A055444FEAB00040EA020B6544F3
:1008900000EA020A0BEAB30BAE444BEA0A0A7F1CD9
:1008A0000AEBFE6554F827A055444FEAB20242EA2B
:1008B0000E0B654402EA0E0A0BEA000B15EBB101C0
:1008C0004BEA0A0A7F1C0AEBF16554F827A055444D
:1008D0007F1C65443C2F05EBB3034FEABE0EA3D348
:1008E00040E700BF9979825AA1EBD96ECDCCCCCC30
:1008F000D6C162CADCBC1B8F00B581B00168074A53
:10090000914200D110B9064801B000BD7C2114F01D
:10091000A6FA4FF4003001B000BD00BF040A000881
:10092000030002002DE9F0410B4A92E8F85188B02B
:10093000694681E8F8510268084B9A4200D118B91B
:10094000074808B0BDE8F0811422083000F04FFBE2
:1009500008B0BDE8F08100BFE4090008040A0008FF
:1009600003000200152904D20268044B9A4200D108
:1009700008B903487047083000F048BB040A000873
:100980000300020010B481B013460268074CA24273
:1009900000D118B901B010BC0548704701B000F192
:1009A000240210BC083000F035BB00BF040A000868
:1009B0000300020010B481B013460268074CA24243
:1009C00000D118B901B010BC054870470A4601B003
:1009D00000F1240110BC083000F070BB040A0008CC
:1009E000030002000123456789ABCDEFFEDCBA9816
:1009F00076543210F0E1D2C3000000000000000085
:100A000000000000F9080008250900086509000831
:100A100085090008B509000809040008810F0008CD
:100A2000CD0F0008890F0008F0B5A3B004460B48AD
:100A300002900D4616461F46094B0822402104A885
:100A400000F0D1FA28980190009733462A462146B3
:100A500002A800F01BF823B0F0BD00BF040A000894
:100A6000180A000810B5040008BF002408D0054883
:100A7000054B20600822402104F1080000F0B3FA81
:100A8000204610BD040A0008180A00082DE9F041AC
:100A900004460E46216817464A681D469047804620
:100AA000B8F5003F19D12268069993682046984707
:100AB0008046B8F5003F10D123683146DE683A46DB
:100AC0002046B0478046B8F5003F06D12368079A14
:100AD00029461D692046A847804621680A682046A5
:100AE00090474046BDE8F08110B500F033FA4FF46E
:100AF000403400280EBF034C4FF4C07114F0AFF91E
:100B0000204610BD0200030010B5044600F022FA92
:100B100008B9054810BD0021A160D0F87C211168FA
:100B200088474FF4403010BD0200030070B5044602
:100B30000D4600F00FFA064E40B1D0F87C01416836
:100B40008847A84224BF65604FF44036304670BDE8
:100B5000020003002DE9FF4715000C4600D02CB120
:100B6000064600F0F7F95FEA000801D16448C3E0E7
:100B7000D8F8F80001684A689047B0F5003F17D1EF
:100B8000D8F87C118A68404690478146B9F1810FB8
:100B900080F09E80A94508F1FC0A17D2D8F8F80029
:100BA0000368D3F80CC02A462146E047B0F5003F61
:100BB00040F08E80D8F8F8000368D3F810C06A4679
:100BC0005146E047B0F5003F76D10AE0002004E04E
:100BD000215C0AF800100098401C00900098A84280
:100BE000F6D34FF0000C4749474A484B01AC0098F8
:100BF000844558D2D3E9007001ADC5E90070107882
:100C000000281ABF042086464FF0000E085854F8FA
:100C10000E5028443E4D05600127D0F800E0876063
:100C2000019D4F681AF80C007D408EEA050585F09D
:100C3000040E65680F687D4085F0FC05754485F0FD
:100C4000A30568400AF80C000CF1010CCFE7D3E9CA
:100C5000004501A8C0E9004510782E4D002814BFBA
:100C60004FF0040E4FF0000E01A8744651F80EE04C
:100C70000459A6440127CEF80050DEF80040CEF813
:100C800008704D68019F40687D406C400D68684069
:100C900084F0040480F0FC00041984F057040AF87E
:100CA0000C400CF1010CCC45D1D3D8F8F800016808
:100CB0004A689047B0F5003F0AD1D8F8F8000368B9
:100CC000D3F80C804A465146C047B0F5003F01D0EA
:100CD000114811E0002006E05AF8201081F06A3136
:100CE0004AF82010401CB0EB990FF5D3B06840F0E3
:100CF0000100B0604FF4403004B0BDE8F08700BFA1
:100D000002000300406D0108A00A00202C0F00081B
:100D1000ADBE4ED70DBE75A10100030038B50C461F
:100D2000017A1546CA0702D500F014F908B9084837
:100D300032BDD0F8F80003682146DC682A46A04797
:100D4000B0F5003F01D0034832BD4FF4403032BD12
:100D500002000300010003002DE9F84191B00546AF
:100D60000E461746402101A814F079F8297AC807E1
:100D700004D5284600F0EEF8040002D1DFF8A48084
:100D80004BE0D4F8F800DFF8A0800368D3F810C077
:100D90006A4601A9E047B0F5003F3ED1D4F8F8001B
:100DA00001684A689047B0F5003F36D1D4F87C110D
:100DB0008A6820469047D4F8F830024618461B68E7
:100DC000D3F80CC004F1FC01E047B0F5003F24D19A
:100DD000D4F87C0141688847D4F8F83002461846B8
:100DE0001B68D3F80CC001A9E047B0F5003F14D14F
:100DF000D4F8F8000268696893689847B0F5003F36
:100E00000BD1D4F8F80003681C693A463146A04774
:100E1000B0F5003F08BF4FF44038404612B0BDE87F
:100E2000F08100BF02000300010003002DE9F8413A
:100E3000A5B0074688461646402115A814F00FF8BD
:100E400000220492402105A814F009F8387AC1075D
:100E50005ED5384600F07EF8050059D0D5F8F80088
:100E60002D4C0368D3F810C06A4605A9E047B0F5D9
:100E7000003F3CD1D5F8F80001684A689047B0F5CA
:100E8000003F34D1D5F87C118A6828469047D5F8C0
:100E9000F830024618461B68D3F80CC005F1FC0177
:100EA000E047B0F5003F22D1D5F87C014168884782
:100EB000D5F8F830024618461B68D3F80CC005A9CF
:100EC000E047B0F5003F12D1D5F8F8000268796824
:100ED00093689847B0F5003F09D1D5F8F80003684A
:100EE0001D6904AA15A9A847B0F5003F01D0204606
:100EF0000FE00A4B0A490B4A0396029101924046C1
:100F00001C68049B009415AA796800F0E5F900E0DC
:100F1000054826B0BDE8F08101000300486D0108D6
:100F2000936E030026C703000200030004B0010112
:100F300000170145E90A0008090B00082D0B0008FD
:100F4000BD030008550B00081D0D0008590D0008D1
:100F50002D0E00080168024A914218BF0020704718
:100F6000340F000810B5040008BF002404D0034863
:100F70002060204609688847204610BD340F0008CD
:100F800020225C3013F069BFF0B58468A30800220A
:100F900004F0030407E000F15C0555F8226035BA5F
:100FA00041F82250521C9A42F5D300220BE000F186
:100FB0005C0502EB830755F82360D500C5F11805E1
:100FC000EE40CE55521CA242F1D3F0BD30B5C468FC
:100FD00003690022E31AD5188C5C0544521C082AC8
:100FE0002C77F8D330BD0360C1600261704738B51B
:100FF000044615460022626023685A689047002024
:101000006061A061A5604FF4003032BD81604FF493
:10101000003070472DE9F84304462079D4F80C805D
:10102000450748BF244845D466691D46A8F101001C
:1010300000EAD60306EBC506B6EBC50F666102D221
:10104000A669761CA6611746A66906EB5576A661C9
:101050000E46E918884225D2A8EB03094A463146D4
:10106000F81813F0FAFE2268136839460FE042467A
:10107000384613F0F2FE23681A6839462046904736
:1010800007E0311811F00300F1D1226813682046FF
:101090009847484600EB0809A9F10101A942F0D39D
:1010A000002300E000202A1A3118F81813F0D5FEAA
:1010B0004FF40030BDE8F283040002002DE9FC4F3C
:1010C000024685B0D0681369DFF86CC1DFF86C8127
:1010D000A0EB030A506840F004005060002703A80A
:1010E00002900DF10C0ED8E9003403A8544DC0E96C
:1010F00000342878534D00280CBF00230423994660
:101100005CF803305EF80940234401261D601C682A
:101110009E60DCF80430039DDCF80090DEF804608B
:101120005D406540484C654089EA0606474C66408C
:101130007519474C6540D8E9006B03AC0028C4E939
:10114000006B0EBF002404200424029E5CF8000003
:10115000345920183F4C04600126046886600398C7
:10116000029E43406340384C7068634089EA000047
:10117000364C6040034438484340280018BF0120E3
:101180005B1E9B41042F2CBFC0B2D80F02F1140389
:1011900053F8200007F00303C3F10303DB00D8403A
:1011A0000DF807007F1C082F9DD315460C466A6971
:1011B000AB69E868D20842EA4372401E00EA0207BF
:1011C000002302409B420AD8524508D28020E055B5
:1011D0007F1C574516D2AAEB0701E01910E08020CA
:1011E000E05500E0E355E8687F1C8742FAD32A689F
:1011F000136828469847BAF1000F03D0514620469D
:1012000013F02DFE2A68069E059F936869462846BE
:1012100098472A68D2F8009021462846C8472B688C
:10122000DA683946284690470EB1A86830604FF416
:10123000003007B0BDE8F08F406D01085C12000877
:10124000A00A00205FC5109304850012FC68017A93
:10125000C0F524FF24AF33D426AF698B04B001015D
:1012600000170145F8B501240094002300240DE087
:10127000009D065D0F5D7E40F643761CF60F86F0FE
:10128000010635400095641C009DEB189442EFD395
:101290001846F2BDF8B5002301240094002A11E09D
:1012A000009C85188F1815F8016C17F8015C6E40CA
:1012B000F643761CF60F86F0010634400094009C3D
:1012C000E318521EECD11846F2BD0000651200086A
:1012D00095120008010000002DE9F84F1D46DDF8C9
:1012E00028900B9F0D9C4FF0FF3300930E469246C3
:1012F000D9F800B0804632465146D847834664B399
:10130000D9F8043032465146404698476FEA0B02FE
:10131000521C42EA0B0200996FEAD2735B1C19401F
:10132000C2430091521C024300996FEAD2735B1CC6
:101330001940009186F05531484087EA000181F05C
:101340005531216080F05531C943491C0843009A4A
:101350006FEAD070401C82430092D9F8080001283F
:1013600009D17540E943491C0D4300986FEAD572D5
:10137000521C90430AE0F11C85EA9102D243521CB0
:10138000154300986FEAD5735B1C984386F0AA3624
:10139000009086EA0B0686F0AA33F243DB430C98F2
:1013A000C2F3C0725B1C42EAD3720099D243521C52
:1013B00091430091774000998843009987F0AA37BC
:1013C0000F403843BDE8F28F00000000000000002D
:1013D00001F0FF01102A2BDB10F0070F08D010F8E6
:1013E000013B013A8B422DD010F0070F42B3F6D1EA
:1013F000F0B441EA012141EA014122F007047FF003
:1014000000070023F0E80256083C85EA010586EA59
:10141000010685FA47F5A3FA87F586FA47F6A5FA95
:1014200087F68EB9EED1F0BC01F0FF0102F00702A1
:1014300032B110F8013B013A83EA010313B1F8D14C
:101440000020704701387047002D06BF354603382D
:10145000073815F0010F07D1013015F4807F02BF66
:10146000013015F4C03F0130F0BC0138704700BFB7
:10147000034613F8012B002AFBD1181A01387047D4
:1014800081F0004102E000BF83F0004330B54FEA35
:1014900041044FEA430594EA050F08BF90EA020FA2
:1014A0001FBF54EA000C55EA020C7FEA645C7FEA35
:1014B000655C00F0E2804FEA5454D4EB5555B8BF58
:1014C0006D420CDD2C4480EA020281EA030382EAC9
:1014D000000083EA010180EA020281EA0303362D5B
:1014E00088BF30BD11F0004F4FEA01314FF4801C2E
:1014F0004CEA113102D0404261EB410113F0004F40
:101500004FEA03334CEA133302D0524263EB4303F6
:1015100094EA050F00F0A780A4F10104D5F1200E94
:101520000DDB02FA0EFC22FA05F2801841F10001EF
:1015300003FA0EF2801843FA05F359410EE0A5F1C3
:1015400020050EF1200E012A03FA0EFC28BF4CF0F4
:10155000020C43FA05F3C01851EBE37101F00045AA
:1015600007D54FF0000EDCF1000C7EEB00006EEBB7
:101570000101B1F5801F1BD3B1F5001F0CD3490841
:101580005FEA30004FEA3C0C04F101044FEA445298
:1015900012F5800F80F09A80BCF1004F08BF5FEA1F
:1015A000500C50F1000041EB045141EA050130BDFF
:1015B0005FEA4C0C404141EB0101013C28BFB1F511
:1015C000801FE9D291F0000F04BF01460020B1FA5C
:1015D00081F308BF2033A3F10B03B3F120020CDA2F
:1015E0000C3208DD02F1140CC2F10C0201FA0CF00D
:1015F00021FA02F10CE002F11402D8BFC2F1200C72
:1016000001FA02F120FA0CFCDCBF41EA0C01904027
:10161000E41AA2BF01EB0451294330BD6FEA040470
:101620001F3C1CDA0C340EDC04F11404C4F120025B
:1016300020FA04F001FA02F340EA030021FA04F36D
:1016400045EA030130BDC4F10C04C4F1200220FAC4
:1016500002F001FA04F340EA0300294630BD21FA02
:1016600004F0294630BD94F0000F83F4801306BFC8
:1016700081F480110134013D4EE77FEA645C18BFBC
:101680007FEA655C29D094EA050F08BF90EA020F53
:1016900005D054EA000C04BF1946104630BD91EA4B
:1016A000030F1EBF0021002030BD5FEA545C05D14E
:1016B0004000494128BF41F0004130BD14F580048D
:1016C0003CBF01F5801130BD01F0004545F0FE4101
:1016D00041F470014FF0000030BD7FEA645C1ABF36
:1016E000194610467FEA655C1CBF0B46024650EA6D
:1016F000013406BF52EA033591EA030F41F4002199
:1017000030BD00BF90F0000F04BF0021704730B51E
:101710004FF4806404F132044FF000054FF00001F3
:1017200050E700BF90F0000F04BF0021704730B5B4
:101730004FF4806404F1320410F0004548BF404289
:101740004FF000013EE700BF42004FEAE2014FEADE
:1017500031014FEA02701FBF12F07F4393F07F4FB9
:1017600081F06051704732F07F4208BF704793F0BC
:101770007F4F04BF41F40021704730B54FF46074CF
:1017800001F0004521F000411CE700BF50EA0102D2
:1017900008BF704730B54FF000050AE050EA01027B
:1017A00008BF704730B511F0004502D5404261EBEB
:1017B00041014FF4806404F132045FEA915C3FF42C
:1017C000D8AE4FF003025FEADC0C18BF03325FEAC9
:1017D000DC0C18BF033202EBDC02C2F1200300FA7A
:1017E00003FC20FA02F001FA03FE40EA0E0021FA9F
:1017F00002F11444BDE600BF70B54FF0FF0C4CF48D
:10180000E06C1CEA11541DBF1CEA135594EA0C0F3E
:1018100095EA0C0F00F0DEF82C4481EA030621EA79
:101820004C5123EA4C5350EA013518BF52EA0335B4
:1018300041F4801143F4801338D0A0FB02CE4FF066
:101840000005E1FB02E506F00042E0FB03E54FF096
:101850000006E1FB03569CF0000F18BF4EF0010E8E
:10186000A4F1FF04B6F5007F64F5407404D25FEA8A
:101870004E0E6D4146EB060642EAC62141EA55513D
:101880004FEAC52040EA5E504FEACE2EB4F1FD0C7F
:1018900088BFBCF5E06F1ED8BEF1004F08BF5FEAFD
:1018A000500E50F1000041EB045170BD06F00046AF
:1018B00046EA010140EA020081EA0301B4EB5C045C
:1018C000C2BFD4EB0C0541EA045170BD41F4801154
:1018D0004FF0000E013C00F3AB8014F1360FDEBF79
:1018E000002001F0004170BDC4F10004203C35DA55
:1018F0000C341BDC04F11404C4F1200500FA05F3D8
:1019000020FA04F001FA05F240EA020001F0004278
:1019100021F0004110EBD37021FA04F642EB0601EE
:101920005EEA430E08BF20EAD37070BDC4F10C0418
:10193000C4F1200500FA04F320FA05F001FA04F2DC
:1019400040EA020001F0004110EBD37041F10001C8
:101950005EEA430E08BF20EAD37070BDC4F12005D3
:1019600000FA05F24EEA020E20FA04F301FA05F23B
:1019700043EA020321FA04F001F0004121FA04F2E3
:1019800020EA020000EBD3705EEA430E08BF20EAB3
:10199000D37070BD94F0000F0FD101F000464000ED
:1019A00041EB010111F4801F08BF013CF7D041EA6F
:1019B000060195F0000F18BF704703F00046520073
:1019C00043EB030313F4801F08BF013DF7D043EA44
:1019D0000603704794EA0C0F0CEA135518BF95EAFA
:1019E0000C0F0CD050EA410618BF52EA4306D1D181
:1019F00081EA030101F000414FF0000070BD50EAA0
:101A0000410606BF1046194652EA430619D094EA29
:101A10000C0F02D150EA013613D195EA0C0F05D113
:101A200052EA03361CBF104619460AD181EA030167
:101A300001F0004141F0FE4141F470014FF000001F
:101A400070BD41F0FE4141F4780170BD70B54FF0BA
:101A5000FF0C4CF4E06C1CEA11541DBF1CEA13553A
:101A600094EA0C0F95EA0C0F00F0A7F8A4EB05041C
:101A700081EA030E52EA03354FEA013100F0888013
:101A80004FEA03334FF0805545EA131343EA1263DC
:101A90004FEA022245EA111545EA10654FEA002691
:101AA0000EF000419D4208BF964244F1FD0404F54A
:101AB000407402D25B084FEA3202B61A65EB0305A6
:101AC0005B084FEA32024FF480104FF4002CB6EB63
:101AD000020E75EB030E22BFB61A754640EA0C00E3
:101AE0005B084FEA3202B6EB020E75EB030E22BF23
:101AF000B61A754640EA5C005B084FEA3202B6EB64
:101B0000020E75EB030E22BFB61A754640EA9C0022
:101B10005B084FEA3202B6EB020E75EB030E22BFF2
:101B2000B61A754640EADC0055EA060E18D04FEAB0
:101B3000051545EA16754FEA06164FEAC30343EA50
:101B400052734FEAC2025FEA1C1CC0D111F4801F1D
:101B50000BD141EA00014FF000004FF0004CB6E716
:101B600011F4801F04BF01430020B4F1FD0C88BFB5
:101B7000BCF5E06F3FF6AFAEB5EB030C04BFB6EBC0
:101B8000020C5FEA500C50F1000041EB045170BDB3
:101B90000EF0004E4EEA113114EB5C04C2BFD4EBE0
:101BA0000C0541EA045170BD41F480114FF0000E64
:101BB000013C90E645EA060E8DE60CEA135594EAE0
:101BC0000C0F08BF95EA0C0F3FF43BAF94EA0C0FE3
:101BD0000AD150EA01347FF434AF95EA0C0F7FF458
:101BE00025AF104619462CE795EA0C0F06D152EAAC
:101BF00003353FF4FDAE1046194622E750EA410690
:101C000018BF52EA43067FF4C5AE50EA41047FF4A0
:101C10000DAF52EA43057FF4EBAE12E74FF0FF3C05
:101C200006E000BF4FF0010C02E000BF4FF0010CD6
:101C30004DF804CD4FEA410C7FEA6C5C4FEA430C4F
:101C400018BF7FEA6C5C1BD001B050EA410C0CBF9E
:101C500052EA430C91EA030F02BF90EA020F002000
:101C6000704710F1000F91EA030F58BF994208BF67
:101C700090422CBFD8176FEAE37040F00100704724
:101C80004FEA410C7FEA6C5C02D150EA013C07D17B
:101C90004FEA430C7FEA6C5CD6D152EA033CD3D0C6
:101CA0005DF8040B704700BF8446104662468C46C0
:101CB0001946634600E000BF01B5FFF7B7FF0028F3
:101CC00048BF10F1000F01BD4DF808EDFFF7F4FF1C
:101CD0000CBF012000205DF808FB00BF4DF808EDA7
:101CE000FFF7EAFF34BF012000205DF808FB00BFCA
:101CF0004DF808EDFFF7E0FF94BF012000205DF8EC
:101D000008FB00BF4DF808EDFFF7CEFF94BF0120A0
:101D100000205DF808FB00BF4DF808EDFFF7C4FF99
:101D200034BF012000205DF808FB00BF4FEA410CE2
:101D30007FEA6C5C02D150EA013C0AD14FEA430CC5
:101D40007FEA6C5C02D152EA033C02D14FF0000002
:101D500070474FF0010070474FEA410212F5001240
:101D600015D211D56FF47873B3EB625212D94FEAE2
:101D7000C12343F0004343EA505311F0004F23FACC
:101D800002F018BF404270474FF00000704750EA21
:101D9000013005D111F0004008BF6FF000407047DE
:101DA0004FF00000704700BF80F0004002E000BF2D
:101DB00081F0004142001FBF5FEA410392EA030F36
:101DC0007FEA226C7FEA236C6AD04FEA1262D2EB80
:101DD0001363C1BFD218414048404140B8BF5B4285
:101DE000192B88BF704710F0004F40F4000020F01E
:101DF0007F4018BF404211F0004F41F4000121F034
:101E00007F4118BF494292EA030F3FD0A2F101027D
:101E100041FA03FC10EB0C00C3F1200301FA03F1BB
:101E200000F0004302D5494260EB4000B0F5000FDE
:101E300013D3B0F1807F06D340084FEA310102F19D
:101E40000102FE2A51D2B1F1004F40EBC25008BF4F
:101E500020F0010040EA03007047490040EB000019
:101E6000013A28BFB0F5000FEDD2B0FA80FCACF11A
:101E7000080CB2EB0C0200FA0CF0AABF00EBC25047
:101E800052421843BCBFD0401843704792F0000F35
:101E900081F4000106BF80F400000132013BB5E788
:101EA0004FEA41037FEA226C18BF7FEA236C21D0FE
:101EB00092EA030F04D092F0000F08BF0846704763
:101EC00090EA010F1CBF0020704712F07F4F04D131
:101ED000400028BF40F00040704712F100723CBF44
:101EE00000F50000704700F0004343F0FE4040F46E
:101EF000000070477FEA226216BF08467FEA23632C
:101F00000146420206BF5FEA412390EA010F40F416
:101F1000800070474FF0000304E000BF10F0004362
:101F200048BF40425FEA000C08BF704743F0964349
:101F300001464FF000001CE050EA010208BF704764
:101F40004FF000030AE000BF50EA010208BF7047EB
:101F500011F0004302D5404261EB41015FEA010C00
:101F600002BF84460146002043F0B64308BFA3F1F8
:101F70008053A3F50003BCFA8CF2083AA3EBC253DA
:101F800010DB01FA02FC634400FA02FCC2F12002F9
:101F9000BCF1004F20FA02F243EB020008BF20F030
:101FA0000100704702F1200201FA02FCC2F1200296
:101FB00050EA4C0021FA02F243EB020008BF20EA8B
:101FC000DC7070474FEA4002B2F1FE4F0FD34FF082
:101FD0009E03B3EB12620DD94FEA002343F0004396
:101FE00010F0004F23FA02F018BF404270474FF044
:101FF0000000704712F1610F01D1420205D110F0CB
:10200000004008BF6FF0004070474FF0000070477D
:1020100053B94AB9002908BF00281CBF4FF0FF314F
:102020004FF0FF3000F06AB9ADF1080C6DE904CE55
:1020300000F006F8DDF804E0DDE9022304B07047A3
:102040002DE9F047089D0C46002B4ED194468C4557
:102050008646B2FA82F262D94AB1C2F120039140B7
:1020600020FA03F30CFA02FC194300FA02FE4FEACD
:102070001C471FFA8CF6B1FBF7F44FEA1E4307FB2F
:10208000141143EA014304FB06F199420AD91CEBFF
:10209000030304F1FF3080F01281994240F20F8176
:1020A000023C6344591A1FFA8EF3B1FBF7F007FBA9
:1020B000101143EA014300FB06F69E420AD91CEBCD
:1020C000030300F1FF3180F0FC809E4240F2F98072
:1020D000634402389B1B40EA044000211DB1D340F9
:1020E0000022C5E90032BDE8F0878B4205D90DB169
:1020F000C5E9000100210846F5E7B3FA83F100299C
:1021000046D1A34202D39042C0F0F080861A64EB1D
:1021100003030120002DE6D0C5E90063E3E7002AB0
:1021200040F09080A1EB0C044FEA1C481FFA8CF79A
:102130000121B4FBF8F64FEA1E4308FB164443EABC
:10214000044307FB06F0984208D91CEB030306F191
:10215000FF3402D2984200F2CD8026461C1A1FFAA4
:102160008EF3B4FBF8F008FB104443EA044300FB91
:1021700007F79F4208D91CEB030300F1FF3402D29A
:102180009F4200F2B0802046DB1B40EA0640A5E7F4
:10219000C1F120068B4022FA06F71F4320FA06FC05
:1021A00004FA01F343EA0C03F44000FA01F8380C96
:1021B0004FEA1349B4FBF0FE1FFA87FC00FB1E44F4
:1021C00049EA04440EFB0CF9A14502FA01F20AD9CE
:1021D0003C190EF1FF3A80F08480A14540F28180E5
:1021E000AEF1020E3C44A4EB09041FFA83F9B4FBE0
:1021F000F0F300FB134449EA044403FB0CFCA44540
:1022000007D93C1903F1FF3067D2A44565D9023BD9
:102210003C4443EA0E40A0FB0293A4EB0C049C4216
:10222000CE469C4651D34ED055B1B8EB0E0364EB6D
:102230000C0404FA06F6CB401E43CC40C5E900640A
:10224000002150E7C2F1200320FA03F10CFA02FC4E
:1022500024FA03F394400C434FEA1C4800FA02FEB0
:102260001FFA8CF7B3FBF8F008FB1031230C43EA9C
:10227000014300FB07F1994208D91CEB030300F16D
:10228000FF362CD299422AD9023863445B1AA4B291
:10229000B3FBF8F108FB113344EA034401FB07F3F5
:1022A000A34208D91CEB040401F1FF3613D2A34268
:1022B00011D902396444E41A41EA004139E704467D
:1022C000F0E6084606E7C845AED2B9EB020E63EB6E
:1022D000070C0138A8E73146EDE7034699E7304699
:1022E000D4E7D6467FE7634402384DE706462346E7
:1022F00008460FE7023E634430E700BF704700BF67
:102300001348144A08B54FF00043C0E900230422E3
:10231000426101220023C2614FF480510722C0E9CB
:102320000233C0E90933C0E90C12036103838376E9
:1023300080F8203080F82C30826380F83C30C36411
:1023400004F032FF18B1BDE8084000F0E5BB08BD5D
:10235000A40A0020002401400268084B9A4282B07F
:102360000AD14FF0B0431A6E42F400721A661B6E27
:1023700003F400730193019B02B0704700240140F5
:102380000268054B9A4201BF4FF0B042136E23F42E
:1023900000731366704700BF0024014030B585B05C
:1023A00000240546CDE901440394FFF7A9FF144832
:1023B00005F08EFA08B100F0AFFB1148039401A9B3
:1023C000CDE9015405F04EF808B100F0A5FB0C482A
:1023D00005F0A8F908B100F09FFB4FF0FF31084865
:1023E00004F0E2FF064805F055FA054805F036F816
:1023F0000446034805F0F8F9204605B030BD00BF9B
:10240000A40A0020014B024A1A607047A40A002067
:102410000024014008B50948FFF7C0FF68B1084B28
:10242000B3F8AA304FF6FF72934216BF40F6E4426B
:10243000044B5343B3FBF0F398B208BD002000B443
:102440000075FF1FD8084C0013B50023ADF8063007
:10245000FFF7E0FF04461948FFF7A0FF184BB3F859
:10246000C820B3F8A8108A4204FB00F018D040F648
:10247000E443B0FBF3F364205B1A4343521A93FB2B
:10248000F2F31E331BB2ADF80630BDF806305BB276
:102490001B02ADF80630BDF8060000B202B010BD58
:1024A0004FF47A7240F6FF73B0FBF3F35343A3F596
:1024B0003923A3F50C6340F6C412E0E7001000B026
:1024C0000075FF1F4FF0B04382B09A6A22F4805229
:1024D0009A629A6C42F480529A649B6C03F4805323
:1024E0000193019B002002B070474FF0B04382B0CF
:1024F0009A6C02439A649B6C03400193019B02B067
:10250000704708B50420FFF7F0FF0120FFF7EDFF4B
:102510000220FFF7EAFF002211460E2005F076FAAE
:102520000E2005F0A5FA002211460F2005F06EFAE4
:102530000F2005F09DFA00221120114605F066FAE1
:10254000BDE80840112005F093BA000008B505F079
:10255000D3FC10B16FF0040008BD064B9A6942F03D
:1025600040429A614CF2FA321A6105F0D7FC002819
:10257000F2D0EFE700400058F0B585B000230D46DB
:1025800000930646A8B3FFF7E1FF044670BB05F0D1
:10259000B3FC88BB1A481B4A02230193D0F8E0150C
:1025A00006F1784302EA8121B3FBF1F701FB17330F
:1025B000DB0A0293D0F8E00505F178410139314496
:1025C00002EA8022B1FBF2F002FB1011C3EBD1232F
:1025D0000133694601A8039305F020FD20B10228CC
:1025E00014BF6FF00104012405F098FC204605B0EB
:1025F000F0BD6FF00504F9E76FF00404F6E700BFE3
:102600000070FF1F00FCFF03014B186000207047A3
:10261000080B00202DE9F04FB0F1006F89B006469D
:102620000F469046C0F0C080DFF89091644DD9F815
:10263000E03505EA832303F10063013B984200F291
:10264000B380002900F0B38040EA02035B0740F04A
:10265000AE80FFF77BFF044690BB05F04DFC0028E1
:1026600040F0A880D9F8E015009705EA812106F12D
:102670007842B2FBF1F301FB132208F17843013BEE
:102680003344B3FBF1F001FB1033DB0A01334FEAB3
:10269000D22AA3EBD222012A039388BFC6F30A05EC
:1026A0000AF58037C6F108038CBFC5F500654546BD
:1026B000FF02B3460693039B9A4505D305F02EFC13
:1026C000204609B0BDE8F08FA6F10803069A1A4427
:1026D00095421CD8009B04950193CDF814B04FF09F
:1026E0000009059B09EB0301049B99453DD3009B21
:1026F000AB442B44A8EB0505B5F5006F009328BF4C
:102700004FF400650AF1010A07F50067D3E753F8B3
:10271000081F5A68B2F1FF3F08BFB1F1FF3FD5D0A3
:10272000284B186810B96FF00504C7E727B14FF4BC
:102730000062394611F070F9DFF888900099D9F8F5
:102740000030CBF30A001844AAB211F065F94FF437
:1027500000613846FFF710FF00BBD9F80030019345
:102760004FF4006305970493B9E7019B07914B442D
:1027700002930120D3E9002305F00AFC88B90799E8
:10278000019BD1E9000259F80310029B5B689A4251
:1027900008BF884205D109F10809A2E76FF00104DA
:1027A0008CE76FF0030489E74FF0FF3488E76FF0A0
:1027B000050485E76FF0040482E700BF0070FF1F87
:1027C00000FCFF03080B0020B1F1006F70B510D3BF
:1027D0000B4BD3F8E0650B4B03EA862303F1006350
:1027E000013B994205D838B192B211F015F9002099
:1027F00070BD4FF0FF30FBE76FF00500F8E700BF5A
:102800000070FF1F00FCFF03B0F1006F10B40DD388
:10281000084BD3F8E045084B03EA842303F1006337
:10282000013B984202D810BCFFF7A6BE4FF0FF3024
:1028300010BC70470070FF1F00FCFF034FF0B04357
:1028400082B0DA6C0243DA64DB6C03400193019BD3
:1028500002B0704770B5012086B00024CDE9044471
:10286000FFF7ECFF0220FFF7E9FF2B4E0420FFF7F4
:10287000E5FF0DEB00014FF6FF7203234FF0904090
:10288000CDE90123039405F017FC01A9304605F0BA
:1028900013FC01A9214805F00FFC4FF0B0424FF4A2
:1028A0000071D36C23F00403D3644FF090400122F5
:1028B00005F028FD01254FF4441301A94FF0904085
:1028C000CDE90153039505F0F7FB4FF404130821FC
:1028D000CDE90113304601A9039405F0EDFB4FF457
:1028E000007301A94FF09040CDE90135CDE90354C3
:1028F00005F0E2FB22462146062005F087F8062077
:1029000005F0B6F822462146092005F07FF8092097
:1029100005F0AEF806B070BD00040048000800489D
:1029200008B51248124A134BC0E9002300230122C4
:10293000C0E90232C0E90433C0E90633036205F09E
:1029400055FE08B100F0E8F80848002105F0CEFF78
:1029500008B100F0E1F80548002105F0EDFF18B1DD
:10296000BDE8084000F0D8B808BD00BFCC0B00207F
:10297000005800405D3E302070B596B005461422E8
:10298000002103A812F0E1F93822002108A812F072
:10299000DCF92A68304B9A425BD18023089308A85F
:1029A0004FF440230E9306F023FD08B100F0B4F875
:1029B0004FF0B0444FF4C050E36C43F00103E364C4
:1029C000E36C03F001030293029B12230026CDE97E
:1029D00003030323CDE905634FF09040042303A9CB
:1029E000079305F069FBA36DDFF870C043F4800323
:1029F000A365A36D1A4C03F480030193019B266227
:102A00000D23C4E900C320468023C4E90266C4E95B
:102A10000436C4E9066605F08BF808B100F07CF8CE
:102A2000104AEC63A562104C0E23C4E90023102168
:102A3000002380222046C4E90213C4E90423C4E928
:102A40000633236205F074F808B100F065F8AC6352
:102A5000A56216B070BD00BF00580040440002409F
:102A60006C0B0020580002400C0B002000B59BB0FE
:102A70004822002108A812F068F91822002102A8B3
:102A800012F063F905F07EFF4FF0B0420120D2F85A
:102A9000903023F01803C2F89030D2F8003423F4B9
:102AA000C06343F40073C2F80034D2F8003403F476
:102AB000C0630193019B2423089381230B9300237C
:102AC000CDE91003B02208A8CDE9122306F0D2F810
:102AD00008B172B6FEE74F23CDE90230CDE904001C
:102AE000CDE90600022102A806F05EFB08B172B62D
:102AF000FEE71BB05DF804FB08B504F01BFBFFF715
:102B0000B5FFFFF7A7FEFFF7FCFCFFF709FF00F09A
:102B100092FD00F097FDFCE772B6FEE70F4808B59E
:102B20000F4B03601F2383604FF080420023C0E9F6
:102B30000433C0E9072383614FF48073436206F0D6
:102B4000D9FD08B1FFF7E8FF044806F0FFFE18B111
:102B5000BDE80840FFF7E0BF08BD00BF200C002023
:102B60000028004010B5044690B03822002102A889
:102B700012F0EBF82268194B9A422CD14FF48033B3
:102B8000029302A84FF480730F9306F031FC08B152
:102B9000FFF7C2FF4FF0B0430220D3F8902042F479
:102BA0000042C3F890209A6D42F480629A659B6D52
:102BB000002203F4806311460193019B04F026FF79
:102BC000022004F055FF00222A20114604F01EFFC7
:102BD0002A2004F04DFF10B010BD00BF00280040B7
:102BE0007047000008B500224FF6FF714FF090408B
:102BF00005F088FB074800224FF6FF7105F082FBC5
:102C000004F0AEFA044B0120C3F88800BDE8084088
:102C100005F010BF000400480004005804F0A7BAF3
:102C200008B504F0A4FA00F039FCFFF713FEFFF733
:102C300068FCBDE80840FFF773BE08B504F090FAE1
:102C4000BDE808400121002005F0A4BE7047704790
:102C5000FEE7FEE7FEE7FEE7FEE7704770477047D6
:102C600070470000014806F097BE00BF200C00200E
:102C7000012005F04DBB704770470000014805F08A
:102C8000CDB800BF6C0B0020014805F0C7B800BFED
:102C90000C0B002070470000014805F0BFB800BFD2
:102CA000A00C0020082005F033BB70477047704728
:102CB000014807F033BA00BF000D0020014806F0BC
:102CC0009FBC00BF200C0020014807F08EB800BF59
:102CD000840C00202DE9F04389B080460020109E2E
:102CE0000790894615461F46FDF7A2FAF0B9104C29
:102CF000CDE90090CDE9020407AB0E4805931423FB
:102D000004933A46434629460068FDF75BFB234699
:102D1000324604F1140153F8044B42F8044B8B4241
:102D2000F9D1079B337509B0BDE8F0830120FAE7BC
:102D30006E0C00203C6D01081FB50E4C00233C2298
:102D400002A8CDE902336275237500F0B7F80423B9
:102D500003AA009412210848FFF7BCFF0749142278
:102D6000204611F0E2FFB0FA80F35B09637504B00E
:102D700010BD00BF580C0020646D0108B10F002089
:102D8000054808B50823036006F04CFE18B1BDE8FD
:102D90000840FFF7C1BE08BD840C00204FF0B043CF
:102DA00007B55A6E42F001025A665B6E002203F0CC
:102DB0000103019311463220019B04F027FE3220CB
:102DC00003B05DF804EB04F053BE00000CB407B58B
:102DD000054A05AB1021019311F028F903B05DF805
:102DE00004EB02B0704700BF766D010830B585B0C6
:102DF000044602A80D4610F045FFBDF90C30064A06
:102E000000931021029B2046FFF7E0FF2046FEF7CB
:102E10002FFB288005B030BD766D01084FF0B04221
:102E200010B5936823F40043936010F0B3FF0D4B8B
:102E300001241C7010F080FC0B4810F097FC0B4B29
:102E40004FF400421A61002010F096FCFFF7DAFA06
:102E500000F0B4F810F08AFD21462046BDE810408D
:102E600010F0A4BD900C0020ED2D0008004000588B
:102E700010F0B2BD08B5FFF7CDFA40F6B83398426E
:102E80000CD8B0F5E16F0BD3FE23A0F5E1605843F9
:102E90004FF49663B0FBF3F0C0B208BDFE20FCE730
:102EA0000020FAE77FB5684600F06CF80198FFF75C
:102EB00089F800B207B05DF804FB0000194A38B584
:102EC000D2F88035591C044619D104F057F905464B
:102ED00004F060F9054404F057F92B0EE3712B0C54
:102EE000A3712B0A6371030EE370C0F30742C0F3B2
:102EF00007232571C0B2A2706370207038BD190A13
:102F0000C3718171190C1B0E41710371D2F88435A4
:102F1000C370D2F88405C0F30722C0F30743000E44
:102F2000E9E700BF0070FF1F38B5094BD3F88035C3
:102F300003600133054609D104F020F9044604F08A
:102F400023F9444004F026F944402C6038BD00BF0A
:102F50000070FF1F0121022010F012BD002102208D
:102F600010F00EBD00207047024B187808B100F039
:102F7000B5B87047900C002082B00190019802B063
:102F800000F048B910B50446FFF75EFA074BA3609E
:102F900040F30F20FEF7C2FF054B064A2360064BA5
:102FA0006060C4E90323002010BD00BF0000484258
:102FB00000007A440D093E00AB0305000020704775
:102FC0000120704708B511F013FF162303604FF07E
:102FD000FF3008BD08B511F00BFF16230360FEE7B4
:102FE00070B50D4614460E46731B9C4201DC20460C
:102FF00070BDAFF3008006F8010BF5E770B50D4624
:1030000014460E46731B9C4201DC204670BD16F828
:10301000010B04F077F8F5E74FF0FF3070474FF4FD
:1030200000534B600020704701207047002070471C
:103030000B4A116810B5034609B90A4911601068B6
:1030400009490A4C0344091B8B4206D911F0D0FEF2
:103050000C2303604FF0FF3010BD1360FCE700BF8E
:10306000940C002010300020000001200008000017
:10307000014B1868704700BF980C00200320704770
:1030800008B501464FF47A7200238002890DFEF7DD
:10309000BFFF08BD4FF47A73A0FB0303800A40EA28
:1030A00083507047034B98689A689042FBD1C043A5
:1030B000704700BF0028004008B5FFF7F3FF014B41
:1030C000186008BD980C002008B5FFF7EBFF024B15
:1030D0001B68C01A08BD00BF980C0020024B18786E
:1030E00008B1FFF7DFBF70479C0C002010B5074BFD
:1030F000074C0122DA654FF48071204606F046FA4B
:103100004FF0FF332363002010BD00BF00280040B4
:10311000200C002002460021014806F04EBC00BFF2
:10312000200C002002460121014806F046BC00BFE9
:10313000200C002010B58CB02C220021044601A8E0
:1031400011F003FEFFF7D2FF0C4B0D481B681C4427
:103150000023089306934FF00053E44307930122A2
:103160004FF4807301A902940B9306F023FB08B17E
:10317000FFF7D2FC00200CB010BD00BF980C00205F
:10318000200C002038B50546FFF78CFF02210446CD
:10319000074806F019FCC4F309024FF47A71A2FB48
:1031A0000121920AA30A2A8043EA805038BD00BF59
:1031B000200C00200148002106F006BC200C002055
:1031C0000148012106F000BC200C0020F8B50F4D8D
:1031D0002E78CEB90E4C4FF0FF372763FFF79EFCD9
:1031E000FFF784FF4FF48071204606F0CFF92046A8
:1031F000276306F08DFB32462046022106F0DDFBF8
:10320000FFF75AFF01232B700020F8BD9C0C002013
:10321000200C0020014610B54FF47A720023800282
:10322000890DFEF7F5FE0146FFF73CFF0446FFF768
:1032300039FF031B8B4200D310BD00BFF7E710F02E
:10324000B1BE000010B5064C0221204606F0BCFBC2
:103250000221421C2046BDE8104006F0AEBB00BF74
:10326000200C00201648174A08B54FF4E133C0E996
:10327000002300230C22C0E90233C0E90523C0E982
:103280000733C0E90933036107F07FFD08B1FFF799
:1032900043FC0B48002107F0F0FE08B1FFF73CFCAF
:1032A0000748002107F009FF08B1FFF735FC044883
:1032B00007F0C3FE18B1BDE80840FFF72DBC08BDFC
:1032C000000D00200044004070B596B00646142260
:1032D000002103A811F039FD3822002108A811F0BF
:1032E00034FD32682C4B9A4253D10223089308A82C
:1032F0002A4B0A9306F07CF808B1FFF70DFC4FF05B
:10330000B04300259A6D42F400329A659A6D02F43A
:1033100000320292029ADA6C42F00102DA64DB6C4B
:1033200003F0010301930422019B0223CDE903234F
:103330000324072303A94FF09040CDE905540793D8
:1033400004F0BAFE082303A94FF09040CDE90334FE
:103350000595134C04F0B0FE124925621423C4E90C
:1033600000131023C4E9023520468023C4E9043544
:10337000C4E9065504F0DCFB08B1FFF7CDFB2520BE
:10338000F46700220221A66204F040FB252004F02D
:103390006FFB16B070BD00BF0044004004000C007D
:1033A000A00C00208000024002680C4B9A4210B52D
:1033B000044612D14FF0B0420C21936D23F4003338
:1033C00093654FF0904004F023FFE06F04F022FC7F
:1033D000BDE81040252004F059BB10BD004400405A
:1033E00008B50A460146024806F0FCFD002008BD6B
:1033F000000D002013B5114B114C18604FF4001351
:10340000009302AB13E90600204607F0BAFD2368DB
:10341000DA69D103FCD4DA695202FCD59A6808480B
:1034200042F480029A6007F0F2FD06490448012246
:1034300007F060FD002002B010BD00BF940D002019
:10344000000D00209C0D002008B5074B1860FFF709
:1034500058F8FFF707FF054AD2F8803043F00063C1
:10346000C2F88030002008BD980D002000080058E8
:1034700008B54FF0B04308489A6B42F400329A63A3
:103480009A6B22F400329A63FFF78EFF112004F04A
:10349000FDFA002008BD00BF000D002008B5074858
:1034A00007F073FC08B1FFF737FB054804F040FB59
:1034B00018B1BDE80840FFF72FBB08BD000D002084
:1034C000A00C00200268044B9A4203D1034B002059
:1034D0001B681847704700BF00440040980D00204B
:1034E00002680B4B9A4210B504460FD1094B1B687A
:1034F0002BB1D0F8902012B90748012198472046F7
:103500000549BDE81040012207F0F4BC10BD00BF22
:1035100000440040940D00209C0D00200248012230
:10352000102104F0EFBE00BF000400480248002252
:10353000102104F0E7BE00BF0004004810B50A4C9B
:1035400023780BB9E37C6BB1FFF7F6FB0038074B30
:1035500018BF0120400018701B78022B02BF002307
:103560002370E37410BD00BFB10F0020A40D002034
:1035700038B5114C2378F3B9E37CE3B90F4D2B68D0
:10358000012B07D92B68042B04D80D4A04210120F4
:1035900000F012FA2B68042B0DD9FFF7CDFB003891
:1035A000084B18BF0120400018701B78022B02BF87
:1035B00000232370E37438BDB10F0020A00D00205C
:1035C000D06D0108A40D002008B5FFF7A7FF01F09A
:1035D00021FABDE80840FFF7A9BF022801D8FFF78C
:1035E0009DBF7047022801D8FFF7A0BF70470000B9
:1035F000022808B51BD8012210210D4804F082FED4
:103600003220FFF7B9FC0A480022102104F07AFEAC
:1036100001221021064804F075FE3220FFF7ACFCB1
:10362000BDE8084002480022102104F06BBE08BD2E
:1036300000040048704708B5FFF7F0FBBDE80840FC
:1036400000F062BB4FF0FF3010F02ABA70477047AD
:1036500070470000014BD870704700BF0C0000207D
:10366000014B1874704700BF0C00002008B5022001
:10367000002110F0DDF9BDE80840014810F040BC21
:10368000140F00200021012010F0D2B910B542F231
:103690001073084C002818BF03460748236010F039
:1036A000E1FB2168044810F065FCBDE810400248C9
:1036B00010F026BC08000020140F002010B5094CA3
:1036C000206023680BB9084B2360084810F0CAFB40
:1036D0002168064810F04EFCBDE81040034810F089
:1036E0000FBC00BFB4000020A0860100A80D002080
:1036F00010B5044680B190F906306BB9094810F056
:10370000B1FB094BE2791A70084B1868FFF7D6FF36
:10371000074B1868FFF7BAFFBDE8104000210220F0
:1037200010F086B9C00D0020AE0F0020B4000020BC
:10373000080000200A460149FFF746B800F00308D8
:1037400038B50C4810F08EFB08F018F960B90A4C37
:103750000A480125257007F0A5FF2078294607F0C3
:10376000F9FC044810F0CCFBBDE83840044810F0E8
:10377000C7BB00BF140F0020700000200C00002009
:10378000FC0E002008F098B930B585B0FFF772FB49
:10379000044607F0D9FD054688B10024384810F0EA
:1037A00061FB384B36481B689C42214638BF19469E
:1037B00010F0E0FB324810F0A3FB05B030BD01462D
:1037C0004FF4807010F034F9684601F001F823B22C
:1037D00003EB4303FE2203EB4313B3FBF2F32A4A4A
:1037E0000B211170294950680978DBB28DF80C3033
:1037F00001705068457050681A2484705068012424
:10380000C47050680371224B187818B31D700C23D4
:103810001370536861F07F01197005231D491E4C18
:103820000978012988BF00235370637A33B107F008
:1038300077FD012802D1204610F014FB174B1248E7
:10384000D978002207F096FD0630A6D107F062FD78
:103850000446A3E7124B1348197811B901780029DF
:10386000DBD0002101701970536802215971BDF835
:1038700000305168180A88715168CB710823CDE770
:10388000140F00200800002000000020080E002077
:10389000AD0F0020A40D0020C00D00200C00002062
:1038A0002C0F0020AF0F002020B1037813B1024885
:1038B00010F026BB704700BFF00D002008B5104B7C
:1038C0000122002102201A7010F0B2F80D4810F009
:1038D00017FB0D4B1B788BB10C4B1A7872B9DB7C44
:1038E00063B90B4B1A68042A9EBF1A6801321A602A
:1038F0000021BDE80840102010F09AB808BD00BFB4
:10390000AD0F0020A80D0020AE0F0020B10F002049
:10391000A00D0020044B1B78022B03D100210820AE
:1039200010F086B8704700BF7000002008B508F09E
:103930002EF880B907F0F4FC01280CD1BFF34F8FAB
:103940000549064BCA6802F4E0621343CB60BFF33B
:103950004F8F00BFFDE708BD00ED00E00400FA0551
:1039600038B504460D4607484FF40061FEF74CFF9A
:1039700030B92A4621460348BDE83840FEF74ABE22
:1039800038BD00BF00F003087047704770477047AC
:10399000022807D0082808D0012809D100210220D8
:1039A00010F046B800210820FAE7024B01221A70F5
:1039B000704700BF2C10002070B505460C46164617
:1039C00007F0C2FC0346002835D000241B4810F045
:1039D00049FA1B4B19481B689C42214638BF1946BF
:1039E00010F0C8FABDE87040144810F089BA4A686F
:1039F000F05CD0540133DAB29442F8D8114B0D7018
:103A00001B78012B88BF00244C700F4C637A33B1B4
:103A100007F086FC012802D1204610F023FA0B4B58
:103A20000B48D978002207F0A5FC0630CDD107F06D
:103A300071FC0446CAE70649DDE700BF140F002009
:103A400008000020A40D0020C00D00200C00002064
:103A500000000020044B1B7823B9044A05210120F3
:103A6000FFF7AABF704700BFA40D0020D56D010865
:103A700010B5002490B03C22214601A8009411F01A
:103A800064F92F4B2022DA7219788DF800105978DA
:103A90008DF8011099788DF80210D9788DF80310FF
:103AA00019798DF8041059798DF8051099798DF8E8
:103AB0000610D9798DF80710197A8DF80810597AFF
:103AC0008DF80910997A8DF80A108DF80B2021468F
:103AD0000DF10B0258180131007B02F8010F1C296F
:103AE000F8D193F828208DF8282093F829208DF814
:103AF000292093F82A208DF82A2093F82B208DF87E
:103B00002B2093F82C206AB193F83F2052B10DF18D
:103B10002B0100229818013290F82C0001F8010FB7
:103B2000142AF7D107484FF40061FEF76DFE20B963
:103B3000044840226946FEF76DFD10B010BD00BF7D
:103B40007100002000F80308014940220FF064BF13
:103B500000F8030870B52A4D28796B794D2BC0B257
:103B600033D1C0EB001080000A2838BF0A204FF480
:103B70007A735843234BAC791860EB794D2BE4B240
:103B80002BD1C4EB0414A40095F82C301E4E63BB5B
:103B900095F83F304BBB42F21070FFF777FD30686D
:103BA000FFF78CFD2B7A194A1949DBB213706B7A37
:103BB000184ADBB213700023EA1892F82C20D2B214
:103BC000CA540133142BF7D170BD6B79482B0ABF4F
:103BD0004FF461636B795843C6E7EB79482B0ABF12
:103BE0004FF46163EB795C43CEE7FFF74FFD012CA7
:103BF00038BF01244FF47A735C433460CFE700BFD1
:103C00007100002008000020B4000020B00F002048
:103C1000B10F0020A40D002010B590B000213C226F
:103C200001A8009111F091F84022344968460FF044
:103C3000F3FE9DF800203AB99DF801001A2803D13F
:103C40009DF8021001290ED0FFF712FF2C48142214
:103C500000210FF0EBFE4FF47A70FFF78DF9FFF7BC
:103C600079FF10B010BD274B1A70587099709DF8ED
:103C70000310D9709DF8041019719DF80510597141
:103C80009DF8061099719DF80710D9719DF80810DC
:103C900019729DF8091059729DF80A1099729DF8D1
:103CA0000B1001F03F01D972D87AD1B288421BD8EB
:103CB0009DF8282083F828209DF8292083F82920C2
:103CC0009DF82A2083F82A209DF82B2083F82B20AA
:103CD0000DF12B0100229818013211F8014F80F8E4
:103CE0002C40142AF7D1BAE701F140006844194486
:103CF00010F8340C08730132D6E700BF00F803084F
:103D0000B10F0020710000201FB5002403A9204638
:103D1000039407F021FE03A9012007F01DFE384B94
:103D20003848009422464FF4FA7110F03DF8364BB3
:103D30003648009422464FF4FA7110F035F8344BAF
:103D40003448009401224FF4FA7110F02DF8204607
:103D5000FEF75AFC08B1FEF7DFFE2F4B009400225D
:103D60004FF4FA612D4810F01FF82D4A0021012070
:103D70000FF01AFF2B4A002102200FF015FF2A4AEC
:103D8000002104200FF010FF284A002108200FF026
:103D90000BFF00F0A3FB2649264807F093FD2648B9
:103DA00007F080FC1B4810F0ABF8244B002118787A
:103DB00007F0D0F922490094224B096822480022DA
:103DC0000FF0F2FF204810F09BF8FFF725FF1F4A85
:103DD000002110200FF0E8FE1D4A00214FF48070F2
:103DE0000FF0E2FE1B4B1C4819681C4B009400228C
:103DF0000FF0DAFF184810F083F804B010BD00BFD0
:103E00008D390008F00D00208F390008D80D0020F2
:103E100089390008C00D002015390008FC0E00206B
:103E2000A9B4000889370008853700084137000821
:103E300000000301240000200C000020700000207E
:103E4000080000206D360008140F002071350008AE
:103E5000C9350008B4000020A80D0020BD380008B6
:103E600010B50024A2B021467C2203A8029410F0D1
:103E70006CFF53238DF808304FF48D73ADF80A3082
:103E80000123ADF804408DF80C30FEF7F3FF00B2CB
:103E900000EB4000FE2300EB4010B0FBF3F08DF888
:103EA0000D0001A800F0AAFC072498B958238DF84A
:103EB0000E3030228021164810F047FF224602A91A
:103EC000134810F0CFFF124A21460120FFF774FD7E
:103ED00022B010BD8DF80E408DF80F0000F09AFD55
:103EE0000C4B1A6812128DF810201A688DF81120E8
:103EF0005A6812128DF812205A688DF813209A68A9
:103F00009B688DF8153012128DF814200E24D0E71E
:103F10002D0F00203010002030B50378592B91B0C0
:103F2000044640F0F481052959D84378443B162BC8
:103F300055D8DFE813F03101540021015400290164
:103F40005400540054005400880054000C015400E4
:103F5000540054009B0154005400A4005400540029
:103F6000540017008578482D11D1B64A142101203C
:103F7000FFF722FD41F28830FEF7FEFF40F6B83031
:103F8000FEF7FAFF11B0BDE83040FFF7CFBC532D6C
:103F90000ED130228021AC4810F0D7FEFFF760FF31
:103FA00041F28830FEF7E8FFA74A152101207AE0A8
:103FB000432D16D1002468468DF8004007F0EAFA38
:103FC000A14A4C2313701A2393709DF8003054704B
:103FD00001204133D07013710521FFF7EDFC11B0C2
:103FE00030BD442DFBD1984C592323705A23637064
:103FF000A57000F0DEFB2B228021601D10F0A5FED5
:1040000000232570637001251A23A370E5702571C4
:10401000FEF730FF8D49FE23B0FBF3F04B686422BE
:104020009BB2B3FBF2F3A3714B6800EB40009BB271
:1040300000EB4010B3FBF2F102FB11336071E3714E
:1040400022460821B2E78378303BDBB2092BC6D881
:104050007F49804A0B700B78DBB253727A4A59233E
:1040600013704D2353700B7801203033032193706C
:10407000FFF7A2FC11B0BDE83040FFF7F9BC85782E
:10408000482D15D1704A56231370002353701A23FC
:104090009370032313711823012053710821042303
:1040A000D0709371D17111B0BDE83040FFF784BC7E
:1040B000432D94D100213C2201A8009110F045FE2F
:1040C0006846FFF741FD644B23228021184610F01B
:1040D0003CFE9DF8002000F80C2C9DF8012000F813
:1040E0000B2C9DF8022000F80A2C9DF8032000F804
:1040F000092C9DF8042000F8082C9DF8052000F8F4
:10410000072C9DF8062000F8062C9DF8072000F8E3
:10411000052C9DF8082000F80D5C00F8042C9DF893
:104120000B509DF8092000F8032C9DF80A2000F898
:10413000022C03A92A46A0F10D0400F8015C10F03E
:1041400091FE05F10D012246C9B2012045E78078B4
:1041500039280CD83038C0B2FFF73FFA3A4A2378F2
:10416000137063785370A378937003211EE711B026
:10417000BDE83040FFF76EBC80783928F7D830387A
:10418000C0B2FFF72FFAE9E780783928EFD8303846
:10419000C0B2FFF72DFAE1E78378303BDAB2092AA3
:1041A000E5D8C0783038C2B2092AE0D82179A1F127
:1041B0004802D2B20B2ADAD8284D45FA02F2D507C6
:1041C000D5D40A224D2902FB030036D13C235843A3
:1041D0004FF47A735843224B1860224B1860FFF754
:1041E00055FA194A2378137063785370A378937043
:1041F000E378D3700521237913710120FFF7DCFBED
:10420000144B00221A701A225A7001229A70DA7026
:10421000A278303A02EB8201E278303A02EB4102B6
:10422000D2B21A7122795A710F4A1278D2B21A7226
:10423000074A1278D2B25A721CE74829C8D14FF403
:104240006163C4E7DB6D01082D0F002030100020F2
:10425000A40D0020710000203A0F0020DEF7FFFFC0
:1042600008000020B4000020B00F00208278303A0F
:10427000D3B2092B3FF67BAFC378303BD9B20929C3
:104280003FF675AF0079A0F14801C9B20B293FF69E
:104290006EAF624D45FA01F1C9073FF568AF0A21DB
:1042A0004D2801FB02332DD13C2253434FF47A7247
:1042B00053435B4A13601068FFF700FA594A2378AA
:1042C000137063785370A3789370E378D3700521EB
:1042D000237913710120FFF76FFB534B00221A70F3
:1042E0001A225A7001229A70DA70A278303A02EBE0
:1042F0008201E278303A02EB4102D2B29A7122791D
:10430000DA7191E74828D1D14FF46162CDE7502BA3
:1043100048D102297FF663AE4378303B012B3FF64C
:104320005EAE8378312B7FF45AAE0B2904D8FFF7A9
:1043300091FB00213B4A39E63B4D0234002214F840
:10434000013FA918303B0132DBB20C2A0B73F6D1C6
:10435000FFF770F9334B50221A211A70997000221E
:1043600001215A70D97003F8041FA9180132097B82
:104370000C2A01F1300103F8011FF6D100232B7044
:104380001A236B700123AB70EB70284B1B78DBB2E8
:104390002B72274B1B78DBB26B72EA72FFF768FB5C
:1043A0001121C7E7412B7FF41AAE4378432B7FF4EA
:1043B00016AE16297FF413AE1E4D421C002312F8D0
:1043C000011FE9540133142BF9D1FFF7B7F81A4B49
:1043D0005B7D012B1DD114490023EA5CC818013311
:1043E000D2B2142B80F82C20F7D1114B00221A7076
:1043F0001B78DBB24B72FFF73BFB0A4A631E153496
:1044000013F8011F02F8011BA342F9D1054A162136
:10441000CCE5074B02221A70EFE700BFDEF7FFFF83
:10442000B40000202D0F002071000020B00F0020EC
:10443000A40D0020B10F0020580C002037B5044611
:104440000D46002939D022480FF05AFD2B78A3B32E
:104450009CB36068237880B3032B0DD00B2B2ED038
:10446000022B2AD16178012927D00B0625D403B06D
:10447000BDE83040FFF750BD6378012B07D10078CD
:10448000012802D0022800D008B907F03DF8002426
:104490000DF107008DF8074007F07CF80D4A4C231A
:1044A00013701A2393709DF8073054700120413324
:1044B0000521D0701371FFF77FFA03B030BD637828
:1044C000012BFAD10378044A03F001031370F4E7D7
:1044D000D80D00202D0F0020080E0020034B0022D5
:1044E000C3E902220122C3E900227047C80F00205D
:1044F00000487047C80F00204FF0B04382B0DA6C1C
:104500000243DA64DB6C03400193019B02B0704705
:104510002DE9F04186B000240220154D0594FFF7E7
:10452000EBFF0420FFF7E8FF124F03944FF480766F
:1045300001230DEB0001CDE9016328460323049319
:104540004FF4005803F0B8FD01A93846CDF80480B7
:1045500003F0B2FD22464146384603F0D3FE28461A
:104560002246314603F0CEFE204606B0BDE8F0817B
:104570000004004800080048032810B50ED80128A0
:1045800010D868B902460B484FF4807103F0BAFEA8
:10459000002209484FF4005103F0B4FE002010BD82
:1045A0000122F0E7002203484FF4807103F0AAFED5
:1045B0000122EEE70004004800080048022070478E
:1045C0000020704701207047002814BF16200F20DC
:1045D000704700000D48854602F0AAFD0C480D49C1
:1045E0000D4A002302E0D458C4500433C4188C424E
:1045F000F9D30A4A0A4C002301E013600432A242B4
:10460000FBD310F0FBFBFEF777FAFEE7000001207A
:1046100000000020840A0020507C0108840A002049
:1046200010300020FEE74FF0B04382B0DA6C42F069
:104630000102DA64DB6C03F001030193019B02B019
:104640007047000030B587B0FFF7EDFF4FF48051A1
:1046500001224FF0904003F055FE01224FF400611B
:104660004FF0904003F04EFE4FF4C0551123CDE9BA
:10467000015301A901234FF09040039303F01CFD67
:1046800008240A2500224FF480514FF0904003F097
:1046900039FE0120FEF770FC01224FF480514FF0EB
:1046A000904003F02FFE0120FEF766FC013DE9D1AA
:1046B0004FF400614FF0904003F01EFE08B9013C3A
:1046C000DFD14FF400614FF0904003F015FE68BB5E
:1046D000FFF7A9FF04240123039001A92A48CDE98B
:1046E000014303F0E9FC284C01220421204603F099
:1046F00009FE2120FEF740FC00220421204603F0A1
:1047000001FE2120FEF738FC01220421204603F09F
:10471000F9FD2120FEF730FC20460022042103F0A1
:10472000F1FD4FF42570FEF727FCDDE7FFF77BFF77
:104730004FF0B04300249A6D42F480029A659B6D5D
:1047400003F4800300934FF4C052009B1223CDE981
:1047500001230323CDE9034304230DEB03014FF0B1
:104760009040059303F0A8FC08480949094B846070
:10477000C0E900130123C0E90334C0E907444461E0
:1047800003F034FF07B030BD00040048D80F00200C
:10479000005800401A091020FFF754BF40B94B1EC3
:1047A0005A425A414FF400714FF0904003F0AABDB5
:1047B000704708B50120FEF710FF6420FEF7DCFB10
:1047C00000F028F9BDE808400120FEF70BBF00000B
:1047D000084B1A685A6802819A68428110B51A68B3
:1047E0005C68996813190B440380034B01221A700B
:1047F00010BD00BF30100020AF0F002010B50446E0
:1048000000F008F810F0FF001FBFEE232370AA236A
:10481000637010BD2DE9F7430024304E304D3460F5
:1048200021462046FFF7BAFF21460120FFF7B6FFD9
:1048300021460220FFF7B2FF5227A046012195F83A
:10484000640185F86071C5F86881FFF7A7FF032050
:10485000FEF792FB00228821284602F0C1FB0DF1F1
:104860000602C021284602F00BFC88BBBDF80620DA
:104870004EF6AA639A422BD14FEA440909F1540932
:104880005FFA89F94946284600F034F900BB85F8FB
:1048900060910DF10602C021284602F0F1FBB8B983
:1048A000284600F0E3FA98B9326801231A443260CE
:1048B0000C4AC5F868311168A3400B4313600134FA
:1048C000032C05F5C875B9D1306803B0BDE8F08395
:1048D0000021E0B2FFF762FFF1E700BF44100020C3
:1048E000B8000020401000202DE9F74F344C054659
:1048F00004F5966B4FF00A0A4FF00E0948F2E808EB
:104900004FF490174FF48046D4F86831002B50D004
:10491000204600F09BFD0DF102020DF10101204641
:1049200000F05CFB0DF1030201A9204600F090FEAF
:104930000021204600F0E2F801220021204600F08C
:10494000A2F901221146204600F09DF9022D0ED851
:104950001C4B33F815601C4B53F825701B4B53F858
:1049600025801B4B13F805901A4B13F805A032460F
:104970000121204600F0D0F93A460021204600F0FF
:10498000CBF94146204600F0D3F84A4600212046A4
:1049900000F0D0F852460121204600F0CBF80DF18E
:1049A00002020DF10101204600F018FB0123C4F8BA
:1049B0007C3104F5C874A345A6D103B0BDE8F08FDF
:1049C000B8000020106E0108046E0108F86D01089F
:1049D000F36D0108F06D010810B50B7E9BB9D0F89E
:1049E0007C21098912B1C0E95E1310BD084BD0F8D3
:1049F00078411A68C2F580734B4304FB02331B12E3
:104A0000C0F87831F1E70123C0F87C31EDE700BF51
:104A1000680500202DE9F84FDFF8C0A0304DFFF702
:104A2000BBFEDAF800300BB12B6813B9FFF7F2FECA
:104A300028602B682B4E0024A34234607460B4605D
:104A400049DDDFF8A480294D2046FFF74DFF88F8A7
:104A50000040D5F86831012B33D1DFF894B003FA68
:104A600004F90A272249284600F050FCB0B95946FB
:104A70002846FFF7B1FF9BF818307BB9D5F878319D
:104A800046F82430DAF8003043EA0903CAF8003067
:104A900098F8003043F0010388F800300120FEF759
:104AA0006BFA9BF818301BB1013F17F0FF07D9D103
:104AB000D5F8783140F6C412002B08BF134646F8EB
:104AC000243001200134FEF757FA032C05F5C87590
:104AD000BFD198F80030BDE8F88F00BF401000202B
:104AE0003C10002030100020AF0F0020B800002044
:104AF000481000204A088A2102F072BA152906D807
:104B0000044BCB40DB0702D50174002070476FF0E7
:104B1000070070470B00300010B50A460C4609210B
:104B200002F080FA18B9237803F00103237010BD56
:104B300001F051BE01F02EBD01F033BEF7B50023E8
:104B40000F46144601210DF1070206468DF8073085
:104B500002F068FA0546D0B9012C9DF8073025D13E
:104B6000042F39D8DFE807F00316191C1F0043F0A3
:104B700010049C420BD022460121304602F030FA4C
:104B800068BB716986F830413046FFF7D1FF28468F
:104B900003B0F0BD43F02804EBE743F00404E8E77A
:104BA00043F04004E5E743F08004E2E7042F13D824
:104BB000DFE807F00306090C0F0003F0EF04D8E765
:104BC00003F0D704D5E703F0FB04D2E703F0BF04FA
:104BD000CFE703F07F04CCE76FF00305D7E7054686
:104BE000D5E713B500230C460DF1070201218DF81E
:104BF000073002F017FA78B99DF80730C3F30012B6
:104C00002270C3F3C002A270C3F380026270C3F3C8
:104C10008012DB09E270237102B010BD37B50D467A
:104C20000DF10202F821044602F02AFA70B901AA35
:104C30000421204602F042FA40B9BDF802201AB120
:104C4000019BB3FBF2F32B602B68A36103B030BD73
:104C5000037F0B700020704737B50D460DF106023B
:104C60002021044602F00CFA28B9BDF8063023B919
:104C7000236A2B60207703B030BDDB002B602362FA
:104C800001232377F7E70529F8B504460E461546B4
:104C900033D862B100EB810301215A6B0023701EEF
:104CA000042807D8DFE800F010191C1F2600114661
:104CB0000123F4E784F82810003D344418BF01258F
:104CC00084F82850002007E0C2F34F2244212046F8
:104CD00002F096F90028EFD0F8BD84F82A10EBE72F
:104CE00084F82B10E8E75B00FE226021204602F0EA
:104CF000B0F9EFE71B01EF22F7E76FF00300EBE7F6
:104D0000052996BF4018002390F82830137094BFEF
:104D100000206FF00300704770B54318044693F805
:104D200028300E4615463BB105291BD8DFE801F0B7
:104D3000030912141616426304EB8604002065630F
:104D400007E0C2F34F224421204602F059F900281F
:104D5000F2D070BDC263EFE70264EDE7C2F34F2209
:104D60006421F1E76FF00300F3E737B50446154619
:104D700005292AD8DFE801F0030614161818436B3A
:104D80002B601FE00DF10602442102F079F9D0B941
:104D9000BDF8062053028AB12B60A36301230FE004
:104DA000C36BEDE7036CEBE70DF10602642102F043
:104DB00067F940B9BDF806305B02E1E7A26B2A60F3
:104DC00084F82930002003B030BD6FF00300FAE70B
:104DD00037B50D460DF107020121044602F022F914
:104DE00038B99DF8073084F83031DB092B7084F82E
:104DF0004C3003B030BD2DE9F843037C0C4601F87C
:104E0000083B0546FFF70AFF40BB207304F1100181
:104E10002846FFF721FF08BB04F11401284600F0E3
:104E200019FCD8B904F1240705F1270904F1170882
:104E300006463A46B1B22846FFF797FF70B90136E9
:104E400019F8013F08F8013F062E07F10407F0D1D9
:104E500004F13C012846FFF7BBFF08B1BDE8F88329
:104E6000211D2846BDE8F84301F01DBDF0B5002224
:104E7000054693B0882102F0B3F84FF47A72A5F892
:104E800052214FF4C872A5F85421514AC5F858214F
:104E90000023504A85F8F030C5F8D4202B6202A9CF
:104EA0002846FFF7A8FF044670B9ADF8080002AE27
:104EB0000FCE05F110070FC70FCE0FC70FCE0FC7CC
:104EC00096E80F0087E80F00434BC5F834314FF4E4
:104ED000FA730126A5F838314FF42063A5F83C3168
:104EE0003246802185F85061284602F079F8324632
:104EF0000746FF21284602F073F8002211460743B7
:104F0000284602F06DF83C4364B204430DF10702F9
:104F10009121284602F086F864B29DF8073085F8A2
:104F20003A31044332460021284602F059F864B26F
:104F300004430022FF21284602F052F864B20443E1
:104F400000228021284602F04BF864B2204340B290
:104F500000283BD013B0F0BD0028FBD1A1B2012244
:104F600028460134FFF78FFE062CF5D10028F1D139
:104F700004466885024604212846FFF784FE00287F
:104F8000E8D1024605212846FFF77DFE0028E1D141
:104F90004FF490136B634FF4804201212846FFF7D2
:104FA000BBFE0028D6D14FF40C13FF22C5E90F3009
:104FB00085F830210121284602F012F8012385F8F6
:104FC00032310028C6D185F81541C3E70446C5E74C
:104FD000856B0100A470090064008403012300F0C4
:104FE00069BD2DE9F0428EB00C460C2304AA1421B1
:104FF000054601F0DDFF8446002860D1BDF816208B
:10500000BDF81830A075BDF81210206052BA5BBA16
:105010006060BDF81A60B5F8520192B29BB249BA0D
:105020005B0252022361A18276BAE260B0F57A7F18
:105030008BB295F831719DF81010B6B20AD070435A
:1050400000F5FA704FF47A76B0FBF6F02E7F002E62
:1050500039D186B2002F40D0B001C0B2B608E07599
:105060000DF10F002681CDE90040284601F072FEC7
:10507000844620BB9DF80FE084F818E005F1500647
:105080000FCE07AF0FC796E80700E37D87E807005C
:10509000D4E90301A28AADF83020D4E90149CDE971
:1050A0000A01CDE9084907AC8DF833308DF834E0BA
:1050B0000FCC50350FC597E8070086E8070060461B
:1050C0000EB0BDE8F0822E8C5E43B2EB262F4FEA85
:1050D000262C04D157B948F6E0260020BFE780B25D
:1050E0005043A2EB0C06B0FBF6F0B2E742F2B82652
:1050F000B2E70000F7B517460E210DF106021D4676
:105100000B4C064601F0BCFFBDF8063004EA4343F1
:105110003B6050B90DF106020C21304601F0B0FFA2
:10512000BDF8063004EA43442C6003B0F0BD00BF74
:105130000000FE1F73B590F8DA30013B022B0646E3
:105140000C4634D801AB6A460121FFF7D3FF009B20
:10515000B3F57F0F054603D8019BB3F57F0F23D925
:1051600015BB34B11349304602B0BDE8704001F0C0
:10517000FFBB0422FF21304601F032FF2A460446DD
:105180007021304601F02CFF2A460443FF213046AF
:1051900001F026FF64B204432A468021304601F024
:1051A0001FFF64B2044365B2284602B070BD0025FB
:1051B000FAE700BF6C05002037B5044601228021C4
:1051C000057C01F00DFF0122FF21204601F008FFC0
:1051D00000221146204601F003FF94F83A21912164
:1051E000204601F0FDFE01220021204601F0F8FEDC
:1051F0000022FF21204601F0F3FE002280212046FC
:1052000001F0EEFE012D24D0032D32D0C5BB0122CA
:105210002946204601F0E4FE01238DF80730B0B99D
:1052200005469DF80730DB0705F101050AD548B9A9
:10523000B5F5FA6F27D001460DF10702204601F0BF
:10524000F1FEEEE7B5F5FA6F08BF6FF0060003B0A8
:1052500030BD18B929462046FFF76CFF0222002115
:10526000204601F0BDFE0028F1D1042384F832313C
:10527000EDE718B901212046FFF75CFF0422EEE7B5
:105280006FF00700E3E76FF00600E0E738B5057C54
:10529000044625B1204600F03BFD28B138BDFFF79C
:1052A0008BFF0028F6D0F9E7002DF7D1032384F80F
:1052B0003231F3E773B50646002501220B21304653
:1052C00001F08EFE002204460B21304601F088FEDC
:1052D0000DF1070204431321304601F0A3FE9DF8AF
:1052E000073064B2044301355B0760B2EDB205D00C
:1052F000032D08D00028E0D002B070BD032D08BFF8
:105300006FF00B00F8E76FF00B00F5E738B50023FE
:10531000037404460D46FFF7B9FF50B929462046ED
:10532000FFF75FFE28B901462046BDE83840FFF789
:10533000C1BF38BD152970B5054616461C4667D154
:105340000122FF2101F04CFE0022114604462846AE
:1053500001F046FE00220443FF21284601F040FEF2
:1053600064B2044301228021284601F039FE64B270
:10537000044302228521284601F032FE64B2044330
:105380000422FF21284601F02BFE64B204430022D0
:10539000CD21284601F024FE64B204431122CC2121
:1053A000284601F01DFE64B204430722FF2128466F
:1053B00001F016FE64B204430022BE21284601F02B
:1053C0000FFE64B204430622FF21284601F008FEC6
:1053D00064B204430922CC21284601F001FE64B2E4
:1053E00004430022FF21284601F0FAFD64B2044381
:1053F0000122FF21284601F0F3FD64B2002204439C
:105400001146284601F0ECFD64B2204340B270BD65
:10541000042A17D80A2101F0E3FD0028F7D1231E42
:1054200018BF01231B01EF228421284601F011FE41
:105430000028ECD185F8DA6001462846BDE87040C6
:10544000FFF738BF6FF00A00E1E7000070B594B0D5
:1054500005464022002104A80FF077FC002301211B
:105460002846ADF806308DF803308DF804300293ED
:1054700000F0A0FC95F8142195F81311012A04D826
:1054800040F0AD80202940F2AC8001AA02A9284654
:1054900000F02BFB0446002840F09E8095F8503128
:1054A000002B40F0A280D5F84C11284601F060FA9C
:1054B0000446002840F09080034601460422284616
:1054C000FFF738FF0446002840F086800122FF21C4
:1054D000284601F085FD0DF1060206468421284686
:1054E00001F0CEFD22460643FF21284601F078FD5B
:1054F00076B2064374B2002C6ED1BDF806301B01A3
:10550000C5F8D43004A92846FFF775FC04460028E6
:1055100062D10DF103012846FFF7FEFA0446002888
:105520005AD19DF8033085F8313104AC0FCC05F128
:1055300010060FC60FCC0FC60FCC0FC694E80F0095
:1055400086E80F000DF103020121284601F06AFDF3
:105550000446002840D19DF8033085F830310246DA
:1055600001462846FFF7EAFA0446A8BB0246022194
:105570002846FFF7E3FA044670BB0323014685F88B
:1055800032310DF10502284601F00BF9044618BB33
:105590009DF8053085F8E8300DF105020121284617
:1055A00001F0FFF80446B8B99DF8053085F8E03001
:1055B00003AA0321284600F0E7FE044660B9039BD6
:1055C000C5F8E43003AA0421284600F0DDFE0446B5
:1055D00010B9039BC5F8DC30204614B070BD0C290F
:1055E00051E7284600F013F954E701495DE700BF91
:1055F0002207002013B50C460DF10702132101F01C
:1056000011FD9DF8073013F0180F03F0070218BFC3
:105610006FF00500226002B010BD13B590F8DA30CB
:10562000042B0C4609D101A9FFF7E4FF019B1A1FC7
:1056300053425341237002B010BD01AA142101F05E
:10564000F1FC0028F7D19DF8043003F00103F1E7E5
:1056500000F04BBA13B50C460DF10602282101F0FB
:105660000FFD78B9BDF80620C2F30B0312F4006FEA
:1056700018BFA3F580534FF0FA0214BF13FB02F3D7
:105680005343236002B010BDF0B54FEAD20C4FF087
:10569000FF341C6002F00702664600278E4200D2EB
:1056A00007B1F0BD845D664503BF1441E4B2154601
:1056B0003D4614F0010705D005EBC6051D60012726
:1056C0000136EBE70135082D4FEA5404F8D014F009
:1056D000010FF0E7034B800953F82000003818BF92
:1056E000012070471808002010B5B1EBD20F4FEA27
:1056F000D20402F0070381BF01229A40035D1343E5
:105700008ABF03556FF03100002010BD0A46062302
:10571000B02101F02FBC0A460623B02101F048BC9D
:105720002DE9F04F85B00546109F0E9E01978A46E1
:1057300093461C464FF00009119B994508D1002360
:10574000129A176013B36FF0310005B0BDE8F08F07
:1057500001AB3A4631465846FFF796FFDDF8048024
:10576000B8F1FF3F0FD00F9B08EB0300FFF7B2FF2C
:10577000504508D142462046FFF7B6FF08F1010721
:1057800009F10109D8E76FF03103D9E7214628462E
:10579000FFF7BCFF0028D8D102A92846FFF7BBFFBE
:1057A00002ABA2199442D0D014F8015B13F8011B8C
:1057B0008D42F7D0C7E770B5C02288B00E460121F0
:1057C00090F83051044601F00BFCF0B901A92046D5
:1057D000FFF79CFDC8B90122FF21204601F000FC23
:1057E00098B93246B621204601F04AFC68B9024613
:1057F000FF21204601F0F4FB38B92A46012120465A
:1058000001F0EEFB08B984F8305108B070BDF0B576
:105810000F4689B01646FF210122044601F0E0FB45
:105820000246A8B94F21204601F0DAFB80B92C22AC
:105830004E21204601F0D4FB024648B9FF21204604
:1058400001F0CEFB20B9B422B621204601F0C8FBFE
:105850000025C4F82451A4F82851DEB9354607AB19
:10586000B422CDE903730623CDE90032029504F595
:10587000927304F5957231462046FFF751FF30B917
:10588000012384F8153184F8137184F8146109B088
:10589000F0BD013505F1B400FFF71CFF0028DED193
:1058A0002C2DF6D1DBE710B541F0010200210446B2
:1058B00001F096FB78B9204600F02AFA58B9014663
:1058C0002046FFF7F7FC30B9024601462046BDE806
:1058D000104001F085BB10BD2DE9F74F4FF0000BD4
:1058E00088461746FF21012205461E469DF838A02E
:1058F0009DF83C908DF807B001F072FB5A460446C3
:105900005946284601F06CFB5A460443FF212846BD
:1059100001F066FB64B2044364B2B8F1000F32D008
:10592000BAF1000F06D00C9ACB21284601F07AFB81
:10593000204344B2B9F1000F07D00DF10702EE2168
:10594000284601F06FFB204344B20122FF21284684
:1059500001F046FB012204430021284601F040FBF0
:1059600064B204430022FF21284601F039FB64B2EF
:105970009DF807300D9A204323F0100340B21370B6
:1059800003B0BDE8F08FBAF1000F06D03A46CB2144
:10599000284601F025FB204344B2B9F1000FD4D0D2
:1059A00033468022EE21284601F053FBCBE72DE958
:1059B000F04387B09146002205460E468DF8172029
:1059C0001F4653B390F8308101221146284601F05A
:1059D00007FB044648BB40212846FFF764FFF0B9A7
:1059E000B9F1010F24D10DF11703CDE90294CDE9EE
:1059F00000632246234649462846FFF76DFF0446CA
:105A000078B947B142460121284601F0E9FA044637
:105A100038B985F83081002403E09846D4E7347023
:105A20000446204607B0BDE8F08300233370F8E752
:105A30003070E6E72DE9F043054687B00E46914603
:105A40001F4653B390F8308102220121284601F00D
:105A5000C7FA044648BB01462846FFF724FFF0B9C1
:105A6000B9F1010F24D10DF11703CDE902490093DB
:105A700022462346019649462846FFF72DFF044655
:105A800078B947B142460121284601F0A9FA0446F7
:105A900038B985F83081002403E09846D4E73470A3
:105AA0000446204607B0BDE8F08300233370F8E7D2
:105AB0003070E6E7F8B51D46164600232A4690F8F2
:105AC00030710446FFF773FF70B903462A4631462A
:105AD0002046FFF7AFFF38B93A460121204601F0D2
:105AE0007FFA08B984F83071F8BD2DE9F04F002332
:105AF00093B0CDE90A12C0F82431A0F82831012270
:105B0000FF21CDE90E33B0F83C818DF834300446E6
:105B10008DF8353001F064FA002840F0F08002463C
:105B20004F21204601F05CFA002840F0E8802C224A
:105B30004E21204601F054FA002840F0E080024651
:105B4000FF21204601F04CFA002840F0D880B42212
:105B5000B621204601F044FA002840F0D0800246E9
:105B60008021204601F03CFA002840F0C88003461E
:105B70000DF135020DA92046FFF79CFF002840F0EB
:105B8000BE8004F5957307930323CDE90203B42186
:105B9000062304F592790EAECDE900310496014654
:105BA0004B4604F595722046FFF7BAFD002840F0F9
:105BB000A6800DF1360120460E9DFFF7FCFD002862
:105BC00040F09D80BDF83630434541D9C4F82401EA
:105BD000A4F8280105F1B400FFF77CFD08B92B2DCE
:105BE0001FD90623B42204960326CDE90032CDE95D
:105BF0000256079A4B4601212046FFF791FD0028E7
:105C00007DD10DF1360120460E9DFFF7D4FD002811
:105C100075D1BDF83630434574D901274FF0010ADC
:105C200019E00135D6E7089E099324E0089E0A9BF7
:105C30001E600B9B1F70012384F815310A9B1B68A3
:105C400084F813310B9B1B7884F81431002056E044
:105C500000273E46BA46BDF836304345E7D2A3EBAF
:105C6000080383EAE372A2EBE3725FFA8AF7099210
:105C7000032604F5927BDBF80000BBF8043010909B
:105C8000ADF844302A460FAB07980621FFF7FCFC1D
:105C90000F9D6B1C39D005F1B400FFF71BFD50457B
:105CA000C5D1731C2A4648460893FFF71DFD30BB3B
:105CB000494620460135FFF729FD00BB0DF13601AD
:105CC0002046FFF778FDD0B9BDF83620A2EB0803D7
:105CD000002BB8BF5B424245A5D9099A9342A5D98A
:105CE00010A92046FFF712FDBDF844200346109886
:105CF000C4F82401ABF804201846002B97D013B049
:105D0000BDE8F08F0746064688E76FF03100F6E7FA
:105D100037B5002304468DF807304FF4FA650DF1CE
:105D200007012046FFF779FC58B99DF80730012B91
:105D300007D0013D03D0204601F0DEF9EFE76FF018
:105D4000060003B030BD02464FF08043934202D8B4
:105D5000002013B970479B08F8E7C11891424FEA39
:105D600050009CBFC018521A9B08F2E773B500227E
:105D70008321054601F034F9044690B906460DF139
:105D800007028321284601F04DF99DF807300343AF
:105D9000DBB204462BB90136B6F5FA6FEFD16FF0DE
:105DA000060401228321284601F01AF9204340B25B
:105DB00002B070BD2DE9F04F90F8F06091B04FF057
:105DC0000009072ECDE9079904460F4600F0A2828C
:105DD0000122802101F004F901228046FF212046A2
:105DE00001F0FEF84A4648EA00084946204601F01C
:105DF000F7F84FFA88F848EA00080622FF21204603
:105E000001F0EEF84FFA88F848EA00080DF11502A3
:105E10008321204601F006F99DF815204FFA88F8F5
:105E200048EA000842F004028321204601F0D8F835
:105E30004FFA88F848EA00080722FF21204601F0BF
:105E4000CFF84FFA88F80122812148EA000820465D
:105E500001F0C6F84FFA88F848EA0008204601F039
:105E60004BF94FFA88F848EA0008012280212046C1
:105E700001F0B6F84FFA88F848EA000517F0010B70
:105E80006DB200F01E82F20700F11E826B22942197
:105E9000204601F0A5F880462046FFF767FF06AAD6
:105EA00048EA00089021204601F008F945EA080573
:105EB000069B6DB22422942105432046C3F3062A93
:105EC000C3F3C03901F08CF86DB205432046FFF7EB
:105ED0004DFF6DB2054306AA9021204601F0EEF871
:105EE000069B6DB21BBA25229421054320460993D7
:105EF00001F076F86DB205432046FFF737FF6DB22B
:105F0000054306AA9021204601F0D8F8069B6DB201
:105F10001A0E05431B0C6DB28DF828208DF8293020
:105F200017F00203029300F0DB8016F0020840F045
:105F3000D78002229421204601F052F80190204699
:105F4000FFF714FF019B0DF1160203439021204639
:105F50001D4301F067F86DB27B2294210543204672
:105F600001F03EF86DB205432046FFF7FFFE6DB22B
:105F700005430DF117029021204601F053F86DB250
:105F8000772294210543204601F02AF86DB205439B
:105F90002046FFF7EBFE6DB2054306AA902120468E
:105FA00001F08CF8069B5A0E8DF82C20C3F3864224
:105FB0008DF82D20C3F3C6228DF82E206DB2C3F3C9
:105FC0000612DB0003F07803942105438DF82F209F
:105FD000204678228DF8153001F002F86DB20543A5
:105FE0002046FFF7C3FE6DB2054306AA9021204666
:105FF00001F064F8069B9DF8152002EB53728DF8B2
:106000003020C3F386528DF83120C3F3C6328DF8A9
:106010003220C3F306228DF833206DB2C3F346025B
:106020009B0103F04003942105438DF83420204662
:1060300079228DF8153000F0D3FF6DB2054320466C
:10604000FFF794FE6DB2054306AA9021204601F0A9
:1060500035F8069B9DF8152002EB93628DF83520EC
:10606000C3F3C6428DF83620C3F306328DF83720CD
:106070006DB2C3F346129B0003F07C0394210543E9
:106080008DF8382020467A228DF8153000F0A8FFD0
:106090006DB205432046FFF769FE6DB2054306AABF
:1060A0009021204601F00AF8069B9DF815208DF8F6
:1060B0003E8002EB93728DF83920C3F3C6526DB265
:1060C0008DF83A20C3F3064205438DF83B20C3F315
:1060D0004622C3F386036DB28DF83C208DF83D3027
:1060E00017F00403019300F0F180730700F1EE80D4
:1060F0007B229421204600F073FF80462046FFF764
:1061000035FE07AA48EA00089021204600F0D6FF95
:1061100045EA08084FFA88F848EA00057C229421ED
:10612000204600F05DFF6DB205432046FFF71EFEDE
:106130006DB2054308AA9021204600F0BFFF6DB262
:10614000732294210543204600F04AFF6DB20543B7
:106150002046FFF70BFE6DB2054306AA90212046AC
:1061600000F0ACFF069B6DB21B0274229421054324
:1061700020461FFA83F800F033FF6DB20543204636
:10618000FFF7F4FD6DB2054306AA9021204600F00A
:1061900095FF6DB29DF81B30752294210543204672
:1061A00043EA080800F01CFF6DB205432046FFF7E4
:1061B000DDFD6DB2054306AA9021204600F07EFF6A
:1061C000069B6DB21B029BB27622942105432046AA
:1061D000039300F005FF6DB205432046FFF7C6FDAF
:1061E0006DB2054306AA9021204600F067FF6DB20C
:1061F0009DF81B20039B05436DB2134300228121B0
:106200002046039300F0ECFE06220543FF212046C2
:1062100000F0E6FE6DB205430DF115028321204624
:1062200000F000FF9DF815206DB2054302F0FB025F
:106230008321204600F0D4FE6DB205430122FF21E8
:10624000204600F0CDFE6DB205430122002120461C
:1062500000F0C6FE6DB205430022FF21204600F08B
:10626000BFFE6DB2054300228021204600F0B8FE3B
:106270006DB205436DB2039BFDB9BBF1000F29D18F
:10628000029AAABB019AAAB1720713D4079AC4F85A
:106290001821089AC4F81C214FEA4822C4F820218A
:1062A0003BB1A3F5C8534FF47A7253431B095B42C9
:1062B0001BB2E3603E4384F8F060284611B0BDE8AD
:1062C000F08FD946DA462BE6CA4629E64FF0000899
:1062D000434693E7F007D3D40998BDF8282084F803
:1062E00013A184F81491C4F82A01A4F82E21C7E759
:1062F000B107C7D49DF8162084F8F1209DF8172027
:1063000084F8F2200BA904F1F30002930EF09DFD36
:10631000029BB7E74D46D0E740B101380023FF2884
:1063200003F1010203D800EB032080B2704740085C
:106330001346F4E7C3B2000A03FA00F001307047D5
:10634000084B5A434FF47A7302F5FA724FF4FA602D
:10635000B2FBF0F0B2FBF3F203FB0100B0FBF2F092
:10636000704700BF002F3A00064B5A434FF47A7033
:1063700002F5FA72B2FBF0F24A4302F5FA72B2FB8E
:10638000F0F07047002F3A002DE9FF4102294FF04D
:106390000005074616468DF80350ADF804501CD88A
:1063A0000DF102022946FEF7C7FB044630B90DF194
:1063B00003024621384600F035FE04469DF80300EE
:1063C000FFF7B8FF81B29DF802203846FFF7CCFFF7
:1063D0003060204604B0BDE8F081032918D10DF1EA
:1063E00002022946FEF7A8FB0446002846D10146D2
:1063F0000DF102023846FEF79FFB044628B901AAB8
:106400005121384600F03CFE0446BDF80400D7E7B1
:10641000042935D102A9FEF7E4FB9DF80B304BB3FC
:106420000DF1020229463846FEF786FB044618BBEA
:1064300001AA5121384600F023FE0446BDF80400AD
:10644000FFF778FF85B2BCB90DF102020121384691
:10645000FEF772FB044678B90DF106027121384649
:1064600000F00EFE0446BDF80600FFF763FF80B2A1
:10647000401BA7E71D46E7E70020F9E72846A7E706
:1064800028462C46A4E7F0B5022985B005461646F5
:106490001ED80DF105020021FEF74EFB0446A0B9FF
:1064A0009DF8052031462846FFF74AFF83B2B3F531
:1064B000807F9ABF00F1FF32D2B2FF22A5F8D82028
:1064C0004621284600F08CFD0446204605B0F0BD6C
:1064D000032920D10DF105020021FEF72DFB9DF8C7
:1064E0000520044631462846FFF72AFF80B2FFF711
:1064F00013FF0246ADF80600A5F8D800002CE4D141
:106500005121284600F07CFD04460028DDD1C5F865
:10651000E4600024D9E7042939D102A9FEF761FB20
:106520009DF80B70B7B10DF1050200212846FEF76A
:1065300003FB04460028C8D10DF10602512128466C
:1065400000F09EFD04460028BFD1BDF80600FFF70D
:10655000F1FE87B20DF1050201212846FEF7ECFAA3
:1065600004460028B1D19DF8052031462846FFF7A2
:10657000E7FE3844FFF7D0FE71210246284600F0BE
:106580003FFD04460028A0D1C5F8DC60C1E76FF0EC
:1065900003049AE7F0B585B000238DF80330D307E4
:1065A00005460F46164605D441B9A2F10C03DAB2EE
:1065B000062A12D96FF0030005B0F0BD012920D1E1
:1065C000A2F10803DAB2062AF4D8062B19D8DFE8BC
:1065D00003F03718651886189900062B11D8DFE8E4
:1065E00003F0041029102B102D00182257212846E3
:1065F00000F0F6FC08225621284600F0F1FC0028A5
:10660000DAD17408013CE4B2002F00F08E80012F33
:10661000D0D101AA04212846FFF7B6FE38B9224698
:106620007021284600F0DCFC002800F0B28085F8DC
:10663000E060C1E73022D9E74022D7E75022D5E712
:106640001022482100F0CCFC08224721284600F007
:10665000C7FC022204463221284600F0C1FC0C226D
:1066600004433021284600F0BBFC64B204430122FD
:10667000FF21284600F0B4FC64B2044364B2302227
:106680003021284600F0ACFC00220443FF212846BC
:1066900000F0A6FC64B2204340B2B0E728224821B3
:1066A00000F09EFC08224721284600F099FC0322B6
:1066B00004463221284600F093FC044364B20922C8
:1066C0003021284600F08CFC01220443FF2128469B
:1066D00000F086FC64B2044364B22022D0E7382282
:1066E000482100F07DFC08224721284600F078FC74
:1066F000032204463221284600F072FC044364B2AF
:106700000822DDE74822114600F06AFC08224721F2
:10671000284600F065FC032204463221284600F09A
:106720005FFC044364B20722CAE702AA0321284699
:10673000FFF72AFE88B903AA02212846FFF724FEA4
:1067400058B922465021284600F04AFC28B9029A3E
:1067500003212846FFF797FE10B185F8E8602BE784
:10676000039A02212846FFF78EFE85F8E86000288C
:106770007FF422AF69692846FEF7DAF900287FF432
:106780001BAF024601230DF103012846FFF752F922
:1067900012E7019A04212846FFF775FE85F8E060AC
:1067A000E5E713B5144629B1012910D06FF00300B5
:1067B00002B010BD0DF10702502100F033FC00289B
:1067C000F6D19DF8073001335B002370F0E70DF13F
:1067D00007027021F1E7F0B5002385B04FF4FA62AB
:1067E000CDE9002344F61F63994206460F4604D8BC
:1067F0006FF00305284605B0F0BD02A9FEF7F1F9D8
:1068000005460028F6D19DF809209DF8083013436D
:106810009DF80A201343A7F636341BD06A4602219E
:106820003046FFF7B1FD00283BD19DF808302BB171
:10683000009B03F24E239C42DAD9E41A9DF80A30F9
:1068400023B3009B03F2B223B4EB430F4FEA43029E
:10685000CED9A41A9DF80B305BB101AA03213046B2
:10686000FFF792FD019B03F525739C42C0D9C0B987
:10687000E41A9DF80C30002BBCD0A4F2262204218F
:106880003046FFF700FE77610546B3E79DF8093013
:10689000002BDFD0009B03F525739C42A8D9E41A96
:1068A000D8E70546A6E770B54FF4FA6286B0002334
:1068B000CDE9022340F636330B600C4604A90646A8
:1068C000FEF78FF90546002836D19DF811209DF876
:1068D000103013439DF81220134319D002AA02214D
:1068E0003046FFF751FD002840D19DF810302BB104
:1068F000029B03F24E222368134423609DF812305A
:10690000EBB1029B03F2B222236803EB4203236044
:106910009DF81330EBB99DF814305BB101AA042146
:106920003046FFF731FD019B03F226222368134412
:106930002360D8B923687361284606B070BD9DF8FE
:106940001130002BE4D0029B03F525722368134419
:10695000DDE703AA03213046FFF716FD039B03F58D
:1069600025722368134423600028D4D00546E3E74A
:106970002DE9F743002406460D46204615F804800D
:10698000B8F1000F00D010B103B0BDE8F083671C70
:10699000B8F1FF0F15F8079029D1A71CEB5DB9F1ED
:1069A000030F36D8DFE809F0020B131B271D2C4418
:1069B000E27802EB0323A6F834313C46DEE7271DDC
:1069C0002C44E27802EB0323A6F83631F5E7271DC5
:1069D0002C44E27802EB0323A6F83831EDE7271DBB
:1069E0002C44E27802EB0323A6F83C31E5E7B8F14A
:1069F000040F0ED802344246291901A80EF032FACB
:106A0000434601AA4946304604EB080700F0B2FAB3
:106A1000D3E76FF00300D0E773B500230E46136091
:106A20000DF1070105461446FEF712F940B99DF82D
:106A300007302BB1B38A2A6A534380331B0A236081
:106A400002B070BD13B5CB681360144601AAFFF7FE
:106A5000E3FF18B92368019A1344236002B010BD04
:106A6000F8B5B0F85451D0F8580168438030000AA6
:106A70000E464543DDE90717144652B1B60206EB50
:106A80005202B2FBF4F202EB4202524302F5004220
:106A9000140C069A534301F50042120C06200332EF
:106AA000B2FBF0F2C2EBC202B2F5803F38BF033155
:106AB00003F500433EBFB1FBF0F1C1EBC10101F5AD
:106AC00000414FEA134334BF090C1B4903FB03F396
:106AD00038BF494303EB57030B44B3FBF7F39B0366
:106AE000FE2205F120007F33B3FBF2F35C434FF449
:106AF0007A7704F5FA748009B4FBF7F42401FFF700
:106B000022F904F5FA74BC4228BF4FF4FA63064632
:106B100029BFB4FBF3F300205B19B4FBF7F428BFE3
:106B2000B3FBF4F0FFF70FF9099B864294BF1E6098
:106B300018600020F8BD00BF0000F0FF2DE9F04F05
:106B400091B0054607930B6908930F46CB680B93EA
:106B500093460FAAFFF776FF0EAA39462846FFF79D
:106B60005BFF48BB0F9C95F8E0A0D5F8DC3005939F
:106B70004FF47A7606FB04F101F50041049180346C
:106B80000E99099124F0FF010A910F910499D5F80B
:106B9000E4300693BAF1080F0CBF02230323090C5B
:106BA00095F8E820DFF898810C9108D1079BCBF885
:106BB0000080C5F84081186011B0BDE8F08F0699DB
:106BC0000D932846FFF7BCFB52460599814628469F
:106BD000FFF7B6FB0D9B5B490C9A814403FB09F957
:106BE0004FEAC92940F2776309F5FA79240AB9FB1B
:106BF000F6F903FB09F909F5FA79B9FBF6F909FB8E
:106C000004F404F18003089C74430C40B4FBF2F4D8
:106C10004D4A1B0A944228BF1446012B38BF01235A
:106C20000C204FF4167258435443FFF78CF83B7E08
:106C30003A894FEA400A002B7FD14249049B0B401E
:106C400003F5FA71414B5A4341F25C23B2FBF3F274
:106C5000099B7343B3F5481F28BF4FF44813A1EBBA
:106C60004303B1FBF6F1B3FBF6F31B02B3FBF1F602
:106C70003602C6F58036564306F50046360C06F554
:106C8000803676087643B60B4FF44873734303F5AA
:106C9000004304F500401B0C5B43000C00FB00307C
:106CA000FFF751F803046422323341F28837B3FB13
:106CB000F2F340F6B532B3FBFAF302FB0377244B51
:106CC0009F429CBF42F21073B7FBF3F7DDE9053238
:106CD000134403F5FA734FF47A7A4FF4FA62B3FB74
:106CE000FAF0B3FBF2F202F5C812B2FBF0F088BF83
:106CF0004FF47047FFF727F8000200F5FA70B0FB79
:106D0000FAF0404307FB0700FFF71DF80AFB00F00D
:106D1000079B404528BF4046CBF80000C5F840011E
:106D2000CDE902934FF448730093DDE90A12019410
:106D300033462846FFF794FE3EE74FF48036A3E73C
:106D4000AE878F020000FFFF666666009A99060014
:106D50000F279F242DE9F04F11F0780F8BB018BF4B
:106D60004FF2A009C1F3C30B18BF29FA0BF99046E3
:106D70009A460DF10E024FF000034FF00001159FEF
:106D80008DF80E3004468DF80F308DF810308DF8E8
:106D90001130ADF81230099314BF09F001094FF01A
:106DA0000109FDF7ADFF9DF80E500646D5B100284C
:106DB00040F09A80149909AB05AA2046FFF7BEFE61
:106DC000002840F09380149A099B5381014606AA3B
:106DD0002046FDF7CAFF069D25B1059B9D422CBFAD
:106DE0000025012520B904AA02212046FDF788FFCD
:106DF0009DF8106026B300287AD107AA0221204608
:106E0000FDF7B3FF88B90122FF21204600F0E8F822
:106E100058B90DF11202B621204600F031F920B91F
:106E20000246FF21204600F0DBF8BDF81230079E35
:106E30005B02C4F848311EB19E422CBF00260126D9
:106E400028B90DF1110203212046FDF759FF9DF8E5
:106E5000113093B100286CD1BAF1000F03D04FEA82
:106E60000828B8FBFAFA08AA03212046FDF77DFF9F
:106E7000089B534594BF0023012320B9B9F1000FAB
:106E800038D0FF223A703A780AB914994A810DF144
:106E90000F02012120460193FDF732FF08BB9DF848
:106EA0000E20019B002A08BF0125BBF1040F18BF6B
:106EB0009DF80F2084F82E501ABFB2FA82F25209C0
:106EC000012284F82F209DF81020002A9DF811201F
:106ED00008BF0126002A08BF012384F8306084F827
:106EE00031300BB0BDE8F08F002581E735467FE7F4
:106EF0000026ACE70BF1FF32092A0AD8DFE802F0DE
:106F0000050505090907090B070B0522BAE7042245
:106F1000B8E7012E01D10322B4E7BBF1040F01D081
:106F2000012B01D10222ADE7012D16BF00233D70D8
:106F30003B700023A7E707B502F10A03009393B261
:106F40000A4690F86011D0F85C0101F0A1FB03B093
:106F50005DF804FB13B502F10A0390F86041009359
:106F6000D0F85C0193B20A4644F0010101F026FC1E
:106F700002B010BD3F2BF8B50E46054611461C4623
:106F800011D80A4F38461A4600F8016B0DF06AFF17
:106F9000621C39462846FFF7CEFF002814BF6FF069
:106FA00013000020F8BD6FF00300FBE76410002021
:106FB00073B515468DF8071001220DF1070104463F
:106FC0001E46FFF7B8FF18B16FF0130002B070BD96
:106FD000324629462046FFF7BDFF0028F6D0F3E7EA
:106FE00008B5064B19705A7019460222FFF7A3FF25
:106FF000002814BF6FF01300002008BD64100020AB
:1070000008B5074B1970110A59709A701946032276
:10701000FFF791FF002814BF6FF01300002008BD98
:107020006410002037B515468DF8071001220DF1C8
:1070300007010446FFF77FFF18B16FF0130003B09C
:1070400030BD012229462046FFF784FF0028F6D0F4
:10705000F3E7F7B515460DF1070206460F461C4645
:10706000FFF7E0FF50B99DF807301D4044EA0502E4
:10707000394630468DF80720FFF7B2FF03B0F0BD68
:1070800073B514468DF8071001220DF1070105466E
:10709000FFF751FF18B16FF0130002B070BD064E3C
:1070A000022231462846FFF755FF0028F3D13388E6
:1070B0005BBA2380F1E700BF6410002073B514466B
:1070C0008DF8071001220DF107010546FFF733FF88
:1070D00018B16FF0130002B070BD064E04223146A5
:1070E0002846FFF737FF0028F3D133681BBA236027
:1070F000F1E700BF6410002008B50220FBF73CFF59
:10710000002008BD37B5084B0190084C187894252D
:107110004FF47A73012201A905FB004003F0AEFD94
:10712000019803B030BD00BFA4100020A8100020BB
:107130007047000010B5032000F056FC01F08AFDF6
:10714000064B18600F20FBF70DFF044618B9FBF73C
:107150007EFD204610BD0124FBE700BF280800206B
:107160004FF0E022136923F00203136170474FF0E0
:10717000E022136943F0020313617047014BD3F817
:10718000900570470070FF1F014BD3F894057047BE
:107190000070FF1F014BD3F8980570470070FF1F68
:1071A0008068C0F380007047F7B500230193044660
:1071B000002800F0E980856D25B9FBF7CDF8E5657D
:1071C00084F8545023689A68D00040F1A1809A68EE
:1071D000D10000F1B480A26D42F01002A265E26D10
:1071E00042F00102E26501251846FFF7D9FFA26DC2
:1071F00002F01002024340F0C980A26D206922F41F
:10720000817242F00202A2659A68D2075DD4226BB5
:10721000A67E94F82CC0003A18BF01221703D4E9C7
:1072200002120A43217E42EA8132617E42EAC13281
:1072300042EA4632002842EA4C02B4BF20F0004144
:107240004FF400113A430A4394F82010012903D166
:10725000002E76D142F48032616A21B1A66A01F42F
:10726000E07131430A43D968E66C21F4FE3121F420
:10727000FF711143D96094F83C206168012A01F044
:10728000404C4CEA060609D1D4E910273A43324370
:10729000A66C324342EA0C0242F001061F693E4AE4
:1072A0003A4032431A6121F00042B2F1804F0CD0D3
:1072B000B1F1004F09D0394ED6F8082701F470110A
:1072C00022F470120A43C6F808275A69666BA16B4C
:1072D00022F0070232435A615A6922F0700242EAF0
:1072E00001125A61002835D19A6A62F00F029A623F
:1072F0005B6903F007039E423CD10023E365A36D65
:1073000023F0030343F00103A365284603B0F0BD57
:107310009A68234922F0104222F0170242F080526C
:107320009A60204A1268B2FBF1F2013252000192D7
:10733000019A002A3FF44BAF019A013AF7E7002582
:1073400052E7A16D41F02001A165E16D41F001011D
:10735000E16581E7B0F5001FCAD19A6AE269013A96
:1073600092006FF00F0102F01C0201FA02F2216E8E
:107370000A43BCE7A36D23F0120343F01003A36597
:10738000E36D43F00103E3650125BEE7A36D43F020
:107390001003A365F8E700BF02FCFF1F00200140B7
:1073A000400D030028080020F8B54569082D044663
:1073B0000E460AD00368DB68D80705D5A36D43F0F5
:1073C0002003A3650120F8BD0425FBF7CDFD07468A
:1073D00023681A682A4220D0A26D42F40072A26586
:1073E000DA6812F4406F14D1A27E92B91A681207BB
:1073F0000FD51846FFF7D4FE20BB5A6822F00C02C6
:107400005A60A26D22F4807222F0010242F0010261
:10741000A265227EFAB10020D5E7711CD9D0FBF716
:10742000A3FDC01BB04201D8002ED1D123681B6838
:107430002B40CDD1A26D84F8543042F00402A265F5
:107440000320C0E7A26D42F02002A265E26D42F087
:107450000102E265DDE70C221A60DCE70368186CC4
:1074600070470000F7B50023019390F85430012BCA
:10747000044600F0C08005680269012380F854309A
:107480002846FFF78DFE002840F0AF80D1E900309C
:10749000022822F004027ED0B2F1004FC3F3110E95
:1074A00035D1AA6A42EA0E02AA628A68686902EACB
:1074B000032222F07C4222F0FF0220EA03210A4349
:1074C000002B6A611DDA4D4A4D4DD2F80817AB42C8
:1074D00001F0E07043D10D0213D4D2F8083723F045
:1074E000E073034343F40003C2F80837454B1A68BE
:1074F000454BB2FBF3F20C2302FB03330193019BD8
:1075000053BB0020002384F8543003B0F0BD226E3A
:1075100000F01F074FF00F0C0CFA07FC6FEA0C0687
:1075200022EA0C0CBEF1000F11D1C3F38462BA4001
:1075300042EA0C0222668008E26901309042B4D827
:10754000A86AC3F38362BA4006403243ACE793FAB9
:10755000A3F2B2FA82F2EAE7019B013BCEE72B4DA0
:10756000AB420BD1C901CCD4D2F8083723F0E07379
:10757000034343F08073C2F80837C2E7244DAB429F
:10758000BFD14B02BDD4D2F8083723F0E0730343D8
:1075900043F48003EFE7B2F1004F01BFAA6AC3F3DF
:1075A00011018A43AA62002BABDA154813498342C2
:1075B000D1F8082709D1D1F8083702F0A07223F0DA
:1075C000E0731A43C1F808279BE71048834204D1AF
:1075D000D1F8083702F44002F1E70D48834290D118
:1075E000D1F8083702F0C072E9E7A26D42F020023C
:1075F000A265184686E7022087E700BF0020014009
:10760000001000B028080020400D0300004000B822
:10761000002000B4026838B504461046FFF7C0FDEC
:1076200008B9002038BD9368990707D4936823F000
:10763000004323F0170343F010039360FBF794FC1F
:10764000054623689B685B07EBD5FBF78DFC401B69
:107650000228F6D923689B685A07F2D5A36D43F038
:107660001003A365E36D43F00103E3650120D9E74F
:1076700073B50023026801939368DD07044602D5C1
:10768000002002B070BD9168214B194209D0A36D52
:1076900043F01003A365E36D43F00103E3650120AC
:1076A000EFE7936823F0004323F0170343F001034F
:1076B0009360184BD3F8083718021CD4637E012B53
:1076C000DED0FBF751FC144E054622681368DB0739
:1076D000D6D49368D9075FBF9368334043F0010362
:1076E0009360FBF741FC401B0228EED923681B681E
:1076F000DA07EAD4CBE7094B094A1B68B3FBF2F37C
:1077000001330193019B002BD8D0019B013BF8E78B
:107710001700008000200140E8FFFF7F28080020BC
:10772000400D030038B504460068FFF739FD0546F3
:1077300020BB94F85430012B20D0012384F854301E
:107740002046FFF795FFB0B9A36D226823F470635C
:1077500023F0010343F48073A3651C23E0651360E9
:1077600084F85400936823F0004323F0170343F098
:107770000403936038BD84F85450FBE70220F9E716
:10778000026838B5936891680446C80701D40020A0
:1077900038BD9907FBD4936803F00503012B19D179
:1077A000936823F0004323F0170343F00203936030
:1077B00003231360FBF7D8FB054623689B68DB07B0
:1077C000E5D5FBF7D1FB401B0228F6D923689B685F
:1077D000DA07F2D5A36D43F01003A365E36D43F020
:1077E0000103E3650120D3E770B5044600284BD0C0
:1077F000836D43F002038365FFF70CFF054668B90C
:107800002046FFF7BDFF054608B90123A36522689E
:10781000936823F0104323F01703936023685A689A
:1078200022F4677222F003025A6040F29F321A601B
:10783000D968164A0A40DA601A6922F040421A6191
:107840005A6922F007025A611A6A02F0F0221A629B
:107850005A6A02F0F0225A62DA6A02F0F022DA6220
:107860009A6A0B4A00269E62D2F8083723F0FE730C
:10787000C2F808372046FAF783FDE6652666A66556
:1078800084F85460284670BD0125FBE700023E8362
:107890000020014010B590F85430012B044615D05B
:1078A000012380F85430FFF7B5FE58B92046FFF7A2
:1078B00067FF38B9A36D23F4807323F0010343F00D
:1078C0000103A365002384F8543010BD0220FCE7B7
:1078D000F7B50023019390F85430012B04467FD074
:1078E000012380F85430FFF74BFF23689A6812F0A9
:1078F0000102054607D0A36D43F01003A3650023E2
:1079000084F854302DE0A16D364F21F4817141F09F
:107910000201A165DE68D96826F4FF4626F07C06E0
:1079200021F40041360421F00301360CD96008200F
:107930009968394041F0004199609968002913DA4B
:107940000199013101910199B1F52E3FF5D3A36D54
:1079500023F0120343F01003A365002384F854308E
:107960000125284603B0F0BDD3F8B410013801F06A
:107970007F010A44DCD199681A48014041F00101B5
:107980009960D3F8B41021F07F0141EAD202C3F824
:10799000B4209A68024042F002029A60FBF7E4FACF
:1079A000074623689A68D20708D4DA683243DA6057
:1079B000A36D23F0030343F001039FE7FBF7D4FA21
:1079C000C01B0228EDD923689B68D907E9D5A36DB0
:1079D00043F01003A365E36D43F00103E365BFE7E4
:1079E0000225BEE7E8FFFF7F0749CA6822F4E0628C
:1079F0000302120403F4E063120C134343F0BF6369
:107A000043F40033CB60704700ED00E0164B30B517
:107A1000DC68C4F30224C4F10703251D042B28BF2E
:107A20000423062D4FF0FF358CBF033C002405FADC
:107A300003F321EA0303A54022EA0502A34000283C
:107A400043EA0203ACBF00F16040084A4FEA031367
:107A5000B8BF00F00F00DBB2AABF00F561401354BD
:107A600080F8003330BD00BF00ED00E014ED00E011
:107A7000002807DB044A4109012300F01F0083406E
:107A800042F82130704700BF00E100E000280CDB25
:107A90004309064900F01F0020330122824041F8CB
:107AA0002320BFF34F8FBFF36F8F704700E100E0DB
:107AB00070B5D0E913456560446D14B1D0E9164541
:107AC0006560D0E9105404F01C060124B4406C60D9
:107AD000046863608368102B0BBFA260A160E16043
:107AE000E26070BD0268416CD3B210B5083B14244B
:107AF000B3FBF4F30B4CA24288BF0B4A21F0030105
:107B000099BF01F1804202F50232521807338264B4
:107B1000064AC26403F01F03012202FA03F303655D
:107B200010BD00BF070402401C080240800802404C
:107B300038B500285CD002682E4B9A424FF01401F1
:107B40004AD82D4B1344B3FBF1F32C499B00C0E9F9
:107B50001013022380F825301368056923F4FF43CE
:107B600023F070031360D0E9024323432B4345699C
:107B700011682B4385692B43C5692B43056A2B4349
:107B80000B431360FFF7AEFFB4F5804F04BF002333
:107B900043604368816C03F07F020A60D0E91314EC
:107BA000013B032B4C601ED8154B164981651344CD
:107BB0009B000121013A01FA02F200214365C265EE
:107BC0001960114B5A6400230122C36380F82430EA
:107BD00080F82520184638BD0C4B1344B3FBF1F355
:107BE0000B499B00B3E70023C0E91533C365EAE7FF
:107BF0000120F0E707040240F8FFFDBF000002404B
:107C00003F8200104009024000090240F8FBFDBF1E
:107C10000004024038B5002841D00268136823F000
:107C2000010313601F4B9A424FF0140130D81E4BD2
:107C30001344B3FBF1F31D499B00C0E91013012469
:107C400003F01C0304FA03F3002515604B60FFF7F3
:107C500049FF836C41681D60D0E913325A604A1EA7
:107C6000032A06D8124B0B449B0094401D60114B15
:107C70005C640023C363C0E91533C0E90B33C0E97A
:107C80000D33C36580F8253080F82430184638BDA0
:107C9000094B1344B3FBF1F308499B00CDE70120E6
:107CA000F5E700BF07040240F8FFFDBF00000240F7
:107CB0003F82001000090240F8FBFDBF00040240B3
:107CC00070B590F82450012D04463BD090F8256003
:107CD0000125AE4280F824504FF000062CD1022539
:107CE00080F825500568C6632E6826F001062E60D0
:107CF000FFF7DEFE036BBBB12B6843F00E032B6076
:107D0000A36C1A68D20342BF1A6842F480721A60E8
:107D1000636D1BB11A6842F480721A602B6843F0DD
:107D200001032B60002070BD2B6823F004032B603F
:107D30002B6843F00A03E2E78023C36380F82460E2
:107D40002846F0E70220EEE7034640B190F82520F0
:107D5000022A06D00422C263002280F824200120D7
:107D600070470268806C116821F00E011160016893
:107D700021F480710160116821F001011160D3E9E3
:107D8000100202F01C0101228A404260D3E9132153
:107D900051605A6D32B1116821F480711160D3E9DC
:107DA000162151600122002083F8252083F8240049
:107DB000704708B590F82530022B03D00423C36325
:107DC000012008BD03681A6822F00E021A601A68C2
:107DD00022F001021A60826C136823F4807313602E
:107DE000D0E9101303F01C02012393404B60D0E94B
:107DF00013325A60436D33B11A6822F480721A60EC
:107E0000D0E916325A60012380F82530002380F82B
:107E10002430836B03B198470020D2E770B4426CE2
:107E2000046C036826681D6802F01C02042191405E
:107E300031420FD015F0040F0CD01A6892065EBFC5
:107E40001A6822F004021A60036B6160002B33D0C1
:107E500070BC184702219140314217D015F0020F33
:107E600014D01A68940606D41A6822F00A021A601E
:107E7000012280F82520114A93428CBF104B114BF0
:107E80005960002380F82430C36ADFE7082191405D
:107E9000314211D029070FD5196821F00E01196060
:107EA000012303FA02F26260C36380F825300023E5
:107EB00080F82430436BC9E770BC704780000240F3
:107EC00000040240000002400A4A536943F4802340
:107ED00030B55361EFF3108472B60023CD58C5500E
:107EE0000433B3F5807FF9D11369DB03FCD484F349
:107EF000108830BD00400058064B5A69002ABFBFA9
:107F0000054A9A6002F188329A60BABF5869C00F78
:107F1000002070470040005823016745044B5A6910
:107F200042F000425A615869C043C00F704700BF19
:107F30000040005870B50546FBF716F8124E04468F
:107F40003369D90313D43369DA0744BF012232619C
:107F50004CF2FA32134011D10B4E306910F48020EC
:107F60000BD0FBF701F8001BA842F6D304E0FAF7A8
:107F7000FBFF001BA842E3D3032070BD024A13613C
:107F8000024A01205360F8E7004000583C110020ED
:107F90002DE9F041184D98462B78012B06460C46EA
:107FA000174626D001232B704FF47A7000236B60A4
:107FB000FFF7C0FFA0B9012E16D1104A536943F054
:107FC000010353612760BFF36F8FC4F804804FF43F
:107FD0007A70FFF7AFFF094A536923EA060353613A
:107FE00000232B70BDE8F08139462046FFF76CFF77
:107FF000EDE70220F6E700BF3C11002000400058EA
:10800000054A536923F47E7343EAC00040F480308C
:1080100040F0020050617047004000582DE9F041E7
:10802000234F3B78012B054688463FD001233B7008
:108030004FF47A7000237B60FFF77CFF044688B919
:108040002B68042B13D11B4A536943F4803343F04C
:10805000040353614FF47A70FFF76CFF0446154B2D
:108060001A681B6800233B702046BDE8F0814FF082
:10807000FF33C8F800306E68D5E901321344B342CB
:108080000AD93046FFF7BCFF4FF47A70FFF752FF72
:1080900050B1C8F800600446064A536923F47E7361
:1080A00023F002035361DAE70136E5E70224DBE758
:1080B0003C110020004000582DE9F04F524C0023A5
:1080C0004FF00F090A6832FA03F501D1BDE8F08FCD
:1080D000012505FA03F818EA020200F08E804E68C6
:1080E000032706F003054FEA430E07FA0EFC6F1E46
:1080F000012F6FEA0C0C32D8876807EA0C0ACF68A8
:1081000007FA0EF747EA0A078760476827EA080870
:10811000C6F300179F4047EA08074760C76807EAA9
:108120000C088F6807FA0EF747EA0807022DC760A8
:1081300017D14FEAD30800EB880803F0070AD8F8F4
:1081400020704FEA8A0A09FA0AFB27EA0B0B0F692B
:1081500007FA0AF747EA0B07C8F8207001E0032D79
:10816000DCD1076805FA0EF507EA0C073D4316F463
:10817000403F056041D023F0030707F1804707F532
:10818000803703F0030CBD684FEA8C0C4FF0070EEC
:108190000EFA0CFEB0F1904F25EA0E0E2FD01B4DBB
:1081A000A8422ED005F58065A84214BF07250225F8
:1081B00005FA0CF545EA0E05BD602568D74316F4AF
:1081C000801F0CBF3D4015432560656816F4001FF5
:1081D0000CBF3D4015436560D4F8805016F4803FD5
:1081E0000CBF3D401543C4F88050D4F88450B6030A
:1081F00054BF3D401543C4F88450013362E7002565
:10820000D6E70125D4E700BF000800580004004865
:10821000374A2DE9F04F00234FF0010A4FF0070BCA
:108220004FF00F0931FA03F401D1BDE8F08F0AFADB
:1082300003FC1CEA010654D023F0030404F180443B
:1082400004F5803403F00307A568BF000BFA07F8B4
:10825000B0F1904F08EA050E45D0264DA84244D013
:1082600005F58065A8420CBF02250725BD40754570
:1082700017D1D2F8805025EA0605C2F88050D2F80E
:10828000845025EA0605C2F88450156825EA0605DB
:108290001560556825EA06055560A56825EA0805B4
:1082A000A560056803265C0006FA04F423FA06F6C6
:1082B000254300EB8606056003F00705376AAD002D
:1082C00009FA05F527EA05073762856825EA0405F6
:1082D0008560456825EA0C054560C56825EA040403
:1082E000C46001339EE70025C0E70125BEE700BF5B
:1082F00000080058000400480369194214BF012017
:10830000002070470AB181617047816270470000A8
:10831000044AD168014208B502D0D060FBF738FBAF
:1083200008BD00BF0008005803689A69910744BF60
:1083300000229A629A69D2075EBF9A6942F00102EE
:108340009A61704730B5039D04682B4343EA0243AA
:10835000064A6068C1F309010B4342EA555223F013
:10836000004320EA02000343636030BDFF63FF0364
:1083700003682DE9F0419C6914F0100405460F468E
:1083800016466FD010220024DA61A0462B689A6945
:10839000900661D4B8F1000F35D044F004040120F8
:1083A0002E68B369D90541BF4FF48072F26144F081
:1083B000010401205A0541BF4FF4806244F00804D3
:1083C000F26101209B054FD54FF4007344F0020485
:1083D000F3612846FFF7A8FF736823F0FF7323F4C7
:1083E0008B3323F4FF7323F0010373606B6C23431F
:1083F0006B64202385F84130002385F8423085F8EE
:108400004030012032E07A1CC1D0FAF7ADFD801B6C
:10841000B84201D8002FB9D12B68596895F842208D
:1084200098690004D2B20AD5490408D4202A06D09B
:108430005A6842F480425A60FAF796FD06462B6865
:108440009B699B06A2D4FAF78FFD801B1928F6D9E9
:1084500020244FF0010899E7B8F1000F9DD12022A8
:10846000DA619AE720469BE70028B2D1BDE8F081A7
:1084700070B504460D46164623689B699B0701D5D7
:1084800000201BE0324629462046FFF771FFA0B9C5
:108490006A1CF1D0FAF768FD801BA84201D8002DB4
:1084A000EAD1636C43F020036364202384F84130F5
:1084B000002384F8423084F84030012070BD70B54C
:1084C00004460D46164623689B699B0601D500208D
:1084D00019E0324629462046FFF74AFF90B9FAF7DD
:1084E00043FD801BA84201D8002DECD1636C43F002
:1084F00020036364202384F84130002384F8423051
:1085000084F84030012070BD70B504460D46164613
:1085100023689B695B070ED4324629462046FFF745
:1085200027FF38BB23689A69910625D59A695207B7
:1085300003D5228D0AB1002070BD9A6912F0100295
:108540001CBF1022DA614FF0200118BF04226264C0
:10855000D9615A6822F0FF7222F48B3222F4FF7242
:1085600022F001025A60002384F8411084F842305E
:1085700084F840300120DFE7FAF7F6FC801BA842C0
:1085800001D8002DC4D1636C43F020036364202321
:1085900084F841300023EBE72DE9F041069F0446C3
:1085A000884616461D462268936938EA03030CBFC5
:1085B00001230023B34201D0002015E06B1CF3D04F
:1085C000FAF7D2FCC01BA84201D8002DEBD1636C96
:1085D00043F020036364202384F84130002384F8AF
:1085E000423084F840300120BDE8F08110B50446E7
:1085F00000284AD090F8413003F0FF021BB980F800
:108600004020FAF7B9F9242384F8413023681A6826
:1086100022F001021A60626822F070621A619A68A0
:1086200022F400429A60D4E90221012924D142F4C3
:1086300000429A605A6842F0007242F400425A6066
:10864000DA6822F40042DA60D4E904210A43A1691D
:1086500042EA0122DA60D4E907210A431A601A6863
:1086600042F001021A6000202023606484F8413047
:10867000206384F8420010BD42F4044202299A604B
:1086800004BF4FF400625A60D4E70120F3E7000012
:108690002DE9F347984690F841300A9F202B044675
:1086A0000E46914640F0868090F84030012B00F055
:1086B00081804FF0010A80F840A0FAF755FC192399
:1086C0000546009052464FF400412046FFF764FFF4
:1086D00018B1012002B0BDE8F087212384F84130B1
:1086E000102384F842306064A4F82A80638DC4F8B3
:1086F00024909BB2FF2B60632F4B26D9FF2222854B
:1087000000934FF0807331462046FFF71BFE638DC8
:108710009BB22A4639462046FBB9FFF7D0FE002817
:10872000D7D123682021D9615A6822F0FF7222F440
:108730008B3222F4FF7222F001025A6084F8411059
:1087400084F8400084F84200C4E7628D92B222852A
:1087500000934FF00073D2B2D5E7FFF789FE0028EF
:10876000B7D1636A226813F8011B91626362638D5B
:10877000228D013B9BB26385638D013A92B29BB21D
:108780002285002BC3D0002AC1D100953B46802111
:108790002046FFF701FF00289BD1638D9BB2FF2B82
:1087A00003D9FF2222850090ABE7628D92B2228529
:1087B0000090CEE702208DE7002000802DE9F347EE
:1087C000984690F841300A9F202B04460E46914669
:1087D00040F0878090F84030012B00F082804FF00D
:1087E000010A80F840A0FAF7BFFB19230546009064
:1087F00052464FF400412046FFF7CEFE18B101204B
:1088000002B0BDE8F087222384F84130102384F8B9
:1088100042306064A4F82A80638DC4F824909BB22F
:10882000FF2B6063304B26D9FF22228500934FF047
:10883000807331462046FFF785FD638D9BB22A4643
:1088400039462046FBB9FFF73AFE0028D7D1236806
:108850002021D9615A6822F0FF7222F48B3222F46F
:10886000FF7222F001025A6084F8411084F840003F
:1088700084F84200C4E7628D92B2228500934FF0E3
:108880000073D2B2D5E7FFF73FFE0028B7D12368C7
:108890005A6A636A1A70636A228D01336362638D58
:1088A000013B9BB26385638D013A92B29BB22285F4
:1088B000002BC2D0002AC0D100953B468021204623
:1088C000FFF76AFE00289AD1638D9BB2FF2B03D974
:1088D000FF2222850090AAE7628D92B22285009045
:1088E000CDE702208CE700BF0024008010B590F88F
:1088F0004120202A0346D4B21CD190F84020012AFE
:1089000018D0242280F841200268106820F001006D
:108910001060106820F480501060106801431160EE
:108920001168002041F00101116083F8414083F893
:10893000400010BD0220FCE710B590F84120202A2D
:108940000346D4B21BD190F84020012A17D024222C
:1089500080F841200268106820F001001060106863
:1089600020F4706040EA012111601168002041F09C
:108970000101116083F8414083F8400010BD0220DE
:10898000FCE70000024A136843F4807313607047E9
:10899000000400580D4B10B55B690C4628B99A05C8
:1089A00007D500F027F820B110BD9B0501D400F0D9
:1089B00019F8074A1369012C23F00403136101D14C
:1089C00030BFF1E740BF20BF20BFEDE700040058F3
:1089D00000ED00E0024B186800F4C060704700BF73
:1089E00000040058024A136843F480431360704740
:1089F000000400580C4A136823F4804313600B4BA7
:108A00001B6832214B430A49B3FBF1F351698905D5
:108A100000D533B9536913F4007F14BF032000203D
:108A20007047013BF2E700BF00040058280800200F
:108A300040420F000B4A136823F0070343F0020380
:108A40001360094B1A69012842F004021A6105D12A
:108A500030BF1A6922F004021A61704740BF20BF7C
:108A600020BFF6E70004005800ED00E04FF0B043EF
:108A70001868C0F3404070474FF0B0431868C0F327
:108A8000400070474FF0B042536823F47F4343EAFD
:108A90000023536070474FF0B0431868C0F3406044
:108AA000704700007FB54FF0B0432C4AD3F808312F
:108AB000C0F3031003F00F0352F82040284A52F885
:108AC0002330B4FBF3F4FFF785FF264B054693E80C
:108AD0000700B5F5007F04AB03E9070010D0224B77
:108AE0009C4218D303F5B70303F67F539C4229D960
:108AF00003F5741303F510639C4225D802230BE0A1
:108B00001A4B9C4207D91A4B9C421BD903F53703D9
:108B100003F5D853F0E7002304AA02EB830353F8CC
:108B20000C4C144D2B6823F0070323432B60FAF7FA
:108B30001BFA06462B6803F007039C4206D100206F
:108B400004B070BD0123E7E70024EAE7FAF70CFA66
:108B5000801B0228EED90320F2E700BF186E01083F
:108B6000786E0108C06C0108C0CF6A00BFEA21011D
:108B70003F933402004000584FF0B04310B59A685C
:108B8000D96812F00C0205D00C2A4AD101F0030377
:108B9000012B51D14FF0B0412B480B6813F0080363
:108BA00006D00B6813F0080337D1D1F8941007E012
:108BB0000C68240756BFD1F894300968C3F3032327
:108BC00050F82330002A0CBF184600204FF0B04167
:108BD0008A6802F00C020C2A1ED1CA6802F0030255
:108BE000022A2ED0032A06D10B68184A13F4801FDC
:108BF000174B18BF13464FF0B042D068D168D26807
:108C0000C0F306205843C1F302130133B0FBF3F065
:108C1000530F0133B0FBF3F010BD0B68C3F3031324
:108C2000CEE7042A05D0082A06D11B6813F4801366
:108C300005D006480023C9E700231846C6E70448C4
:108C4000C4E7024BD7E700BF186E01080024F40008
:108C50000048E80108B5FFF78FFF4FF0B043044A22
:108C60009B68C3F3031352F82330B0FBF3F008BD45
:108C7000786E01082DE9F0410446002853D04FF0EA
:108C8000B0439D68DE6803689B0605F00C0506F09E
:108C9000030668D5026A1DB10C2D46D1012E44D1C0
:108CA000002A40D04FF0B043A16A1A68170756BF98
:108CB000D3F894301B681B0903F0F00399421FD9C5
:108CC0000846FFF7EFFE00282DD14FF0B0421368A1
:108CD00043F0080313601368A16A23F0F0030B4309
:108CE0001360606AFFF7CEFEFFF7B4FFAB4B18606E
:108CF000AB4B1868FAF736F9002834D0BDE8F0819C
:108D00004FF0B042136843F008031360136823F078
:108D1000F0030B431360606AFFF7B4FE0846FFF7E9
:108D2000C1FE0028E0D00120E8E74FF0B043002A60
:108D300054D01A6842F001021A60FAF715F9074692
:108D4000FFF79AFE002842D04FF0B042136843F07C
:108D5000080313601368A16A23F0F0030B43136048
:108D6000606AFFF78FFE2368D80748D42368990705
:108D700000F18C8023681E0740F1FA80A3694FF050
:108D8000B046002B00F0E180D6F89430E16903F0A2
:108D90001002914200F0C48003F00302022AC2D004
:108DA000D80740F1B380D6F8943023F00103C6F819
:108DB0009430FAF7D9F80746D6F89430990740F17D
:108DC000A580FAF7D1F8C31B112BF5D904E0FAF707
:108DD000CBF8C01B0228B3D903208FE71A6822F012
:108DE00001021A60FAF7C0F80746FFF745FE0028AF
:108DF000B9D0FAF7B9F8C01B0228F6D9ECE7082D6C
:108E000003D00C2D05D1032E03D16368002BADD107
:108E100089E74FF0B043A1681A6822F480120A4330
:108E20001A606268B2F5803F10D11A6842F480324D
:108E30001A60FAF799F80746FFF718FE002895D14F
:108E4000FAF792F8C01B6428F6D9C5E7B2F5041FFB
:108E500004D11A6842F400121A60E6E7196821F496
:108E600080311960196821F400111960002AE0D1DD
:108E7000FAF77AF80746FFF7F9FD00283FF476AFD6
:108E8000FAF772F8C01B6428F5D9A5E7042D236909
:108E900003D00C2D0ED1022E0CD1002B3FF443AF8A
:108EA0004FF0B0426169536823F0FE4343EA016327
:108EB00053605FE74FF0B046BBB1336843F4807353
:108EC0003360FAF751F8074633685A0505D4FAF7C4
:108ED0004BF8C31B022BF7D97EE77368626923F056
:108EE000FE4343EA0263736044E7336823F480730C
:108EF0003360FAF739F8074633685B057FF53AAF18
:108F0000FAF732F8C31B022BF6D965E74FF0B042EF
:108F1000E169D2F8943023F010030B43C2F8943087
:108F20004FF0B047D7F8943043F00103C7F89430BE
:108F3000FAF71AF80646D7F894309A0718D4FAF7D1
:108F400013F8831B112BF6D946E7D6F8943023F09B
:108F50000103C6F89430FAF707F80746D6F89430BC
:108F60009B0705D5FAF700F8C31B112BF6D933E799
:108F70002368580754D50B4F3B68D90514D4FFF725
:108F800001FDF9F7F1FF06463B68DA050CD4F9F765
:108F9000EBFF831B022BF7D91EE700BF2808002038
:108FA0002C08002000040058E3684FF0B046002B66
:108FB00058D023F08003052B02BFD6F8903043F041
:108FC0000403C6F890304FF0B046F9F7CDFFD6F85D
:108FD000903043F001030746C6F8903041F28838DC
:108FE000D6F890309B0705D4F9F7BEFFC31B434565
:108FF000F6D9F1E6E36823F00403812B1BD1F9F7DE
:10900000B3FFD6F8903043F08003C6F8903007469F
:109010004FF0B04641F28838D6F89030180504D5A4
:10902000E36A002B4AD1002068E6F9F79DFFC01BD8
:109030004045F1D9D0E6F9F797FFD6F8903023F004
:109040008003C6F8903007464FF0B04641F28838AA
:10905000D6F890301905E3D5F9F786FFC01B4045D7
:10906000F6D9B9E6F9F780FFD6F8903023F08003FF
:109070000746C6F8903041F28838D6F890301A0585
:1090800016D4F9F771FFD6F8903023F00103C6F833
:10909000903007464FF0B04841F28836D8F890300B
:1090A0009B07BDD5F9F760FFC31BB342F6D993E622
:1090B000F9F75AFFC01B4045DFD98DE60C2D4ED085
:1090C000022B4FF0B0431A6822F080721A6033D13D
:1090D000F9F74AFF0546FFF7DEFC38BBD4E90C314F
:1090E0004FF0B0420B43D0682D4901400B43E16B78
:1090F0000B43216C0B43616C0B43A16B43EA0123CF
:10910000D360136843F080731360D36843F08053D7
:10911000D360F9F729FF0446FFF7BDFC002882D190
:10912000F9F722FF001B0A28F6D955E6F9F71CFFCC
:10913000401B0A28CFD94FE6F9F716FF0446FFF780
:10914000AAFC30B94FF0B042164BD1680B40D36047
:1091500069E7F9F709FF001B0A28F0D93CE6012B63
:109160003FF4E1AD4FF0B043D868236B00F0030249
:109170009A427FF4D8AD626B00F0700393427FF4A3
:10918000D2ADA26B00F4FE43B3EB022F7FF4CBAD64
:10919000636C00F06040C01A18BF0120AEE500BF4C
:1091A0008C80C111FCFFFEEE2DE9F0410D46044616
:1091B00010B90120BDE8F081684E336803F0070361
:1091C0008B4216D323689A0727D54FF0B047A26881
:1091D000BB6823F0F0031343BB60F9F7C5FE0646F6
:1091E000BB68DB0319D4F9F7BFFE831B022BF7D949
:1091F00011E0336823F007030B433360F9F7B4FE43
:109200000746336803F00703AB42DBD0F9F7ACFE47
:10921000C01B0228F5D90320CCE72368580617D5D0
:109220004FF0B0476269D7F8083123F00F0343EAE3
:109230001213C7F80831F9F797FE0646D7F8083138
:10924000D90305D4F9F790FE831B022BF6D9E2E788
:1092500023685A0713D54FF0B047E268BB6823F480
:10926000E0631343BB60F9F77FFE0646BB689B03D0
:1092700005D4F9F779FE831B022BF7D9CBE72368D6
:10928000180714D54FF0B0472269BB6823F4605328
:1092900043EAC203BB60F9F767FE0646BB685903A1
:1092A00005D4F9F761FE831B022BF7D9B3E72368D6
:1092B000DA070FD4294C236803F00703AB4239D8EF
:1092C000FFF7C8FC264B1860264BBDE8F041186834
:1092D000F9F748BE6268022A1DD1FFF7C7FB0028D4
:1092E0003FF467AF4FF0B04641F28838B36823F0DF
:1092F00003031343B360F9F737FE0746B3686268A8
:1093000003F00C03B3EB820FD4D0F9F72DFEC01B92
:109310004045F3D97FE7032A02D1FFF7BCFBDEE724
:1093200012B9FFF7A9FBDAE74FF0B0431B685B0502
:10933000D8D43EE7236823F007032B432360F9F7D3
:1093400013FE0646236803F00703AB42B8D0F9F7D3
:109350000BFE801B0228F5D95DE700BF00400058D6
:10936000280800202C08002008B5FFF773FC4FF0F8
:10937000B043044A9B68C3F3022352F82330D84019
:1093800008BD00BF586E010808B5FFF763FC4FF039
:10939000B043044A9B68C3F3C22352F82330D84039
:1093A00008BD00BF586E01084FF0B043D3F89000DD
:1093B000C0F3400070474FF0B0410209D1F8883047
:1093C00002F47F22000123EA020300F47F2003431A
:1093D000C1F8883070474FF0B041020CD1F88830A6
:1093E000120423EA020343EA0040C1F888007047F0
:1093F0000368DA0370B5044639D5FFF7C3FAF9F705
:10940000B3FD614E05463368DB0532D54FF0B043FE
:10941000616BD3F8902002F4407291421DD0D3F8D2
:109420009010D3F8902042F48032C3F89020D3F803
:10943000902021F4407022F480328D07C3F89020F0
:10944000C3F8900009D5F9F78FFD41F2883605463B
:10945000FFF7AAFF012840F090804FF0B042616B07
:10946000D2F8903023F440730B43C2F890300026BA
:1094700005E0F9F779FD401B0228C4D903262568C9
:10948000E8070AD54FF0B0416268D1F8883023EA86
:10949000124392B21343C1F88830A9070AD54FF09E
:1094A000B041A268D1F8883023EA124392B2134344
:1094B000C1F88830AA0609D54FF0B0422169D2F828
:1094C000883023F440630B43C2F88830AB0502D5E3
:1094D000206AFFF780FF680502D5606AFFF77BFF0F
:1094E000290502D5A06AFFF776FF6A0602D56069F2
:1094F000FFF761FF2B0602D5A069FFF75CFFE805C7
:1095000002D5E069FFF757FFE90610D54FF0B042EA
:10951000E168D2F8883023F440730B43C2F88830F6
:10952000B1F5807F02BFD36843F08073D3602A0413
:109530000ED54FF0B042216BD2F8883023F0404373
:109540000B43C2F8883019B9D36843F08073D360F5
:109550006B0410D54FF0B042E16AD2F8883023F0A6
:1095600040530B43B1F1005FC2F8883003D1D36898
:1095700043F48033D360304670BDF9F7F5FC401BEF
:10958000B0427FF665AF79E70004005830B590F837
:109590002C30012B02464FF0020022D0174B82F8EC
:1095A0002D00CA24012582F82C505C6253245C6291
:1095B000B1F5807F146B996914D121F488519961B8
:1095C000596C24F0010421F0004159641463DD65F5
:1095D0000A4BFF2159620020012382F82D3082F8C6
:1095E0002C0030BD21F408519961D96C24F002049B
:1095F00021F00041D9641463D865E9E700280040F0
:1096000070B50B4E036B756D1D40EA07044603D51C
:109610000123F365F9F713FEAB0704D50223F365C5
:10962000204600F0C9F9012384F82D3070BD00BF39
:109630000028004038B50A4CE36823F02003E360BB
:10964000F9F792FC0546E3689B0601D5002038BD7A
:10965000F9F78AFC401BB0F57A7FF4D90320F6E7CE
:1096600000280040F8B5114DEC6814F0400406469F
:109670001AD1EB6843F08003EB60F9F775FC2346E1
:109680000746EC6814F0400401D1032B01D11846C1
:10969000F8BDF9F769FCC01BB0F57A7F234684BF9B
:1096A000032386F82D30ECE70023F0E70028004084
:1096B00038B50F4CE36823F08003E360A3699B0691
:1096C000054606D4FFF7B6FF10B1032085F82D003C
:1096D00038BDA36923F02003A361FFF7ABFF10B1EE
:1096E000032085F82D00A36943F02003A361EFE771
:1096F0000028004038B5044600284BD090F82D30A3
:1097000003F0FF021BB980F82C20F9F72BFA022393
:10971000214D84F82D30EB68DB0636D4CA236B620A
:1097200053236B622046FFF79DFF10B1FF236B624E
:1097300038BDAB6923F08E6323F04003AB61216930
:109740006368AA690B431343A2691343AB61D4E96D
:10975000022343EA02432B61D4E90931EA680B434F
:1097600022F4F8521343EB602046FFF7A1FF0028D4
:10977000DCD1D4E90713AA690B4322F060421343FA
:1097800062691343AB61FF236B62012384F82D30C0
:109790000020CDE70120CBE7002800400023092866
:1097A00003D840EA0310C0B270470A380133C0B290
:1097B000F5E700002DE9F04790F82C30012B054625
:1097C0004FF0020069D0012385F82C304E4B85F80C
:1097D0002D00DE6806F44076B6F5807F78D04C69BF
:1097E000087891F8019091F802A091F82470002A6D
:1097F00055D19B6913F0400308BFCB70FFF7CEFF34
:1098000080464846FFF7CAFF02465046FFF7C6FFAC
:1098100081463846FFF7C2FF0B6ACF78234343EAFD
:10982000875343EA090343EA084343EA022343EA2E
:109830000063354ACA205062532050628C6A88699E
:10984000B4F5807F946945D124F48854946101244F
:10985000D465B6F5807F09BFCB69136403435364B5
:1098600018BF5064284B4A681A672A6B42F00102FD
:109870002A639A6942F488529A61244AD2F8803065
:1098800043F40033C2F880301F4BFF225A6200209D
:10989000012385F82D3085F82C00BDE8F087B4F160
:1098A000803F07D0B4F5000F04D09B6913F040034C
:1098B00008BFCB700B6ACA781C4344EA0A0444EA26
:1098C000004343EA092343EA825343EA0763B0E7CC
:1098D0000023AEE724F4085494610224D465B6F55D
:1098E000807F09BFCB6993640343D36418BFD064FE
:1098F000054B4A685A672A6B42F002022A639A694A
:1099000042F40852B8E700BF0028004000080058A1
:1099100090F82C20012A03464FF0020012D00A4A88
:1099200083F82D00CA21516253215162916941F09F
:1099300020019161FF2151620020012283F82D2036
:1099400083F82C00704700BF0028004090F82C20BE
:10995000012A03464FF0020019D00D4A83F82D006A
:10996000CA2151625321516291690A4841F0800134
:109970009161D0F8801041F48021C0F88010FF215F
:1099800051620020012283F82D2083F82C007047BB
:109990000028004000080058064B5A6D520610B5CA
:1099A000044603D54022DA65F9F74CFC012384F81C
:1099B0002D3010BD002800407047890001F1804122
:1099C00001F531410A607047890001F1804101F5DC
:1099D0003141086870470000034AD2F8903043F4E0
:1099E0000043C2F89030704700040058034AD2F890
:1099F000903023F40043C2F89030704700040058C0
:109A0000074B1A6822F040021A6040F441704FF48C
:109A1000B85218605A601A6842F040021A607047E3
:109A20000000015837B5054600284ED0837903F071
:109A3000FF046BB1032C0BD0254B4FF400629A61ED
:109A40002868FFF7DDFF002401232B71AC602FE0B5
:109A500000236B712846F9F7A1F91E4AD2F890301D
:109A600043F48053C2F89030002CE5D102234FF02C
:109A7000B042AB71D2F8943023F40043C2F8943072
:109A8000154B1B681C214B43DB0C64214B4301939A
:109A9000019B93B90124AC60FFF79EFF0C4B9A68C1
:109AA00042F400629A604FF400629A61002CC7D0C1
:109AB0000123AB71204603B030BD019B013B0193F4
:109AC000D2F894305B04E3D4E6E70124F2E700BF68
:109AD00000040058000800582808002037B5174D2A
:109AE0002B6802461C204343DB0C6420434314488C
:109AF0000193019B93B901209060114C21732B6855
:109B00001C214B43DB0C64214B430193019B6BB93C
:109B1000012090600A4BDB6803B030BD019B013B24
:109B2000019383689C07E4D50020E6E7019B013B95
:109B30000193A368DB07E9D5ECE700BF2808002004
:109B40000000015837B5184D2B6802461C204343CE
:109B5000DB0C6420434315480193019BA3B901200A
:109B60009060124CFF2323732B681C256B43DB0C86
:109B700064256B430193019B73B9012090600B4BEB
:109B8000DB680B7003B030BD019B013B0193836820
:109B90009C07E2D50020E4E7019B013B0193A36809
:109BA000DB07E8D5EBE700BF2808002000000158DC
:109BB0000E4B0F491B681822534382B01B0D6422C1
:109BC000534301934B69019AC3F3800322B90223E3
:109BD0008360012002B07047019A013A01924A69FC
:109BE000920701D5002BEDD10020F3E728080020D3
:109BF0000004005807B50379012B0FD10A4B1B68ED
:109C0000182253431B0C0193FFF7F0FE019B013B0D
:109C10000193019B002BF9D1FFF7DEFE03B05DF845
:109C200004EBFFF7C5BF00BF28080020F8B51E46AB
:109C30008379012B154604460F46DAB22DD14379BC
:109C4000012B2AD0022342718371FFF7D3FF0D212C
:109C50002046FFF7CBFEFFF741FF390A2046FFF70A
:109C60003DFFF9B22046FFF739FF2E44B5420ED131
:109C70002046FFF7B1FEFFF79BFFA06801230038E5
:109C8000A3714FF0000318BF01206371F8BD15F8F0
:109C9000011B2046FFF722FFE8E70220F6E7F8B5B0
:109CA0001E468379012B154604460F46DAB22FD1A2
:109CB0004379012B2CD04271FFF79CFF1D212046D8
:109CC000FFF794FEFFF70AFF390A2046FFF706FF69
:109CD000F9B22046FFF702FF00212046FFF7FEFE03
:109CE0002E44B5420ED12046FFF776FEFFF760FF07
:109CF000A06801230038A3714FF0000318BF0120B2
:109D00006371F8BD29462046FFF71CFF0135E8E7DF
:109D10000220F6E7F8B51F468379012B1546044665
:109D20000E46DAB22CD14379012B29D04271FFF7CC
:109D300061FF06F0EF03A3F1840253425341237104
:109D400031462046FFF752FEFFF7C8FE2F44AF42D0
:109D500010D1FFF741FE842E02D02046FFF728FFE6
:109D6000A06801230038A3714FF0000318BF012041
:109D70006371F8BD15F8011B2046FFF7AFFEE6E75B
:109D80000220F6E7F8B51E468379012B15460446F6
:109D90000F46DAB227D14379012B24D04271FFF765
:109DA00029FF39462046FFF721FEFFF797FE0021E5
:109DB0002046FFF793FE2E44B5420ED12046FFF712
:109DC0000BFEFFF7F5FEA06801230038A3714FF0EA
:109DD000000318BF01206371F8BD29462046FFF734
:109DE000B1FE0135E8E70220F6E737B50023ADF80C
:109DF000043001AA022312210546FFF7C3FFBDF874
:109E00000440022364BA01AAA4B219462846FFF707
:109E100081FFE20702D5284609F090FBA30702D58F
:109E2000284609F091FB600702D5284609F0B6FBE9
:109E3000210702D5284609F0B7FBE20602D52846DD
:109E400009F0B8FBA30602D5284609F0A1FB60067D
:109E500002D5284609F07EFB210606D514F4807150
:109E600018BF0121284609F07BFBA20502D5284630
:109E700009F086FB630402D5284609F0A1FB03B074
:109E800030BDF8B51E468379012B154604460F46B2
:109E9000DAB227D14379012B24D04271FFF7AAFE11
:109EA0000E212046FFF7A2FDFFF718FE3946204697
:109EB000FFF714FE2E44B5420ED12046FFF78CFD6D
:109EC000FFF776FEA06801230038A3714FF000036E
:109ED00018BF01206371F8BD15F8011B2046FFF77C
:109EE000FDFDE8E70220F6E7F8B51E468379012B71
:109EF000154604460F46DAB22BD14379012B28D000
:109F00004271FFF777FE1E212046FFF76FFDFFF736
:109F1000E5FD39462046FFF7E1FD00212046FFF729
:109F2000DDFD2E44B5420ED12046FFF755FDFFF76B
:109F30003FFEA06801230038A3714FF0000318BF53
:109F400001206371F8BD29462046FFF7FBFD01356E
:109F5000E8E70220F6E7026852E8003F23F0C0037A
:109F600042E8003102680029F5D102F1080353E804
:109F7000003F23F4000302F1080C4CE800310029F3
:109F8000F3D12023C0F888307047000010B5026874
:109F900052E8003F23F4907342E800310268002940
:109FA000F5D10F4C02F1080353E8003F234002F1C2
:109FB000080C4CE800310029F4D1C36E012B07D105
:109FC00052E8003F23F0100342E800310029F7D1A6
:109FD0002023C0F88C300023C366436710BD00BF48
:109FE000FEFFFFEFF8B504461346D4F88850202D45
:109FF00032D1F1B1EAB1E06FA4F85620A4F85420B0
:10A0000000262122C4F890602165C4F888202268C7
:10A0100088B1124FC762124F0763124F2832C0E94E
:10A020000D76FDF74DFE30B11023C4F89030C4F822
:10A0300088500120F8BD236840221A62226802F18C
:10A04000080353E8003F43F0800302F1080141E8B0
:10A0500000300028F3D1EDE70220EBE769A000080B
:10A06000B1A00008BDA0000808B50346806A1B68BF
:10A070001B6813F0200317D1A0F85630026802F1D4
:10A08000080353E8003F23F08003083242E8003120
:10A0900002680029F2D152E8003F43F0400342E851
:10A0A00000310029F7D108BDF9F70CFAFBE770473A
:10A0B00008B5806AFFF7FBFF08BD7047806A38B5B6
:10A0C0000468D0F88830D0F88C50A268120606D503
:10A0D000212B04D10023A0F85630FFF73CFFA368E2
:10A0E0005B0606D5222D04D10023A0F85E30FFF7D1
:10A0F0004DFFD0F8903043F01003C0F89030FFF7D8
:10A10000DCFF38BD08B5806A0023A0F85E30A0F8F7
:10A110005630FFF7D2FF08BD704700000368D969C9
:10A120001A682DE9F04140F60F0631429D68044659
:10A1300010D18E0640F1978002F0200605F080577E
:10A140003E4300F09080436F002B00F08580BDE817
:10A15000F0411847AB4EAC482E401040304300F061
:10A160008280CF0709D5D00507D501201862D4F821
:10A17000900040F00100C4F890008F0709D5E8076F
:10A1800007D502201862D4F8900040F00400C4F80B
:10A1900090004F0709D5E80707D504201862D4F8C6
:10A1A000900040F00200C4F890000F070BD502F0B9
:10A1B0002000304307D008201862D4F8900040F007
:10A1C0000800C4F890000E050AD5500108D54FF4D8
:10A1D00000601862D4F8903043F02003C4F8903047
:10A1E000D4F89030002B37D08B0609D502F020022E
:10A1F00005F080552A4303D0636F0BB12046984782
:10A200002668D4F89020B36802F0280203F04003D7
:10A2100053EA0205204621D0FFF7B8FEB3685F0677
:10A2200017D5226802F1080353E8003F23F04003EA
:10A23000083242E800310029F3D1D4F8800040B15F
:10A24000724B8363FDF7B5FD30B1D4F88000836BAA
:10A250007DE72046FFF731FFBDE8F081FFF72DFFD6
:10A26000C4F89050F8E7E06E012840F08980CE06EF
:10A2700040F18680D00640F1838010221A629A68ED
:10A2800051064BD5D4F8802011684A6892B2002A52
:10A29000E2D0B4F85C009042DED9A4F85E200A68EF
:10A2A00092062FD453E8002F22F4807243E8002155
:10A2B0000029F7D103F1080252E8002F22F0010231
:10A2C00003F1080040E800210029F3D103F108025E
:10A2D00052E8002F22F0400203F1080040E800217C
:10A2E0000029F3D12022C4F88C20E16653E8002F26
:10A2F00022F0100243E800210029F7D1D4F88000B1
:10A30000FDF722FD02232367B4F85E30B4F85C1039
:10A31000C91A89B22046FFF7FFFE9DE7B4F85E2018
:10A32000B4F85E00B4F85C1080B292B2002893D00A
:10A33000891A89B200298FD053E8002F22F4907235
:10A3400043E800200028F7D1314D03F1080252E81C
:10A35000002F2A4003F1080646E800200028F4D127
:10A360002022C4F88C206067E06653E8002F22F0BA
:10A37000100243E800200028F7D102232367C9E731
:10A38000CF0209D56E0207D54FF4801220461A621B
:10A39000BDE8F04100F0F2BD08060BD502F08000E8
:10A3A00005F40005284305D0A36F002B3FF454AFFC
:10A3B0002046CCE64F0611D556060FD553E8002FA0
:10A3C00022F0400243E800210029F7D12023C4F8FD
:10A3D0008830A1672046F9F775F83DE70D0206D5EC
:10A3E000500004D52046BDE8F04100F0C9BDCB01C6
:10A3F0007FF532AF002ABFF62FAF2046BDE8F0410F
:10A4000000F0BDBD010000102001000405A10008FE
:10A41000FEFFFFEFD0F88C20B0F86010222A08B5BC
:10A42000036855D15B6A826D0B401370836D0133F5
:10A430008365B0F85E30013B9BB2A0F85E30B0F8A7
:10A440005E309BB2002B42D1026852E8003F23F4F9
:10A45000907342E8003103680029F5D103F1080246
:10A4600052E8002F22F0010203F1080C4CE8002111
:10A470000029F3D12022C0F88C20184A416793426A
:10A48000016705D1C26E012A0ED0F9F729F81EE046
:10A490005A681102F6D553E8002F22F0806243E893
:10A4A00000210029F7D1EDE70022C26653E8002F12
:10A4B00022F0100243E800210029F7D1DA69B0F850
:10A4C0005C10D20644BF10221A62FFF725FE08BDB9
:10A4D0009A6942F008029A61F9E700BF00800040E3
:10A4E000D0F88C20B0F86010222A08B5036852D149
:10A4F0005A6A1140826D22F8021B8265B0F85E2014
:10A50000013A92B2A0F85E20B0F85E2092B2002A22
:10A5100040D153E8002F22F4907243E80021002933
:10A52000F7D103F1080252E8002F22F0010203F1F3
:10A53000080C4CE800210029F3D12022C0F88C201F
:10A54000174A41679342016705D1C26E012A0ED0B6
:10A55000F8F7C6FF1EE05A681102F6D553E8002F3F
:10A5600022F0806243E800210029F7D1EDE70022C4
:10A57000C26653E8002F22F0100243E800210029B0
:10A58000F7D1DA69B0F85C10D20644BF10221A6223
:10A59000FFF7C2FD08BD9A6942F008029A61F9E727
:10A5A000008000402DE9F84F0368B0F86060D3F8F0
:10A5B0001CB01F689D68D0F88C20222A044640F009
:10A5C000B980B0F8683043B1DFF87491DFF874A156
:10A5D0004FF000081BF0200F20D1B4F85E309BB282
:10A5E000D3B1B4F868209A4216D9226802F1080360
:10A5F00053E8003F23F08053083242E800312268DC
:10A600000029F2D1504B636752E8003F43F020032A
:10A6100042E800310029F7D1BDE8F88F2368A26D28
:10A620005B6A33401370A36D0133A365B4F85E30E9
:10A63000013B9BB2A4F85E302368D3F81CB01BF03A
:10A64000070F2ED01BF0010F09D0F90507D5012205
:10A650001A62D4F8902042F00102C4F890201BF056
:10A66000020F09D0EA0707D502221A62D4F8902017
:10A6700042F00402C4F890201BF0040F09D0E80750
:10A6800007D504221A62D4F8903043F00203C4F8CC
:10A690009030D4F8903023B12046FFF70EFDC4F877
:10A6A0009080B4F85E309BB2002B93D1226852E8C0
:10A6B000003F23F4807342E8003123680029F5D17C
:10A6C00003F1080252E8002F02EA090203F1080030
:10A6D00040E800210029F3D120225345C4F88C2002
:10A6E000616721670AD05A68110207D553E8002F25
:10A6F00022F0806243E800210029F7D1E26E012AAE
:10A7000014D10022E26653E8002F22F0100243E841
:10A7100000210029F7D1DA69B4F85C10D20644BFF1
:10A7200010221A622046FFF7F7FC53E72046F8F79D
:10A73000D7FE4FE79A6942F008029A616CE700BFC2
:10A74000FEFFFFEF0080004015A400082DE9F84F40
:10A750000368B0F86060D3F81CB01F689D68D0F83B
:10A760008C20222A044640F0B780B0F8683043B10C
:10A77000DFF87091DFF870A14FF000081BF0200F98
:10A7800020D1B4F85E309BB2D3B1B4F868209A42BD
:10A7900016D9226802F1080353E8003F23F08053E2
:10A7A000083242E8003122680029F2D14F4B63673A
:10A7B00052E8003F43F0200342E800310029F7D17E
:10A7C000BDE8F88F2368A26D596A314022F8021B58
:10A7D000A265B4F85E20013A92B2A4F85E20D3F8E4
:10A7E0001CB01BF0070F2ED01BF0010F09D0F9058C
:10A7F00007D501221A62D4F8902042F00102C4F871
:10A8000090201BF0020F09D0EA0707D502221A6236
:10A81000D4F8902042F00402C4F890201BF0040FFA
:10A8200009D0E80707D504221A62D4F8903043F023
:10A830000203C4F89030D4F8903023B12046FFF7DB
:10A840003CFCC4F89080B4F85E309BB2002B95D1EC
:10A85000226852E8003F23F4807342E80031236805
:10A860000029F5D103F1080252E8002F02EA09029B
:10A8700003F1080040E800210029F3D120225345CC
:10A88000C4F88C20616721670AD05A68110207D585
:10A8900053E8002F22F0806243E800210029F7D11D
:10A8A000E26E012A14D10022E26653E8002F22F062
:10A8B000100243E800210029F7D1DA69B4F85C10EE
:10A8C000D20644BF10221A622046FFF725FC55E746
:10A8D0002046F8F705FE51E79A6942F008029A61AE
:10A8E0006EE700BFFEFFFFEF00800040E1A400081C
:10A8F00038B5044603682169A2681D68C0690A4327
:10A9000061690A437749024329400A431A605A6839
:10A91000E16822F440520A435A60734AA1699342A3
:10A920001CBF226A11439A6822F06E4222F4306200
:10A930000A439A60DA6A616A22F00F020A43DA6215
:10A940006A4A934219D14FF0B043694AD3F888302C
:10A9500003F0030343F44033934200F0B480B3F1B7
:10A96000031F24D0013A934240F0B580B0F5004F68
:10A9700040F08F80FEF700F96EE05E4A93421CD1F2
:10A980004FF0B0435C49D3F8883003F00C0343F434
:10A9900040228A4200F0978006D8002B7CD0574B8B
:10A9A0009A42E3D0012026E0B2F10C1FFAD1B0F5B3
:10A9B000004F53D04FF4004075E04B4A9342F1D121
:10A9C0004FF0B043D3F8883003F44063B3F5006F21
:10A9D00018D006D85BB1B3F5806FE3D1FEF7CCF8A1
:10A9E00007E0B3F5406FDDD14FF400400BE0FEF718
:10A9F000BBFC40B900204FF00113A3660023C4E95B
:10AA00001D3338BD3E4865683E4B626A05EB450123
:10AA100033F81220B0FBF2F39942C3D8B3EB053FF1
:10AA2000C0D800231946F7F7F3FA090241EA10618A
:10AA30006B080002C0182A464FF0000341F10001E4
:10AA4000F7F7E6FA304BA0F540729A42AAD823688D
:10AA5000D860CFE7FEF788FC0028CBD06168294B8F
:10AA6000626A33F81220B0FBF2F24B0803EB4203A8
:10AA70004FF6EF72B3FBF1F3A3F11001914291D8BD
:10AA800023F00F02216892B2C3F342031343CB6059
:10AA9000B0E7FEF771F804E0B0F5004FDAD0FEF74A
:10AAA00063FC0028A6D06368616A164A32F8112058
:10AAB000B0FBF2F000EB5300B0FBF3F04FF6EF7396
:10AAC000A0F11002C1E7B0F5004F0D48EBD1C5E78A
:10AAD000FEF75AFCC0E7B0F5004FF9D0FEF754FC82
:10AAE000DFE700BFF369FFCF00800040003801407E
:10AAF000020003000044004008000C0004000C00A9
:10AB00000024F400B86E0108FFFC0F00836ADA0726
:10AB100010B506D50168C46A4A6822F4003222439F
:10AB20004A609C0706D50168046B4A6822F48032AB
:10AB300022434A60590706D50168446B4A6822F4EB
:10AB4000802222434A601A0706D50168846B4A684E
:10AB500022F4004222434A60DC0606D50168C46B39
:10AB60008A6822F4805222438A60990606D50168D9
:10AB7000046C8A6822F4005222438A605A060FD578
:10AB80000168446C4A6822F480122243B4F5801FA5
:10AB90004A6005D14A68846C22F4C00222434A60AC
:10ABA0001B0606D50268C16C536823F400230B43CF
:10ABB000536010BD2DE9F843DDF8209005460F469F
:10ABC000164698462A68D36937EA03030CBF012367
:10ABD0000023B34201D0002029E0B9F1FF3FF2D0B9
:10ABE000F8F7C2F9A0EB080048452C6802D8B9F183
:10ABF000000F1ED154E8003F23F4D07344E8003224
:10AC0000002AF7D104F1080353E8003F23F00103C1
:10AC100004F1080141E80032002AF3D12023C5F8ED
:10AC20008830C5F88C30002385F884300320BDE8D7
:10AC3000F88323685A07C5D5E3691B05C2D54FF4CD
:10AC40000063236254E8003F23F4D07344E80032E9
:10AC5000002AF7D104F1080353E8003F23F0010371
:10AC600004F1080141E80032002AF3D12023C5F89D
:10AC70008830C5F88C30C5F89030D4E72DE9F7431B
:10AC80009846D0F88830202B04460E46174643D10C
:10AC9000002943D0002A41D021230025C0F890503C
:10ACA000C0F88830F8F760F9A368A4F85470B3F5D9
:10ACB000805F8146A4F8567003D123690BB93546ED
:10ACC0001E46B4F85620CDF8008092B24B4642B9E9
:10ACD00040212046FFF76EFF48B92023C4F8883092
:10ACE00006E0002280212046FFF764FF18B1032010
:10ACF00003B0BDE8F08322685EB935F8023BC3F3C8
:10AD000008039362B4F85620013A92B2A4F8562090
:10AD1000D7E716F8013BF4E70220E9E70120E7E76F
:10AD200073B504460026C0F89060F8F71DF9236853
:10AD30001B681A07054619D423681B685B070AD5E8
:10AD40006FF07E43009300222B464FF48001204693
:10AD5000FFF730FFB0B900202023C4F8883084F812
:10AD60008400C4F88C30E06620670CE06FF07E430E
:10AD70000093324603464FF400112046FFF71AFFB6
:10AD80000028D9D0032002B070BD10B5044650B3DE
:10AD9000D0F888301BB980F88430F8F795FA22682B
:10ADA0002423C4F88830136823F00103136020467D
:10ADB000FFF79EFD012816D0A36A13B12046FFF7C6
:10ADC000A5FE23685A6822F490425A609A6822F0DD
:10ADD0002A029A601A6842F0010220461A60BDE811
:10ADE0001040FFF79DBF012010BD000030B5816508
:10ADF0008168A0F85C200023B1F5805FA0F85E2098
:10AE0000436735D10369002B40F2FF1318BFFF23BE
:10AE1000A0F860300023C0F890302223C0F88C30B6
:10AE2000016801F1080353E8003F43F001030831D2
:10AE300041E800340368002CF2D1456E8468016952
:10AE4000B5F1005F32D1B0F8685095422ED8B4F514
:10AE5000805F244A03D1244C002908BF2246426760
:10AE6000B1B153E8002F42F4807243E80021F7E7C4
:10AE700029B90369002B14BF7F23FF23C8E7B1F171
:10AE8000805FC5D10369002B14BF3F237F23BFE739
:10AE900003F1080252E8002F42F0805203F108004B
:10AEA00040E800210029F3D1002030BDB4F5805FD7
:10AEB0000E4A03D10E4C002908BF2246426741B119
:10AEC00053E8002F42F4907243E800210029F7D1A3
:10AED000EAE753E8002F42F0200243E8002100296E
:10AEE000F7D1E1E7A5A500084DA7000815A40008C3
:10AEF000E1A40008D0F88C30202B30B415D1B9B1C2
:10AF0000B2B100230468C3660A4B9C420AD063684E
:10AF10001B0207D554E8003F43F0806344E8003546
:10AF2000002DF7D130BCFFF761BF022030BC704765
:10AF30000120FBE700800040436E30B52BB90123B0
:10AF4000A0F86A30A0F8683030BD0368094D9A68EF
:10AF50009968094C490FC2F342626B5C615CDB008B
:10AF6000B3FBF1F3A0F86A30AB5CA25CDB00B3FB8F
:10AF7000F2F3E7E7D86E0108D06E0108704770471A
:10AF800070471FB504AB03E9060090F88430012B2D
:10AF900004463AD0012380F884302423C0F8883056
:10AFA00003681A6822F001021A609A6822F44012BB
:10AFB0000A439A6071B95A68BDF80C009DF80E10EA
:10AFC00022F0100202435A605A6822F07F4242EA9D
:10AFD00001625A601A6842F001021A60F7F7C4FF72
:10AFE0006FF07E42034600924FF48001002220461B
:10AFF000FFF7E0FD38B92023C4F88830002384F837
:10B00000843004B010BD0320F8E70220F9E790F87F
:10B010008430012B0FD0012380F88430016851E87F
:10B02000002F42F0020241E80023002BF6D180F805
:10B030008430184670470220704710B590F884306D
:10B04000012B044617D02423C0F8883003681A68FF
:10B05000196821F00101196042F000524FF00051CF
:10B0600041661A60FFF768FF2023C0F8883000208F
:10B0700084F8840010BD0220FCE770B590F884309D
:10B08000012B044617D005682423C0F888302E68A9
:10B090002B6823F001032B60AB6823F06043194356
:10B0A000A960FFF749FF20232E60C0F888300020F8
:10B0B00084F8840070BD0220FCE770B590F88430FD
:10B0C000012B044617D005682423C0F888302E6869
:10B0D0002B6823F001032B60AB6823F060631943F6
:10B0E000A960FFF729FF20232E60C0F888300020D8
:10B0F00084F8840070BD0220FCE7000038B5084DDC
:10B10000052455F8043B2BB9013C14F0FF04F8D199
:10B11000204638BDDB6898470028F5D0F9E700BF26
:10B1200090120020034BD870034B1B681B6C03B1BB
:10B13000184770477812002074120020034B1874CF
:10B14000034B1B685B6C03B11847704778120020F3
:10B1500074120020F0B5314D314B95F90420314E79
:10B1600091B00C46012795F905108DF8047002285E
:10B170008DF809208DF80A1010D18DF80800D871CB
:10B180001C7202F063FD337803B114B101A803F01F
:10B19000C1F9254B059A1A6011B0F0BD59714FF4F1
:10B1A00080711A71D9801C7233788DF8087053BB86
:10B1B0001F2306A88DF81C208DF8183002F024FFFC
:10B1C00020238DF8183006A82B798DF81C3002F05A
:10B1D0001BFF22238DF8183006A86B798DF81C30E0
:10B1E00002F012FF21238DF8183006A86B798DF834
:10B1F0001C3002F009FF29238DF8183006A80B4BEC
:10B20000079302F001FF02F021FD012306A88DF84B
:10B2100018308DF81C3002F0F7FEB4E778120020E9
:10B220006008002054110020481200200004000192
:10B230007FB5092301A88DF8043003F06BF90038BD
:10B24000044B059A1A6018BF0120404207B05DF810
:10B2500004FB00BF4812002070B504460B46144999
:10B2600062784A700020A2780A7208701A884A72BE
:10B270009A788A72DB780B746368CB600D4B1B681D
:10B28000DA6A2AB1237803F0FB030A2B00D0904737
:10B29000094E002556F8043B1BB15B6A0BB12046F2
:10B2A00098470135EBB2052B6DB2F3D170BD00BFED
:10B2B00030080020741200209012002070B504465F
:10B2C00011480123037063784370A3788372E368A5
:10B2D000C360E378037623694376237943720B4B8B
:10B2E0001B689B6A03B19847094E002556F8043B3A
:10B2F0001BB19B690BB1204698470135EBB2052B7A
:10B300006DB2F3D170BD00BF44080020741200205C
:10B3100090120020014B1868704700BF48120020AF
:10B3200000B58BB0012368468DF8003002F046FD71
:10B3300038B99DF80400003818BF01200BB05DF843
:10B3400004FB0020FAE7000008B501F037FE40B921
:10B35000FFF7E6FF012806D0054B197AD879FFF7E9
:10B36000F9FE012008BDBDE80840FFF7C7BE00BFD9
:10B37000600800202DE9F04186B005460E461746CC
:10B3800001F01CFE002873D101F030FE044640B9E4
:10B39000FFF7C6FF01280AD03D4B197AD879FFF78D
:10B3A000D9FE6FF00204204606B0BDE8F081DFF858
:10B3B000E48088F80860003E18BF01268DF804601C
:10B3C000354E687833798DF81230694602F094FC76
:10B3D00000283FD08DF804400394ADF810406FF082
:10B3E000060495E803002D4B83E80300337988F8C1
:10B3F0000A30394601A803F091F9294B059A1A60E1
:10B4000011283FD801A353F820F000BF77B40008FB
:10B4100071B4000885B4000885B4000885B400083C
:10B4200085B4000885B40008A3B3000885B40008FB
:10B4300085B4000885B400086BB4000885B4000822
:10B4400085B4000871B4000871B4000871B4000834
:10B450008BB400082B788DF808306B78ADF810307D
:10B460006B6803934FF0FF34BBE76FF005049AE776
:10B470006FF0010497E70B4B00221A70E31D18BF11
:10B48000144690E74FF0FF348DE76FF004048AE72D
:10B490006008002044080020781200205408002092
:10B4A000481200204712002037B501F0A9FD134DC6
:10B4B000052455F8043B4BB11A693AB19B682BB18E
:10B4C000984718B155F8043C1B699847013C14F0A3
:10B4D000FF04EED1FFF712FE68B9094D2B7853B186
:10B4E000084BADF80040D978019422466846FFF732
:10B4F00041FF00B92C7003B030BD00BF9012002096
:10B50000471200207812002030B58BB0044601F0BD
:10B5100055FD0546002835D1FFF702FF012834D13B
:10B5200068468DF8005002F049FC40BB9DF804309D
:10B53000A34204D0012C22D0022C12D014B100203E
:10B540000BB030BD002BFAD068468DF8044002F0F5
:10B550005BFDA0B90E4B1B681B6B002BEFD098470F
:10B56000EDE763B968468DF8044002F04DFD30B94F
:10B57000074B1B681B6B002BE1D02046EFE74FF019
:10B58000FF30DDE76FF00100DAE76FF00200D7E788
:10B590007412002010B504468AB018B94FF0FF307D
:10B5A0000AB010BD002368468DF8003002F006FC9A
:10B5B0000028F3D19DF804302370F1E77FB5002215
:10B5C0000B4620498DF8072001220A7042784A7004
:10B5D0000446002A33D102790A721A884A729A788C
:10B5E0008A72DB780B740369CB60C378164D8DF8D3
:10B5F0000830037B8DF80930836803932B68DB6A7E
:10B600000BB102A898472B689B6B13B1227E02B145
:10B6100098470E4E052556F8043B1BB1DB690BB16C
:10B6200020469847013D15F0FF05F4D10DF10700C4
:10B63000FFF7B0FF637913B1054B01221A7004B014
:10B6400070BD00BF3008002074120020901200204E
:10B650004712002010B504468AB018B94FF0FF30E9
:10B660000AB010BD202368468DF8003002F0A6FB1A
:10B670000028F3D1024A9DF9043023701371EFE7DB
:10B680007812002000B58BB02323019068468DF816
:10B69000003002F0B9FC003818BF012040420BB066
:10B6A0005DF804FB70B5654C01468EB0182220464B
:10B6B00006F0C0F8624B00221A70F8F719FF2378E1
:10B6C0004068012202FA03F1014004D15D4B0846B3
:10B6D00008F09CF8FEE75C495C481A4602F0F8F86E
:10B6E00018B14FF0FF300EB070BD272304A88DF8BD
:10B6F000103002F089FC564E564D002870D10123BF
:10B7000033702B68DB690BB100209847272304A80E
:10B710008DF8103002F052FB059B93F84820227000
:10B7200093F8182193F81A316270A370464BD3E94D
:10B73000020105F06FFF05460028D2D1464E0623D0
:10B7400004A88DF8103002F039FB059B736104A842
:10B7500002F05AFC022304A88DF81030059602F07E
:10B760002DFB0836032304A88DF81030059602F04F
:10B7700025FB0F2606F014F8012304A88DF81430D9
:10B780008DF8106002F040FC10230DEB03008DF8E3
:10B7900010308DF8145002F037FC04238DF810306F
:10B7A00004A8A3788DF8143002F02EFC3A238DF80B
:10B7B000103004A86369059302F026FC02A92078E2
:10B7C0008DF8086004F09CF8003818BF0120E07183
:10B7D0001420FFF757FFE07903F062F9284682E76B
:10B7E00028238DF810302B681B6943B104A802F0A0
:10B7F000E5FA2B6805981B6940F2C4519847272346
:10B8000004A88DF8103002F0FFFB50B9012304A802
:10B810008DF8103002F0D2FA9DF81430002B7FF42E
:10B820006EAF3378002B7FF46CAF052204A88DF83F
:10B830001020059302F0E8FB78E700BF78120020A3
:10B8400047120020E06E01084C1200206412002014
:10B850005411002074120020B412002037B50023C8
:10B860000D4601930446D0B900F0A8FB0190019B5E
:10B87000D3B10F4A42F824300E4A9A620E4A126837
:10B88000916B1963916C596392690C49D9625A6141
:10B8900028465B680A49F2229847002006E001A981
:10B8A00000F092FB0028E2D04FF0FF3003B030BD33
:10B8B0009012002055B100087412002031B2000827
:10B8C00055110020194B07B51860194B194A1A6019
:10B8D000194A5A60194A9A60194ADA60194B026883
:10B8E0001A6042685A6082689A60C268DA60164AD2
:10B8F0001A6182695A61154BC26B5A60144A0191F0
:10B9000019609A601946134ADA600020FFF7A6FF13
:10B9100048B901A800F056FB003818BF012040428A
:10B9200003B05DF804FB4FF0FF30F9E7741200201C
:10B9300064120020BDB20008BDB50008D1B90008EE
:10B9400059B200084C120020B1F80008A4120020DF
:10B9500025B100083DB1000849B118B1012804D053
:10B9600000207047034B0B60FAE7034BFBE74FF0F7
:10B97000FF307047000400010100010208B503F028
:10B98000ABF8002814BF6FF00100002008BD08B517
:10B9900002F084F9002814BF6FF00100002008BDF8
:10B9A00010B504468AB018B94FF0FF300AB010BD88
:10B9B000212368468DF8003002F000FA0028F3D108
:10B9C000024A9DF9043023705371EFE7781200208A
:10B9D0002DE9F0412F4D304F00232B7043786B70D1
:10B9E0003B689B6A8AB004460BB128469847DFF84B
:10B9F000AC80002658F8043B1BB11B6A0BB12046F3
:10BA000098470136F3B2052B76B2F3D12378052B94
:10BA10002FD00B2B35D0012B25D1214C0623684686
:10BA20008DF8003002F0CAF90199E07905F038FE8E
:10BA300010B91C4B019A5A611B48FFF70BFE1B48BB
:10BA4000FFF7AEFF6B788BB9A371194B5878FFF7EE
:10BA50005BFD3B685B6A0BB1114898476B7813B983
:10BA6000E07905F0AFFE0AB0BDE8F081FF23A371D5
:10BA7000EFE7104B01225A74227A9A74627ADA74D0
:10BA8000F1E76378002BEED00AB0BDE8F041FFF794
:10BA9000CFBB00BF44080020741200209012002089
:10BAA00060080020B412002064080020650800200F
:10BAB000781200203008002030B58BB0FFF767FF08
:10BAC0000446F0B903F0FCFE831C1DD0F8B9134DF9
:10BAD0002B685B69DBB1272368468DF8003002F0E4
:10BAE0006DF92B6801985B694FF4B961984703F0D1
:10BAF000F9FE78B92CB9094B1B68DB690BB1012041
:10BB0000984720460BB030BD6FF00704EFE74FF0C9
:10BB1000FF34ECE74FF0FF34F3E700BF741200206E
:10BB2000014B1878704700BFE8120020014B58788D
:10BB3000704700BFE812002070470000044B9A7A5B
:10BB40000AB101225A70034B5B6903B11847704771
:10BB5000E81200206C08002073B5224C6378002B9B
:10BB600033D008F03BF966680546FFF7D3FB06447F
:10BB7000AE4214D2A37A93B1E0228DF800208DF862
:10BB80000130217AE368019301226846FFF7F2FB56
:10BB900008B1073010D100236370A372656094F878
:10BBA0003430EBB1002384F834300F4B5B6BBBB106
:10BBB00002B0BDE87040184740F2DC510B4808F075
:10BBC000D9F90A4808F09CF9E8E794F83520002AEA
:10BBD000E5D094F8360084F83530FFF795FCDEE7C1
:10BBE00002B070BDE81200206C080020CC120020CA
:10BBF00037B5104D104CC8B1C1B16272012300229B
:10BC00002860E16023700D480D4B00924FF0FF312A
:10BC100008F0CAF800250B4825822022294605F0A5
:10BC20001DFE6570A574A58603B030BD00232B6092
:10BC30002370EFE7E4120020E8120020CC1200206D
:10BC40003DBB0008FC1200202DE9F0478E4C237804
:10BC50008CB0002B56D0C2780AB9837B13B1238AEB
:10BC600001332382437B002B4CD0E02A4AD10023AE
:10BC7000A372876897F80080B8F1220F27D8B8F12F
:10BC8000220F30D8DFE818F04100FB0052005A00C4
:10BC900061006E0075008E009D00B400C7002F008B
:10BCA0002F002F002F002F002F002F002F002F001C
:10BCB0002F002F002F002F002F002F002F002F000C
:10BCC0002F002F002F002F00C900D000D400B8F1A2
:10BCD0007E0F00F0CC80B8F17F0F00F0DF80B8F16C
:10BCE0007D0F00F0AB80A57A002D00F05B81674CE2
:10BCF000637A3BB94FF47A71204608F03BF920464D
:10BD000008F0FEF80CB0BDE8F087E36801220021DE
:10BD1000A2721970A37AE1689818A0720620C8541C
:10BD2000A37AE1689818A072CA54DCE7584B9B6A62
:10BD3000002BD8D0012102209847D4E77B7884F8E3
:10BD40003630012384F83530CDE704238DF80430F4
:10BD50007B78003B18BF012301A88DF8083002F062
:10BD600053F9C0E77878003818BF012002F098FE38
:10BD7000B9E7484E0FCE01AD0FC50FCE0FC596E8FF
:10BD8000070085E807007B780A2BACD8424A126886
:10BD90005268002AA7D00CA901EB830353F82C0C9E
:10BDA0009047A0E77878431E012B9CD83A4B013886
:10BDB0001B6818BF012020729B68002B93D0984706
:10BDC00091E7E26801230821A3721170627A057B72
:10BDD000A17AAA4228BF2A46934284D285685A1C77
:10BDE000EB5CE56801334E1CA6726B54D3B2EDE7F1
:10BDF000E3680122A27209221A70A37AE268218AFA
:10BE0000581CA072D154A27A238AE1681B0A501CE4
:10BE1000A0728B5467E7238265E705238DF8043011
:10BE200001A802F077FB5EE7194BDB6A98475AE7F7
:10BE3000194B78781B686075DB68BEE7037B072BBE
:10BE40007FF451AF06238DF80430B7F80130ADF818
:10BE500008307B793A791B0443EA0223FA781343CA
:10BE6000642253430393BB798DF81030D8E73B220B
:10BE700001A88DF804208DF8083002F0C5F80123E0
:10BE800084F834302FE700BFE8120020CC120020E5
:10BE90006C080020CC6C0108E41200202A2301A8C1
:10BEA0008DF8043001F08AFF94F80A90E6689DF856
:10BEB00008009DF809509DF80A709DF80BC09DF888
:10BEC0000D309DF80E209DF80F109DF80CE009F143
:10BED000010A84F80AA006F80980354E94F80A9001
:10BEE0003668D4F80C8009F1010A84F80AA096F8A3
:10BEF00003A008F809A094F80A90D4F80C8009F17E
:10BF0000010A84F80AA096F802A008F809A094F89B
:10BF10000A90D4F80C8009F1010A84F80AA096F876
:10BF200001A008F809A094F80A9009F1010A84F820
:10BF30000AA096F80080E66806F8098094F80A805E
:10BF4000E66808F1010984F80A9006F808C094F838
:10BF50000AC0E6680CF1010884F80A8006F80C7043
:10BF6000A77AE66807F1010C84F80AC0F555A57AAE
:10BF7000E6686F1CA7727055A07AE568461CA67229
:10BF80002954A17AE0684D1CA5724254A27AE16856
:10BF9000501CA0728B54A37AE268591CA17202F85B
:10BFA00003E0A0E6034807F05DFF6570AAE600BF66
:10BFB000E4120020CC1200207047000000487047B7
:10BFC0006C080020002070474FF0FF3070470000E1
:10BFD000044B054A93F81831022B18BF062382F848
:10BFE000903470478C190020501F0020034BD3F869
:10BFF000483313B15B6903B118477047501F0020E5
:10C00000034A137843F004031370FFF7EFBF00BF38
:10C01000341300201FB50A4B8DF8090093F87C20DB
:10C020008DF80A2093F88C2093F848000D3202A96D
:10C030008DF8082003F064FCC0B205B05DF804FB85
:10C040008C19002008B5074807F00CFF064B93F841
:10C050001A2412B1012283F81924BDE80840FFF721
:10C06000C5BF00BF50230020501F002010B50C4C4E
:10C07000D4F8403343F08003C4F8403394F81A34C2
:10C0800013B10020FFF7DEFF94F8913423F0120380
:10C0900043F0120384F89134BDE81040FFF798BFD5
:10C0A000501F00202DE9F041DFF8AC8098F81831DE
:10C0B000022B06460D4602D0284BDB6A984702F059
:10C0C000A6FD044628B1022002F097FD002002F0F0
:10C0D00099FD98F81831012B17D102F09AFD074607
:10C0E00030B1002002F08AFD002002F08CFD3C46B9
:10C0F00002F091FD48B1002002F081FD002002F025
:10C1000083FDBDE8F041FFF763BF002CF9D1144C6B
:10C1100094F8902494F81A34BAB90BB184F84164B5
:10C12000304602F017FFD8F82C0007F061FED4F873
:10C13000B4339842E5D30B4807F094FE94F8913459
:10C1400043F0100384F89134DBE70BB184F84154D9
:10C15000284602F0FFFEF1E78C1900205C7601080A
:10C16000501F0020E8220020074A10B5137843F042
:10C1700002031370FFF73AFFBDE81040034B0122A2
:10C180000021022007F042BB34130020296F010870
:10C19000074A10B5137843F008031370FFF726FF22
:10C1A000BDE81040034B01220021022007F02EBB06
:10C1B00034130020396F01082DE9F0410F4616466F
:10C1C0001D46804607F00AFE0B4A0C4C1378278167
:10C1D00023F0110343F01103C4E9000813706681D2
:10C1E0002573FFF703FFBDE8F041054B0122002155
:10C1F000022007F00BBB00BF3413002020130020E7
:10C20000496F010813B507F0E9FD0D4B6C46186046
:10C21000204607F037FD94E803000A4A0A4B83E8FA
:10C220000300137843F020031370FFF7DFFE074B82
:10C2300001220021022002B0BDE8104007F0E6BA5A
:10C24000301300203413002088220020566F01088C
:10C250002DE9F04192B0064602F0D9FC002840F0EA
:10C260005881AD4D95F81831012B09D02B6BAB4C93
:10C2700093B194F80431BBB1042B6FD0032003E0D9
:10C2800002F0C7FC18B10F2012B0BDE8F08102F037
:10C29000C2FC0028EAD0F6E7B5F82031D4F81C2417
:10C2A000013B53432B63E4E79D4803F060FA002809
:10C2B00040F0128194F80C3123802B6B0C930DF11C
:10C2C000180895F839308DF83830404695F81C310B
:10C2D0008DF83A3007F0FCFCD5F82831009302AF16
:10C2E00098E80600D5F82431384607F088FC97E82E
:10C2F00003000FAB83E80300EB6A0D9300238DF876
:10C3000044302388ADF8463095F8303101228DF85D
:10C3100039201BB98DF844208DF83930814B0093BA
:10C32000814B95F84800A3F179020CA903F05DFB5D
:10C33000C0B10B28A8D1D4F8941499B1002EA3D081
:10C34000D4F84033794843F02003C4F8403307F071
:10C3500011FE764807F0D4FD002095E7704803F001
:10C360003AFAA4E795F8487095F9693095F93920BB
:10C3700095F87D106E4E384603F044FB009641B2AE
:10C38000EB6C95F850203846183603F0DFFA00962B
:10C39000EB6C95F8502095F9701095F8480003F073
:10C3A000D5FAD4F8C413AB6DD4F8DC230B44C4F82D
:10C3B000B033EB6D1344C4F8B43394F80431042B58
:10C3C00007D02B6E0B44C4F8B0336B6E1344C4F823
:10C3D000B4330023089395F83031002B40D100236B
:10C3E0008DF8133095F839308DF8213095F83830C4
:10C3F0008DF82230D5F880300993D5F884300A932F
:10C400002388ADF82C3095F8303194F81B648DF802
:10C410002E3095F84800474B8DF820600DF113023F
:10C4200008A903F0A7FA012384F8413495F83930BC
:10C4300084F842349DF8133084F84334D4F81C3423
:10C44000C4F85064C4F84834C4F8583402F0E5FB2A
:10C45000C8B1D4F81C0402F0F2FBA0B1102013E71D
:10C4600008A802F0A7FC60B995F9390094F8376282
:10C470009DF82070FFF7CEFD3E44B042AFD20820B9
:10C4800002E7132000E795F81831012B01D102F0E3
:10C49000D8FB02F0C5FB0023059394F8043195F90D
:10C4A000395094F81B649BB1042B7FF4E7AE05A8C8
:10C4B00002F0B4FE58BB94F8183413B1059B013B4D
:10C4C0000593174B05983246E9B202F00DFF02E0E2
:10C4D000134802F0DDFE08B11120D5E6D4F8403350
:10C4E00094F80C11218043F00203C4F8403394F80F
:10C4F000183411480133DBB284F8183484F8453419
:10C500000E4B00259B6AC4F89854984724E71220E4
:10C51000BAE60E20B8E600BF8C190020501F00209C
:10C5200058200020BC190020E4230020B82200205D
:10C53000082300206C230020521F00205C76010895
:10C5400073B5134D134E0096EB6C95F8502095F98A
:10C55000781095F8480003F0F9F995F83031337503
:10C5600095F8480040F2012306F13C0231467382FF
:10C5700003F0F8F950B196F83C3086F88230064B5B
:10C5800000205B6B9847F37C86F8A83002B070BD42
:10C590008C190020382300205C760108F8B5324C55
:10C5A00094F81831012B05460ED0022B4ED0002BEB
:10C5B00057D138B9D4E91B0104F1740383E80300AF
:10C5C0000020F8BD012806D102F02CFB0028F8D18C
:10C5D00084F81851F5E7022843D1244E84F8180155
:10C5E00006F5747CBCE80F0006F57A770FC79CE867
:10C5F000030094F8E92094F8003187E8030086F8F6
:10C60000FB53D2B1022B18D1D4F804316367C6F8BA
:10C61000EC3394F87D3094F8082186F8F83394F8D8
:10C620008C3084F8782086F8F93396F81B2486F845
:10C63000E82340F20133A6F8FA33002386F81A34CF
:10C640000B4BDB6A9847FFF77BFFB9E748B9074B0D
:10C6500084F81801062283F89024054BDB6A98477A
:10C66000AEE70320ADE700BF8C190020501F00206B
:10C670005C760108F0B5504C504EB4F8DC202287AF
:10C68000D4E92D0194F8B12084F8692004F16C02FA
:10C6900082E80300D4E92F0104F1740282E8030068
:10C6A000B4F8C420A4F87C2091B0D4F8CC20D4F8FD
:10C6B000C810C4F884200025D4F8D020C4F88820FD
:10C6C0000123A4F82031C4F8801084F83051A56209
:10C6D00084F81B5184F83A5084F81D5184F81E5197
:10C6E000C4F83451C6F89854A6F8185486F81A5469
:10C6F000A4F838518DF8183004F50973039304F544
:10C700000A7394F84800049303A92D4B84F845510B
:10C71000C4E94F55A4F84651059303F0FFF8E36EC2
:10C72000C6F8D43394F87D3086F8E03394F88C3032
:10C7300086F8E1334FF48073A6F8E23386F8D053DD
:10C7400094F8303186F8E43306F574770FCF06F5A8
:10C750007A740FC497E8030040F2012384E80300D1
:10C76000A6F8FA33D6F8483386F81B54CDE90155BC
:10C770001BB15A685B6901920293124B0793A3F1B4
:10C7800048020892A3F1140209920F4A0B9229332E
:10C790000A93A2F19C030C93A2F198030D93131D2D
:10C7A0000E9301A902F14C0307A802F599620F93B9
:10C7B00002F022FA11B0F0BD8C190020501F0020A9
:10C7C00038130020B8230020701A0020F8B50D4F50
:10C7D0000D4E0C4607F046FB3B6B98470B4A96F80C
:10C7E0004800214603F0BEF850B1094D706D95F830
:10C7F000243485F86A347B6B9847E37C85F8903461
:10C80000F8BD00BF5C7601088C190020742300205D
:10C81000501F00200F4890F81B3480F8B8330E4B9F
:10C8200093F8692080F8BB2393F87D2080F8C82313
:10C8300093F88C2080F8C92393F8303180F8CC33FA
:10C840000022A0F8CA2300F56E7100F56070FFF7B2
:10C85000BDBF00BF501F00208C190020114890F868
:10C860009034EBB190F81B3480F8D0330E4BDA6E75
:10C87000C0F8D42393F87D2080F8E02393F88C202F
:10C8800080F8E12393F8303180F8E4334FF480727C
:10C89000A0F8E22300F5747100F56670FFF796BF0B
:10C8A000704700BF501F00208C19002070B5344C19
:10C8B0002421204604F0D4FF636A984218BF6062C6
:10C8C0004FF01C012F4814BF0125002504F0C8FFBC
:10C8D000636C984218BF60644FF480712A4818BF97
:10C8E00045F0020504F0BCFFD4F84831984218BF67
:10C8F000C4F848014FF0D401244818BF45F004059E
:10C9000004F0AEFFD4F82032984218BFC4F82002D9
:10C910004FF000011E4818BF45F0080504F0A0FFC5
:10C92000D4F82432984218BFC4F824024FF460713E
:10C93000184818BF45F0100504F092FFD4F8A83548
:10C94000984218BFC4F8A8054FF01401124818BF48
:10C9500045F0200504F084FFD4F8C03598420F4B11
:10C9600018BFC4F8C005D3F8483318BF45F04005D8
:10C970002BB11B691BB12846BDE87040184770BD3C
:10C980008C190020B4190020D4190020D81A0020D6
:10C99000B01B0020B41B0020381F0020501F0020B7
:10C9A0002DE9F04F8FB04FF00009012B06460F46DE
:10C9B00090468DF80D90ADF8109002D84C46BC42D0
:10C9C00002D30FB0BDE8F08F305D02F033FA20449F
:10C9D000B842F6DC335D651C023BEDB2112BF0D89A
:10C9E00001A252F823F000BF31CA00085BCA000858
:10C9F00059CB000881CB0008FFCB000825CC0008EC
:10CA00008BCC0008B3CC000839CD0008C3C900089E
:10CA1000C3C900088DCD0008C3C90008C3C90008F8
:10CA200035CE00085DCE000895CE0008C9CE0008BE
:10CA3000052002F0A7FA70B10521002002F068FA83
:10CA4000725DBA4BE51C0234E4B283F85C24325DBB
:10CA500083F85D24EDB22C46B1E700238DF80E304B
:10CA60008DF80F308DF814308DF81830B9F1000FB3
:10CA70006DD1AF4C4FF0050994F87C208DF8312032
:10CA80006B1E94F839208DF83320334494F8382005
:10CA90000B938DF8342094F81A3194F868208DF8AF
:10CAA0003520D4F82C218DF832300A9273B37B1CD8
:10CAB0005B1BDBB28DF8303006AB019305AB009306
:10CAC00094F848000DF10F030DF10E020AA902F0CF
:10CAD0005DFF8DF80D0000F00700072813D194F9D1
:10CAE00039209DF90E3084F839309A429DF80F3084
:10CAF00084F83830B8BF01229DF81430B8BF84F8EC
:10CB00001D2184F868304FF0000A09E00523D1E7C1
:10CB100001220DF10D01032002F0A4F80AF1010A2F
:10CB20005FFA8AF29DF81830B3FBF9F19142EFD821
:10CB30002B44DDB26B1EDBB29F420BD9F25C032AA1
:10CB40009AD0AF4288BF1D464FF0010983E70534F4
:10CB5000E5B2F9E71D46F7E7735D754903F00F038A
:10CB6000012281F81B31023402FA03F3A1F82031CB
:10CB7000E4B2002204A9042002F074F825466AE712
:10CB800007238DF80D30735DC3F3021203F00F031A
:10CB90008DF82830E31CDBB28DF82920F25C231DD0
:10CBA000DBB2651DF35C0234E4B21B0443EA0223EA
:10CBB000325D5F4C13436422534394F848000B9357
:10CBC0000AA902F0F2FE00F00703072BEDB28DF880
:10CBD0000D000CD19DF8283084F8703084F878303E
:10CBE0000B9BE36663679DF8293084F869308DF804
:10CBF0001000012204A9052002F034F82BE74B4B6A
:10CC0000D3F8483363B11B6853B1984708F03F032A
:10CC10008DF810008DF81130022204A90620EBE7F0
:10CC2000FF20F3E703238DF80D30735D8DF81C3082
:10CC30000AAB0693E31CDBB2A51DF25C231DDBB23D
:10CC400006A9F35C1B0443EA0223A21CD2B20534FA
:10CC5000B25C134364225343E4B20A9300230B9360
:10CC6000335D8DF83030324B93F8480002F0A3FE6C
:10CC7000C3B20028EDB28DF80D30FFF6ECAE8DF8A2
:10CC80001030012204A90720B6E7735D03F00F03FB
:10CC9000012B4FF47A7238BF01235343244A0234E4
:10CCA000936503F57A73D365E4B2002204A90820E2
:10CCB00062E7735D1E4DC3F340128DF8152095F8A1
:10CCC0004800C3F3001205A903F00F038DF81420E8
:10CCD0008DF8163002F075FE02340130E4B23FF4F4
:10CCE0004DAFBDF81430134AA5F87C309DF81630CE
:10CCF0009DF814A0D05CF5F70DF90223C5F880006B
:10CD00000AA995F848008DF828308DF82AA002F07D
:10CD1000F7FD95F93930069040B29842B8BF1846F1
:10CD200085F83900002204A9092025E7501F0020BA
:10CD30008C190020636F010803238DF80D30735D9B
:10CD40008DF82830E31CDBB2651DF25C231DDBB2DD
:10CD50000234F35CE4B21B0443EA0223325D134362
:10CD6000642253430B93644B0AA993F8480002F0E2
:10CD70002EFEC3B20028EDB28DF80D30FFF66BAE7B
:10CD80008DF81030012204A90A2035E7092002F0AD
:10CD9000F9F8DFF868B1002849D00921002002F035
:10CDA000B7F80023ADF81E30A31CDBB2F25CE31C25
:10CDB000DBB216F803A0735D4FEA0A4A4AEA022A78
:10CDC0004AEA030A231DDBB2A51D0534F35CE4B275
:10CDD0004AEA036A335D4FF47A7253430AAC1B127A
:10CDE0002046ADF81C3006F04DFF454B53440693EA
:10CDF000DBF83C3300930DF1180A9AE80600DBF8E3
:10CE0000383308A806F0FBFE099B009394E806005F
:10CE1000089B504606F0D8FE9AE8030006F00AFF89
:10CE200001F00AFF0123EDB28BF8383413E68BF8DA
:10CE3000380410E60C2002F0A5F800283FF40BAEF1
:10CE40000C21002002F064F82C4B93F89034043B42
:10CE5000012B7FF600AE01F0EBFEFCE5A31CDBB27C
:10CE6000725DF15CE31CDBB2651DF35C0434E4B27B
:10CE70001B04305D43EA012313436421594300F04E
:10CE80000F0001F0D6FEEDB28DF81000012204A9CA
:10CE90001120B1E60D2002F075F800283FF4DBAD5B
:10CEA0000D21002002F034F8A31CDBB2154AF05C1F
:10CEB000735D1268251D0334E4B243EA0020315D3E
:10CEC000EDB201F0B8FEC6E5725DA31C251D03346A
:10CED000DBB2E4B2F15C335D1B0443EA012313438C
:10CEE0006420584301F0A9FEEDB28DF81000012234
:10CEF00004A9132080E600BF8C190020501F0020D9
:10CF0000803DD512201300200E4B93F891249207F8
:10CF100003D593F88F24012A08D90B4991F81A21D7
:10CF200022B18A6A501C18BF01328A620022A3F81B
:10CF3000182483F81A24D3F8402322F00202C3F8FD
:10CF400040237047501F00208C19002070B5184CEA
:10CF50001848194D06F086FFD4F84033D4F89804E9
:10CF6000D5F8906023F02003C4F8403338B106F0C0
:10CF70003FFF864203D2002385F83A3070BD01207E
:10CF8000FFF766F90028F9D00B28F7D095F839306B
:10CF900084F84234092094F8183484F8453484F82D
:10CFA000410401F0D7FFBDE87040FFF7ADBF00BFFF
:10CFB000501F0020B82200208C190020094BD3F804
:10CFC0004023012A0AD008490978C90708D43AB988
:10CFD00093F89204013818BF012070470020704771
:10CFE00001207047501F002034130020034BD3F85A
:10CFF0004003431E58425841704700BF501F002055
:10D000002DE9F04FA9B0EFF3108272B6DFF8F0B25D
:10D010000021DBF80030CBF8001082F31088B94C07
:10D02000002B00F0E180DAB29B06039264D5B64D86
:10D0300095F81831022B02D0B44BDB6A9847EFF316
:10D04000108872B6B24F06F0C9FE3E68D4F8B0132D
:10D05000361A3144AF4806F08DFFAE4806F050FF57
:10D06000D4F8B413AC48314406F084FFAA4806F063
:10D0700047FF88F3108894F81A34002B00F06B8176
:10D08000152312A995F848008DF8483002F038FCB5
:10D09000D4F8B4130F900144A04806F06BFF9F48EA
:10D0A00006F02EFF3B6894F81B24EB620DAF384668
:10D0B0008DF870201D9306F00BFED5F828310093F3
:10D0C00006AE97E80600D5F82431304606F097FD05
:10D0D00096E803001FAB83E80300D4F81C341E93CA
:10D0E00095F8303195F84800003B18BF01231CA982
:10D0F0008DF8713002F00DFC039BDF0648D5824DA0
:10D10000DFF81CA2D5F8E42004929BF80020BAF9BD
:10D110000A809AF90C90A4F88C84002363F300022F
:10D120000A9384F84434A4F8223484F82534C4F8EB
:10D130002834A4F82C3484F82E34C4F8303484F81D
:10D140002034C4F8343484F83834C4F83C346F4B99
:10D150008BF8002094F89024DB6A84F88E9484F88D
:10D160008F24DAF80470BAF80860984794F88F347E
:10D1700013B9694806F076FE3146384601F045FDA0
:10D180008346002800F0EA80A4F87E8484F8809426
:10D19000039B19071AD55C4B93F81831022B02D068
:10D1A0005A4BDB6A98470220FEF712FF84F84104CD
:10D1B00001F0D0FE94F81A3413B1012384F8193425
:10D1C00094F8913443F0100384F89134039B5A0788
:10D1D00003D506210520FEF765FF039B9B0703D5BA
:10D1E00004210320FEF75EFF01F02DFD94F8912449
:10D1F000D7065FD5002384F89234D4F840331E0656
:10D2000044BF23F08203C4F8403312F0050F00F04E
:10D21000FB820B2001F0B6FE002800F0F58294F8A6
:10D220009134DD0700F1F082580740F10783D4F80C
:10D23000403323F00203C4F84033D4F8402382BBC8
:10D2400094F8915415F001011EBF2B4662F30003C0
:10D2500084F8913494F891345E0744BF6FF38203ED
:10D2600084F89134012384F8923421B1D4F8443302
:10D270002C481B6898476D070BD52B4801F08EFE94
:10D2800001F0BCFE28B194F8913443F0040384F813
:10D29000913401F0C6FC94F891346FF3041384F8D0
:10D2A0009134012384F8923494F8913443F02003AC
:10D2B00084F8913494F8913418070AD56FF3C303B6
:10D2C0001A4984F89134D4F84433A1F12400DB687E
:10D2D000984794F8913499070AD56FF3410313499D
:10D2E00084F89134D4F84433A1F16C005B6898471A
:10D2F00094F89034022B1BD1FFF722F918E000BFFD
:10D3000034130020501F00208C1900205C76010887
:10D3100030130020D0220020E822002050230020DB
:10D320002013002090230020A4230020DC230020D1
:10D3300094F891349A0640F1C4826FF3451384F84F
:10D340009134D4F84033002B40F0BB8229B0BDE8C3
:10D35000F04FFFF7ABBA84F84134A3E695F81831E3
:10D36000012B0CD101F055FC804668B1584601F004
:10D3700045FC584601F047FC042384F88F347EB9FD
:10D38000012384F821344FE101F045FC0028F6D058
:10D39000404601F034FC404601F036FC0523ECE742
:10D3A0003B7805935B09013B062B00F21782DFE80F
:10D3B00013F00700150295001502920015020602EF
:10D3C000102EDDD995F830311297F6B28DF84C60F9
:10D3D000002BD5D11CA804F055F912AA1CA9FF20D6
:10D3E00002F09EF89DF85830C3F3030307468DF80A
:10D3F0002C3095F8480095F87D308DF82D300722B7
:10D400000BA902F090FA002F5DD100285BD09DF8A7
:10D4100053309DF852201599C5F8E4101B0443EAD7
:10D4200002239DF8512002201343C5F8E03004F098
:10D4300037F99DF8583095F8480085F82E71C3F3F8
:10D440000212C3F3030385F8703085F878309DF835
:10D45000593085F86920012B38BF01234FF47A72C7
:10D460005343AB651344EB650DF15A034FF00108CC
:10D470001093113E94F81B348DF83C300FA985F8B9
:10D4800068808DF8446002F056FA0223404685F821
:10D49000303101F077FD18B14146384601F038FDD2
:10D4A00094F88F34012B00F2A78194F81A34002BE2
:10D4B00040F09A8194F8913443F0100384F8913449
:10D4C000FEF786FD64E6012001F05CFD0028E7D050
:10D4D00001210720E2E7012384F8203495F87D300C
:10D4E0008DF82E3094F824348DF82D3095F88C304A
:10D4F00095F848000D330BA98DF82C3002F000FA96
:10D50000A6F10D031BB2099023EAE37300B2834234
:10D510003FF736AF0B2E7FF633AFBA4B25931CA8DF
:10D52000FF231C978DF874608DF8983002F0C4F8D2
:10D53000074600287FF424AF95F81831012B13D14A
:10D5400001F067FB002872D0384601F057FB3846DF
:10D5500001F059FB04239DF87C101E9884F88F3449
:10D56000C1F3001101F06EFB9DF87C301E99C4F8E8
:10D57000341413F00F0203D09DF89000002862D1FC
:10D580009DF89800002861D0002A7FF4F9AE9DF83C
:10D590009020002A14BF4FF003084FF00208002229
:10D5A0000A92D5F8EC2095F8E900914251D1002873
:10D5B0004FD0D5F80C1195F8EAB009680A9195F8A2
:10D5C0001811022902D1032184F88F14B8F1030F36
:10D5D0007FF4D6AE13F0600F7FF4D2AE0492012731
:10D5E00095F82E31BBF1000F36D0BBF1010F13D1EE
:10D5F000012B33D16FF0090646FA08F606F0010652
:10D60000C6F10206F6B2BDF87E100AAA304601F055
:10D6100011FE38B3072823D0012384F821340A9B54
:10D62000C4F83034C4F86C34FEF720FDB0E501F0E6
:10D63000F2FA002898D0384601F0E1FA384601F0B5
:10D64000E3FA052387E74FF00008A8E74FF0010849
:10D65000A5E74FF0010BC3E70426D4E70326D2E782
:10D660000823DAE71CAB009304990A9B324658461C
:10D6700001F0A2FE20B1022814BF0B230A2380E68A
:10D680000A9BC4F83034C4F86C349DF87C3084F8BC
:10D690002104C3F3401384F82E3484F8443494F8FE
:10D6A0008F3484F82274012B9EBF0122A86285F872
:10D6B0001E21012FC4F8280484F82C0484F84104A6
:10D6C00038D1022284F8202495F83A20002A4AD141
:10D6D0009DF87C20D60646D4012B94F840149DF882
:10D6E0007C2005D8012901D1900601D501F04CFB21
:10D6F000B8F1020F94F88F3443D0B8F1030F0AD079
:10D700009DF87C10B8F1010F4A4601F00F0120A8E6
:10D710003BD0FFF745F99DF8903084F82334259BE2
:10D72000C4F828349DF8983084F82C34012384F808
:10D730002D3430E0059A02F0E002A02A1BD195F8C2
:10D740002E11012285F83A2009B927996963012B26
:10D7500084F8202407D9D5F89020C4F83C24DAF8BE
:10D760000020C4F8982495F81821002AB4D1012289
:10D7700084F82524B0E7002285F83A2084F8202494
:10D78000A6E79DF8981025984A46FFF709F99DF8F5
:10D79000903084F823349DF89020E02A08D195F841
:10D7A0001F312BB984F82324C4F82834A4F82C346E
:10D7B00094F8913443F0020384F8913470E6114DEB
:10D7C000013EB2B2791C284604F034F80323A4F8D1
:10D7D0002034C4F8285484F82C64E9E7012384F841
:10D7E0002134FEF743FC5BE694F84434002B3FF40D
:10D7F00061AE0020FEF726FC94F88F34022B3FF434
:10D800005FAE57E68821002094F89134590715D56A
:10D81000012001F0B7FB60B1012001F08BFB08B9DA
:10D8200084F81804D4F8403323F00203C4F84033DA
:10D8300004E0062001F0A6FB0028F3D194F891340F
:10D84000DA077FF5FAAC94F840240AB1032A18D11C
:10D850001D4A94F8181492F86820914205D29B074B
:10D8600023D594F88F34012B1FD8184806F0FAFA04
:10D87000D4F8403323F02003C4F84033FFF744FBCF
:10D88000DBE4012A11D194F81924002A3FF4D5AC25
:10D890000D4A94F8181492F868209142E5D29F0737
:10D8A00003D594F84434002BDFD194F89134002050
:10D8B0006FF3041384F8913484F81904FFF746FBDE
:10D8C000BBE429B0BDE8F08F8C190020B8220020FD
:10D8D0002DE9F04F89468DB090460746002800F0AC
:10D8E0008F81002900F08C810368002B00F0888173
:10D8F0004368002B00F084818368002B00F0808156
:10D90000C368002B00F07C81104601F0F5FF002871
:10D9100000F07881BD4CBE4D384601F0AFFA40F2C0
:10D92000C4520021204603F099FF40F21C5200210E
:10D93000284603F093FFB74BC4F82C3104F5097364
:10D94000089304F50A7300264046099308A9B24BD0
:10D9500084F848800A9384F8186184F88C608DF804
:10D960002C6001F0DBFF0F2306A994F848008DF826
:10D97000183001F0C5FF801B18BF01204FF00A0BC3
:10D9800084F81C0106A994F848008DF818B001F03D
:10D99000B7FF4FF0060A84F8DC0006A994F84800A7
:10D9A0008DF818A001F0ACFF102384F8DD0006A963
:10D9B00094F848008DF8183001F0A2FF1123C4F844
:10D9C0009C0006A994F848008DF8183001F098FFE3
:10D9D0001223C4F8A00006A994F848008DF8183066
:10D9E00001F08EFF1323C4F8A40006A994F84800A0
:10D9F0008DF8183001F084FF1423C4F8A80006A99C
:10DA000094F848008DF8183001F07AFF1623C4F816
:10DA1000AC0006A994F848008DF8183001F070FFAA
:10DA2000172384F8B10006A994F848008DF818303F
:10DA300001F066FF18230DEB0301C4F8B400C4F82D
:10DA4000BC0094F848008DF8183001F059FFC0B2BE
:10DA50001D2384F8B80084F8C00006A994F8480093
:10DA60008DF8183001F04CFF1E2384F8C40006A97D
:10DA700094F848008DF8183001F042FF1F2384F815
:10DA8000C50006A994F848008DF8183001F038FF59
:10DA90002023C4F8C80006A994F848008DF818306F
:10DAA00001F02EFF0B23C4F8CC0006A994F848001F
:10DAB0008DF8183001F024FF0C2306A9A4F8D0003B
:10DAC00094F848008DF8183001F01AFFD4F89C3013
:10DAD0006365D4F8A030A365D4F8A430E365D4F826
:10DAE000A83023664FF00108D4F8AC300590A4F8B4
:10DAF000D200636684F8B080C4F894B084F898A02B
:10DB0000C4F84CB084F850A084F8688084F81F8171
:10DB1000C5F84893FEF7AEFDC5F84473C4E90B663B
:10DB20003E4B84F8198185F89164C5F840833246EC
:10DB30004FF0FF31009605F55A7006F035F9384B75
:10DB4000009632464FF0FF3105F5607006F02CF973
:10DB5000344B009632464FF0FF3105F5667006F003
:10DB600023F902AF304B009632464FF0FF3105F5F6
:10DB7000806006F019F9384606F0AAF897E8030025
:10DB800004F5927383E80300284B294F1E60294B4C
:10DB9000C5F84C33284BC5F85433284BC5F85C33D3
:10DBA000274BC5F85033274BC5F8583305F553704C
:10DBB0003B68984704F5A67003F080FB20B111265E
:10DBC00030460DB0BDE8F08F204601F003FB002881
:10DBD000F5D101F039F8B8B91B4801F04DFB064604
:10DBE0000028ECD17B69984703F002FEBB6D94F8E6
:10DBF00019019847FB6A9847012385F89234DFE7BB
:10DC00000326DDE70926DBE71326D9E78C19002078
:10DC1000501F002000040001381300204DCF0008E1
:10DC200015C800085DC8000845C00008341300206E
:10DC30005C76010805C20008B9C1000801C00008EF
:10DC400091C1000869C10008741A002008B5034B8F
:10DC50000020C3F84003FEF7BBF908BD501F0020A9
:10DC600010B5FFF7ABF90A4C60B90A4B93F81831BD
:10DC7000022B02D1084BDB6A98470123C4F84033DA
:10DC8000002010BDD4F84003013818BF0120F8E788
:10DC9000501F00208C1900205C76010838B5124C0A
:10DCA000204606F0DFF804F1180006F0DBF804F176
:10DCB000300006F0D7F804F1980006F0D3F800F031
:10DCC000AFFF0A4B0025DB6A984744F8285CFEF753
:10DCD000EDFD0749074840F2C45203F0ABFD0123B4
:10DCE00044F8283C284638BDB82200205C7601085C
:10DCF0008C190020C813002070B52E4B8AB0054641
:10DD000093F8DD008DF8090093F8DC008DF80A0027
:10DD100029489A6A90F81804039200268DF80B009F
:10DD200004960C46002940D00692D3F8882007922A
:10DD30001A8F93F81A118DF8151052BAADF82020E9
:10DD400093F87C2093F848308DF8243003AB8DF89D
:10DD500022008DF8232000930DF10A020DF10B0330
:10DD60000DF1090105A88DF8146000F0D7FE9DF9AA
:10DD70000900FEF74FF9607004A801F01BF8B0B974
:10DD8000049A0F2A0DD863789A420AD81544AB42F8
:10DD9000A3EB02012CBF002001202170C0000AB0BB
:10DDA00070BD002323700820F9E70320F7E7132054
:10DDB000F5E700BF8C190020501F00201FB5044656
:10DDC000002800F010810378412B00F20781DFE882
:10DDD00013F0420049004D005100550059005E000B
:10DDE0000501050105010501050105010501050103
:10DDF000650069006D0078007F00820085008A0060
:10DE000088008C0090009300960099009C009F0071
:10DE1000AE00B200BA00B600BE00C100C500CE0020
:10DE2000CA00CC000501D20005010501050105016C
:10DE300005010501050105010501050105010501B2
:10DE4000050105010501DA00DE00E200E700EB0054
:10DE5000EF00F300FC00664B93F8183123710020AB
:10DE600004B010BD624B93F83031F7E7406803F01F
:10DE7000C3FBF4E7406803F005FCF0E75C4B93F864
:10DE80001A31EBE75A4BD3F8E0306360E7E7584BC1
:10DE9000011D93F8300103F00DFCE0E7544B93F8BB
:10DEA0001931DBE7524B93F88C30D7E71C238DF800
:10DEB00008304F4B02A993F8480001F021FD606043
:10DEC000CDE74C4B043493E8030084E80300C6E735
:10DED000494B0434F7E7494B0434F4E7484B043426
:10DEE000F1E71A23E3E71923E1E7414B93F86830A0
:10DEF000B4E73F4B5B6DC8E73D4B9B6DC5E73C4BC3
:10DF0000DB6DC2E73A4B1B6EBFE7394B5B6EBCE77C
:10DF100002238DF80830364B02A993F87C2093F841
:10DF200048008DF80A2001F0EBFC207197E7304B98
:10DF300093F8DD3092E72E4B93F839308EE72C4B77
:10DF400093F8DC308AE72A4B93F8383086E7284B81
:10DF5000DB6C9AE7264B93F850307FE7244BD3F8DD
:10DF6000843063607BE7224B8FE7264B8DE7204BA5
:10DF7000D3F8CC30F5E71E4BD3F82C31436001F0D9
:10DF80004DFDA0606BE71A4BD3F890307DE7184B3E
:10DF900093F81F3162E7164BB3F88830A3805EE731
:10DFA000134BB3F88A30F9E7114BB3F8D030F5E7EB
:10DFB0000F4BB3F8D230F1E70D4B93F848200AB17C
:10DFC000062A12D1B3F8A035E8E7094B93F84820A8
:10DFD0000AB1062A09D1D3F8A43556E704B0BDE842
:10DFE000104000F021BE03203AE7182038E700BFB8
:10DFF0008C190020F8190020401A0020001A002077
:10E00000481A0020C81300207FB5044610B9032029
:10E0100004B070BDA34DD5F840339A0700F16F826C
:10E020000278412A00F26882DFE812F042004700DD
:10E0300055005B005F006400690076008100870086
:10E040008D00930099009F00A500AB00B50066020B
:10E05000BA00DC00EF0016013801290142014B0132
:10E060004F01530157015B0166025F017101990184
:10E070008701AB01B101B801BD01C20166022802EE
:10E080006602660266026602660266026602660250
:10E090006602660266026602660266026602660240
:10E0A000340239023E02430248024D0252025C022F
:10E0B0000079FEF773FA30B1AAE70379022BA6D0F4
:10E0C000794A82F8303195F8913443F0200385F88D
:10E0D000913400209CE7406803F080FA0028F2D0D9
:10E0E00095E7406803F0BEFAF8E76F4B027983F8D2
:10E0F0001A21E8E76C4B4268C3F8E020E3E76A4E78
:10E10000416896F8300103F0CBFA00287FF47FAF26
:10E110006368C6F8E430D6E7416800293FF477AF7A
:10E12000002001F0DDF90028CDD0112070E7416812
:10E1300000293FF46CAF0120F3E7416800293FF468
:10E1400066AF0820EDE7416800293FF460AF092081
:10E15000E7E7416800293FF45AAF0C20E1E7416846
:10E1600000293FF454AF0D20DBE7416800293FF45C
:10E170004EAF0E20D5E7416800293FF448AF0F208D
:10E18000CFE74A4C484B007983F81901A36D9847B3
:10E19000E36A984797E7444B027983F88C2092E72B
:10E1A000414E037A8DF8043096F8480096F87D3099
:10E1B0008DF80530072201A901F0B5FB00283FF4D6
:10E1C00026AF636896F848000193002201A901F088
:10E1D000AAFB00283FF41BAF6C36D4E9010186E8A6
:10E1E000030070E7304E037A8DF8043096F848004B
:10E1F00096F87D308DF80530072201A901F093FBD8
:10E2000000283FF404AFB436E7E7274E037A8DF8D1
:10E21000043096F8480096F87D308DF805300722D6
:10E2200001A901F080FB00283FF4F1AED4E901011F
:10E2300006F1740383E8030096F81831022B7FF48B
:10E2400042AF96F83031002B3FF43DAF174BDB6AFD
:10E250009847FEF775F936E7134E037A8DF80430C8
:10E2600096F8480096F87D308DF80530072201A910
:10E2700001F059FB00283FF4CAAEBC36ADE7436855
:10E28000029301238DF80C30074B02A993F8480044
:10E2900001F056FB00287FF416AFB8E643680293FE
:10E2A0000023EFE7501F00208C1900205C76010846
:10E2B00003795A1E0E2A3FF6AAAE934A82F86830B6
:10E2C00001E7914B42685A65FDE68F4B42689A65BB
:10E2D000F9E68D4B4268DA65F5E68B4B42681A66C3
:10E2E000F1E6894B42685A66EDE6874C037994F86B
:10E2F00048008DF80430062201A901F014FB002823
:10E300003FF485AE9DF8043084F8DD30DBE67E4CCA
:10E3100003798DF8043094F8480094F87C308DF837
:10E320000630052201A901F0FEFA00283FF46FAE85
:10E330009DF8043084F83930C5E6734C037994F8BD
:10E3400048008DF804300A2201A901F0ECFA0028F7
:10E350003FF45DAE9DF8043084F8DC30B3E66A4CDF
:10E36000037994F848008DF80430092201A901F0DE
:10E37000DAFA00283FF44BAE9DF8043084F83830C8
:10E38000A1E6614B4268C3F89420DA649BE65E4BD9
:10E39000027983F8982083F8502094E65A4B42681B
:10E3A000C3F884208FE6584B4268C3F8CC208AE635
:10E3B000012B40F0A480554C2421204603F050FA54
:10E3C000636A984201D0172022E61C2104F128003C
:10E3D00003F046FA636C9842F5D14FF4807104F172
:10E3E000480003F03DFAD4F848319842EBD1D421EB
:10E3F00004F5A67003F034FAD4F820329842E2D142
:10E40000002104F5097003F02BFAD4F82432984265
:10E41000D9D14FF4607104F50A7003F021FAD4F8F1
:10E42000A8359842CFD1142104F2AC5003F018FA69
:10E43000D4F8C0359842C6D1334E2146304640F21A
:10E44000C45203F0F7F9204640F2C452002103F011
:10E4500005FA95F81B3485F8E833736FC5F8EC338B
:10E4600096F87D3085F8F83340F20123A5F8FA33A9
:10E47000274B96F819019B6D984724E68379012B69
:10E480003FF6C5AD204B42684068C3F82C2100F030
:10E49000BDFE48E61C4B4268C3F8902013E61A4BB9
:10E4A000027983F81F210EE6174B8288A3F8882093
:10E4B00009E6154B8288A3F88A2004E6124B82886D
:10E4C000A3F8D020FFE5104B8288A3F8D220FAE50C
:10E4D0000D4B93F848200AB1062A12D1A288A3F85E
:10E4E000A025F0E5084B93F848200AB1062A08D188
:10E4F0006268C3F8A425E6E500F098FBDBE501209F
:10E5000086E5182084E500BF8C190020C813002080
:10E510005C7601082DE9F04387B00023ADF80030A8
:10E520000646002800F0EE800361FEF747FD20B1AB
:10E530000124204607B0BDE8F08300F065FD002807
:10E54000F6D100F05BFD014618B96F48142203F0C4
:10E5500085F96E4D95F89134012243F0040385F856
:10E56000552485F8913433788DF804300021013B2F
:10E570008DF80520ADF806100C2B00F2BB80DFE80B
:10E5800003F007B9B9B97982B9B990B9AD9AA900C0
:10E59000D5F8407317F02007CAD196F80480B8F177
:10E5A000020F46D1DFF868815A4CFEF763F896F9FE
:10E5B000051098F848003A4601F00FFA88F839003B
:10E5C000B37988F83830384607238DF80530FDF7E1
:10E5D000E5FFFF2304F58670A5F80C31C5F8084166
:10E5E00085F8047103F04EF804F58A7003F004F81E
:10E5F0003846FDF72DFE0446002839D096F905105F
:10E6000098F84800012201F0E8F988F83900D5F8B7
:10E6100094343361002C71D000F0F0FC002888D1D4
:10E6200095F8913485F81A0460F3820385F89134E3
:10E630007FE7B8F1010F4FF00204E8D1DFF8D09086
:10E640008DF8144099F8480089F81D7102A901F06D
:10E6500065F9337989F830318DF805708DF80680C9
:10E66000FDF7C4FC95F8913443F0100385F891341C
:10E670000024CCE700226946022000F0F3FA0028CB
:10E68000F6D01324C3E7244BB288DB6B96F90C1049
:10E69000B0689847D5F8403343F00203C5F84033DB
:10E6A000E6E702A90D2000F053FB0028E0D000228D
:10E6B00069460D20E1E7164B93F81831D3B9347948
:10E6C00004F0070000F0ABFA8DF800400122694623
:10E6D0001020D2E7002269461220CEE78DF80720ED
:10E6E00000F08EFA044638B900F087FA204600F0B0
:10E6F00089FABDE702248AE7012488E701A800F02F
:10E70000D1FB16E7032414E7A4230020501F0020A8
:10E710008C190020521F00205C7601082DE9F04F73
:10E7200099B08046059118B9032019B0BDE8F08F63
:10E7300000230361FEF742FC0446002840F0A58058
:10E7400046460FCE0EAD0FC51422524898F800A0D1
:10E75000B8F80C7098F90EB04F4E214603F07EF8D1
:10E760004E4B012283F8412496F83021022A254697
:10E770000BD196F81821022A07D196F81E2122B94A
:10E78000BAF1010F38BF4FF0010ABAF1010F2BD0D7
:10E79000BAF1030F2AD0BAF1000F33D102229DF84B
:10E7A0003C30DDF84090029362F34715012496F85F
:10E7B0007C108DF8321002220CA996F848008DF8D2
:10E7C000302001F09DF896F81A3196F830C196F88D
:10E7D0001D1140B2002B63D0BCF1010F57D10029AD
:10E7E00055D1002C61D153E00422D8E70023DDF895
:10E7F0003C90BDF840709DF942B0029365F01F0552
:10E800000124D4E74FF0000BD946CDF808B0CEE78D
:10E810004FF0010084F81A04D2E005F29A420BA9E5
:10E8200000F0D4FA002800F015811320049B3387F0
:10E830001A4B002283F81A2423E105F29A452A464E
:10E840000BA900F0C3FA0028EFD10B9B84F8280134
:10E85000C4F82C5184F83031FCE0B9F1000F00F01D
:10E86000F980002A00F0F6804946E01C02F0E2FF41
:10E8700094F8373201332380ECE01220D6E70220EF
:10E88000D4E70720D4E71320D2E701204DE7FCB9F5
:10E890000220F6E0902300208C190020501F002059
:10E8A000002CF5D05845B8BF584696F87C308DF806
:10E8B0002000052296F848008DF8223008A901F0C2
:10E8C00032F800283FF430AF9DF8203086F8393018
:10E8D0006F4A704BD2F89804D3F8904038B105F0E5
:10E8E00087FA6C4B84423CBF002283F83A20198F90
:10E8F0001A8F93F830010491996A099152BA00284D
:10E90000BFD093F81B0100B9186393F81801ADF854
:10E910005820013893F87C2093F81A411491D0F1D3
:10E92000000BD3F888108DF85B204BEB000B93F8AD
:10E93000482093F83A0093F868308DF85A3009ABC4
:10E940000093554B03904FF001008DF84C0015914A
:10E950008DF85C20A3F12F01A3F1300213A88DF8EC
:10E960004D4000F0DBF8039B4FEA0B1B4BEA431BC7
:10E9700000264BEA801B4BEAC413B145444C039379
:10E9800008BF37463A46494604F59C70CDE90A6609
:10E990009B46268084F81A6402F04CFFE9B2A57009
:10E9A000C5F34215FAB2042D3A4E039B84F8372280
:10E9B0003FF42EAF072D3FF450AF022D7FF45FAF31
:10E9C000364D84F80D110420029984F80401FF20CB
:10E9D00084F80C0184F8281184F81431D6F8E41076
:10E9E000C4F8085105F59B730AA8C4F8101184F8FF
:10E9F0003021C4F82C3100F011FC00287FF43DAF29
:10EA00000A9BA4F844040BA8A4F81631C4F84C34AB
:10EA100000F0D0F900287FF408AF0B9BD3B196F932
:10EA20003900FDF7F7FA94F83732002B3FF405AFC1
:10EA30000B9B0F2B3FF6F1AE05F58B720BA90F2048
:10EA400000F0C4F900287FF4F0AE0B9B63F3030BD6
:10EA500084F814B10598FDF7FBFB00287FF4E6AEBF
:10EA6000099B86F83A00B36200F080F900287FF431
:10EA70000AAF94F8913484F840A443F0010384F879
:10EA80009134034BD3F89434C8F810304DE600BFEE
:10EA9000501F00208C190020F4190020521F002064
:10EAA00037B50B4D8DF8040004460F2295F8480049
:10EAB00001A900F038FF40B1064A85F81C4192F8E0
:10EAC000913443F0200382F8913403B030BD00BF8D
:10EAD0008C190020501F002010B5FFF7C1F8044624
:10EAE00088B90A4805F0BEF9094805F0BBF909489C
:10EAF00005F0B8F900F094F8FDF7BCFD064BDB6AB1
:10EB00009847204610BD0124FBE700BFB822002033
:10EB1000D0220020E82200205C7601082DE9F04F89
:10EB20008BB047780093149B90F90C8090F90D609E
:10EB300090F80EB08A464168196004469146002F4D
:10EB400058D002238DF8103004A9C37B007C8DF8C7
:10EB5000123000F0D5FEB4F808C0618943B2606895
:10EB6000984545466144B8BF1D46604534BF0027FF
:10EB70000127884209D30A218DF81010207C0193C7
:10EB800004A900F0BDFE019B46B2B4F808C060893C
:10EB900061680CEB400E714519D3A1EB0C01B1FB80
:10EBA000F0FC00FB1C1191B9984503DC2378CBB92C
:10EBB0004FF0010B21238DF81030207CE37B8DF882
:10EBC000115004A98DF8123000F09AFE45B2009B56
:10EBD0008AF80050384689F8006083F800B00BB01E
:10EBE000BDE8F08F0223207C8DF8243006A900F0C8
:10EBF00095FEDDE74546EAE7704770477047704786
:10EC00000020704770477047704700207047002011
:10EC10007047002070470020704700207047704701
:10EC200070477047022070470220704702207047EB
:10EC300070470020704770477047002070470020E1
:10EC4000704770477047704710B5054C4FF403721A
:10EC50002046002102F002FE0020C4E9000010BDA1
:10EC60006C2400202DE9F8438146904600293CD0D1
:10EC70001F4C2023224604F1100012F8017F6FBBC5
:10EC80008242FAD11B4E3368013403B93460736891
:10EC900003B11C6000252560C4F8088074601FFA69
:10ECA00088F284F80490601D02F0C4FDB9F1110FE0
:10ECB0004FF0000398BF104D6373D6F8083298BF29
:10ECC00025FA09F503F1010398BF05F00105434456
:10ECD0002573C6F808323846BDE8F883013B13F0C7
:10ECE000FF030446C6D10227F5E70127F3E700BF7B
:10ECF000732400206C2400202007020010B518B3F4
:10ED0000124A1368984204D103681360002305E097
:10ED10000B46002BFAD019688842F9D15168884215
:10ED200008BF53600BB101681960D2F808328168DE
:10ED3000013B00245B1A04602146C2F8083210220D
:10ED400002F08CFD204610BD0120FCE76C24002061
:10ED5000054B1B6813B11A798242FAD1002B0B6064
:10ED60000CBF0320002070476C24002010B5054B19
:10ED7000186800B910BD037B04680BB9FFF7BEFF2C
:10ED80002046F6E76C24002038B5084B084C18687C
:10ED900000B938BD03790568112B05D824FA03F3AF
:10EDA000DB0701D5FFF7AAFF2846F1E76C24002016
:10EDB0002007020028B1044BD3F80832036000207A
:10EDC00070470120704700BF6C2400202DE9F041FE
:10EDD00007460E46154642B339B3154B1C6800234F
:10EDE0002CB93046FFF7E6FF0020BDE8F081A268AD
:10EDF000F91A0132914215D32279EA54581C22891A
:10EE00005FFA80F8611D55FA80F002F013FDA368E7
:10EE1000246898445FFA88F3E2E720462568FFF704
:10EE20006DFF2C46002CF8D1DBE70120DDE700BFA9
:10EE30006C2400200238C0B211289ABF014B185C24
:10EE400000207047736F010830B50B4B93F82020FA
:10EE50000446084672B100211C330578A54208D04B
:10EE600001319842CDB214BF04301038AA42F4D810
:10EE7000002030BD1046FCE77826002010B5084C75
:10EE800000232060142204F10C00FF2184F82030BC
:10EE9000C4E9010002F0E2FC012384F8213010BD36
:10EEA0007826002010B50E4A92F82010042915D8B3
:10EEB000936804781C7044785C70C478807898708B
:10EEC0000131DC7082F8201002F11C018B4214BF6A
:10EED000043302F10C039360012010BD0020FCE715
:10EEE00078260020094B93F8200068B15A6803F196
:10EEF0001C018A4200F1FF3014BF043203F10C02FE
:10EF000083F820005A600120704700BF7826002057
:10EF100010B5074B93F820200446084632B15968D3
:10EF2000FFF792FF10B101234470837010BD00BF42
:10EF30007826002008B5064B93F820202AB159689E
:10EF4000FFF782FF08B1407808BD0120FCE700BF51
:10EF50007826002030B50A4A92F82010536882F8CB
:10EF6000210061B1916801241C32DD78587005B927
:10EF70009C70934214BF0433103B9942F5D130BDCD
:10EF80007826002008B5044B5968FFF75DFF00386C
:10EF900018BF012008BD00BF78260020F7B5042265
:10EFA000154E044600210DEB020096F8207002F089
:10EFB00055FC0025EBB29F4201D803B0F0BD736849
:10EFC000197821705A786270987838B13368204681
:10EFD0009B689847FFF786FF0135EBE7DB788DF8F4
:10EFE00004108DF805208DF80730FFF77BFF01A88E
:10EFF000FFF758FFF0E700BF78260020014B93F899
:10F000002000704778260020034B93F82000042846
:10F0100094BF002001207047782600201FB50024EF
:10F02000CDE90244C41F8DF800408DF801100C0A90
:10F03000ADF80420090C120C8DF803108DF8062091
:10F040008DF8073002461B0A012168468DF8024000
:10F050008DF8083002F05DFA002818BF0E2004B0C9
:10F0600010BD2DE9F04188B090460D460F9A074635
:10F07000002847D000240121CDE904448DF8101068
:10F080009DF838108DF81510ADF81630190CCDE933
:10F0900000441B0ECDE902448DF81930ADF81A205A
:10F0A000130C120E07948DF818108DF81C308DF883
:10F0B0001D20E3B21E01002DF6B203DC002008B0D3
:10F0C000BDE8F081013310218DF81F3042466B46B8
:10F0D0000DEB010002F0B3F90346A8B9102D284644
:10F0E0003E44A8BF10206946327811F801CB0133A5
:10F0F00082EA0C02984206F8012BF5DC103D2DB295
:10F100000134D6E70920DAE70E20D8E701380328D2
:10F1100015D8DFE800F002080C100A4B1B681B69C9
:10F120000B6000207047074B1B685B69F8E7054BD5
:10F130001B689B69F4E7034B1B68DB69F0E705205C
:10F14000704700BF9C2600202DE9F041C4B00C465A
:10F150004A9E17461D468046B8B3B1F5807F36D823
:10F160004FF488720021684602F078FB492300932F
:10F170004FF48073ADF804302B0C8DF80830330C4D
:10F18000ADF80650ADF80A608DF80C302246002329
:10F19000414604A82D0E360E8DF80E308DF809501C
:10F1A0008DF80D608DF80F4002F044FB04F1100162
:10F1B0004B9A3B4689B2684602F02BF910B1012800
:10F1C00018BF0E2044B0BDE8F0810920FAE70D20F9
:10F1D000F8E7000010B590B10A4C28220021206009
:10F1E00002F03CFB2368084A1A6000204FF0FF320F
:10F1F000C3E90302C3E90522C3E9072210BD0820C1
:10F20000FCE700BF9C26002000010101024B1B68A7
:10F2100018600020704700BF9C26002030B1044BCE
:10F220001B68DB68013303600020704709207047CA
:10F230009C26002013B500230C460193CAB101A9F6
:10F24000FFF764FF18B9019B591C02D1146002B08A
:10F2500010BD99B2611A002901DD5C18F6E702D1F0
:10F2600013600720F3E71B0C1B0403F580331C44D9
:10F27000ECE70920EBE7000028B1044B1B681C33C6
:10F280004362002070470920704700BF9C26002081
:10F290001FB5044600B3002303A8039302F090F9BE
:10F2A000104ABDF80C30126820469380E38200F0CB
:10F2B0005EFA98B904F11803009321680123132220
:10F2C00002F09CF860B9204600F051FA003818BFEF
:10F2D0000120000104B010BD0920FBE71020F9E770
:10F2E0000E20F7E79C260020F0B5054687B01C46A7
:10F2F00013B9092007B0F0BD2E4E3368DB68834296
:10F3000055D894F82020002A0CBF082209228342F5
:10F3100005D3204600F05FFA68B11020EAE7002329
:10F3200001900093A36894F82810606AFFF799FE93
:10F330000028EED0DEE723792168B4F808C0A7687A
:10F34000043B9AB20029D4D0B2F5807F2DD8ADF815
:10F350000EC08DF817304FEA174C04F12C033F0E06
:10F360008DF8117000932F0C08234FF0490EADF863
:10F370000C008DF814708DF816002F0E0DEB0300A5
:10F38000CDF808E08DF810C0ADF812508DF815706A
:10F3900002F034F808B10E20ACE7204600F01BFA6A
:10F3A0000028BAD13368DD60A4E70D20A2E706206B
:10F3B000A0E700BF9C2600202DE9FF410A9D804662
:10F3C0000F4616461C46002D5AD0002303A91046AE
:10F3D0000393FFF79BFE18B1062004B0BDE8F0814F
:10F3E000039B9C4201D80133F6D1284600F064F912
:10F3F000002847D1264B1A78424503D01A79424556
:10F4000042D10120AA68BA4240D103EB8002EB6AE4
:10F4100092F801802979CDE900430439927828686F
:10F420003B4689B2FFF790FE0028D6D195F82030F0
:10F430000194002B4FF00103009314BF42460822B1
:10F4400095F82810686A3B46FFF70BFE0028C4D1E8
:10F45000013E032EC1D8DFE806F002070B0F0D4B6B
:10F460001B681C611C62B8E70A4B1B685C61F9E70A
:10F47000084B1B689C61F5E7064B1B68DC61ACE739
:10F480000920AAE70F20A8E70B20A6E70220A4E79F
:10F49000A40800209C2600201FB50B294FF0000374
:10F4A000CDE90033CDE902330A4607D00C2914D048
:10F4B0000A2910D00A2005B05DF804FB012802D10A
:10F4C00020238DF800300021684602F022F8002841
:10F4D00018BF0E20EFE73023F3E70B21F4E700001D
:10F4E00038B5054602F010F8044610B10E24204647
:10F4F00038BD002DFBD1094B1B680B219878FFF715
:10F50000CBFF0028F2D10C21FFF7C6FF0028EDD178
:10F510000A21FFF7C1FF0028E9D0E7E79C26002079
:10F520002DE9F04380468FB00C461746002A6BD079
:10F53000002969D0002529461D2206A8059505F059
:10F5400004FC8DF81350344D2B680DF114099E887E
:10F55000CDF804900DF1130302933B7900933B68BF
:10F5600032462146404601F0F0FF00284ED138686F
:10F570003A79494602F05EF9384600F04FF8002823
:10F5800046D13C7AFA79BB79240444EA02241C432C
:10F590002B689A6894423DD99C609DF813000B211A
:10F5A000FFF77AFF034658BB0C21FFF775FF0346B0
:10F5B00030BB0A21FFF770FF034608BB7B7ABA7A9B
:10F5C000FF7A3F0447EA02271F433A463346214663
:10F5D0000920FFF723FD034690B933463A462146FA
:10F5E0000820FFF71BFD034650B92A689DF8131049
:10F5F00091700021D1604FF0FF31C2E90411916197
:10F6000018460FB0BDE8F0830923F9E70E23F7E7AA
:10F610000F23F5E70323F3E79C26002010B50446EB
:10F62000002845D00168002942D011F8013B437100
:10F630000322063002F0FEF82046032250F8091B90
:10F64000043102F0F7F82168CB79E3600A7A43EAE3
:10F650000223E3604A7A43EA0243E3608A7A43EA98
:10F660000263E360CB7A23740B7B63742379212BD1
:10F670001AD110220D3104F1120002F0DBF81D2224
:10F680002168501C8B5C6362085C43EA0023901C79
:10F690006362085C033243EA004363628A5C43EAC4
:10F6A00002636362002010BD112B03DC0D22E7E72B
:10F6B0000220F8E70120F6E710B50446002854D0F0
:10F6C0000168002951D00B7843714B7883608A78A8
:10F6D00043EA02238360CA7843EA024383600A79DB
:10F6E00043EA026383604B7903738B79C381CA79E0
:10F6F00043EA0223027BC38102F00F02083110307B
:10F7000002F098F8237B002203F00F0384F82020F6
:10F7100084F82820227903F10800111A04290DDD4C
:10F7200021680933043AD21A085C84F82000D2B266
:10F73000606A84F82820194402F07CF82379226852
:10F740001A44002012F8043CE36212F8031C43EA56
:10F750000123E36212F8021C43EA0143E36212F858
:10F76000012C43EA0263E36210BD0220FCE710B5FE
:10F77000044660B3036853B30279162A29D9427943
:10F780001A700146082251F8060B013002F05CF8AD
:10F790002146082251F80E0B093002F055F8236873
:10F7A000E28A5A74E38A22681B0A93742368A26966
:10F7B000DA74A36922681B0A13752368628B5A7571
:10F7C0002368E27E9A7517232371002010BD012063
:10F7D000FCE70220FAE738B50446002863D0016848
:10F7E000002960D0037B90F8282003F00F03002A43
:10F7F00057D10833207904321344984255D36379A2
:10F800000B702368A2685A70A36822681B0A937061
:10F8100023686289DA702368E27A1A712368227B8E
:10F820005A712368E2899A71E38922681B0A21468A
:10F83000D371227B51F8100B02F00F02083001F057
:10F84000F9FF237B94F8282003F00F0303F1080548
:10F850002AB1226894F82010515503F10905206857
:10F8600094F82820616A284401F0E4FF94F82830D5
:10F870002268E16A2B44D1545A1CE16A206892B292
:10F88000090A81549A1C2168E08D92B28854DA1CCE
:10F89000216894F82F0092B2043388542371002019
:10F8A00038BD0933A6E70120FAE70220F8E7000097
:10F8B000024B1A8810431880704700BFA026002012
:10F8C00008B5074B1B883BB1FEF7CAF9002814BFE7
:10F8D0006FF00200002008BD6FF00100FBE700BFE1
:10F8E000A026002010B5034B00241C80FEF7AEF9C3
:10F8F000204610BDA0260020B0FA80F040097047D5
:10F9000082B018B9084602B000F0CAB8002002B0B0
:10F91000704710B9084600F077B9704710B908462B
:10F9200000F08EB970470346084611460BB900F047
:10F93000E5B90020704710B9084600F06DBD70476A
:10F9400010B9084600F006BA0020704710B404460B
:10F95000084611461A46019B14B910BC00F014BAAF
:10F9600010BC70470346084611460BB900F03EBA7A
:10F970000020704710B40446084611461A4614B9D0
:10F9800010BC00F0ABBA002010BC704730B4054684
:10F99000084611461A46DDE902341DB9029430BC0E
:10F9A00000F02ABB002030BC704710B9084600F0B8
:10F9B000DBBB0020704710B9084600F06BBD00208B
:10F9C000704710B9084600F0EABB0020704710B934
:10F9D000084600F0E7BB0020704703460846114682
:10F9E0000BB900F001BC0020704710B40446084673
:10F9F00011461A46019B14B910BC00F0F7BB092050
:10FA000010BC704710B40446084611461A4614B993
:10FA100010BC00F061BDC8B210BC70470048704710
:10FA200001000102064B10B51B6A0446984730B12D
:10FA30000448054B204498428CBF0020012010BD93
:10FA40005C76010840C220C980B92A00F0B5114B8C
:10FA500085B00C4610491F56054601F04BF80F4B78
:10FA6000E4B25E6A072D4FF00103CDE9024301467F
:10FA70000AD105220023CDE900234FF47A727A439C
:10FA80001846B04705B0F0BD08220020CDE900209F
:10FA90003A46F5E740700108207001085C760108DD
:10FAA0001FB5002300930378013B372B21D8DFE8F3
:10FAB00003F01C242020201E202020204143454EFE
:10FAC0002055585B5E6164206C1E6E73787A20202E
:10FAD0007D81262020202020202020202020202062
:10FAE00083858A2020838A208C90C3780BB10223DF
:10FAF0000093009805B05DF804FB8378F6E743783F
:10FB00008DF8043005238DF805308378003B18BF4D
:10FB100001235B008DF8063010238DF80730304B41
:10FB20001B6801A803F55872CDE9022300F0C2FF5B
:10FB30000090DEE74023DBE72023D9E7827890F9C5
:10FB4000013012B9274AD35CD2E7274AFBE7827813
:10FB500090F90130002AF8D1244AF4E740F6B8338E
:10FB6000C6E74FF47A73C3E74FF4FA63C0E741F294
:10FB70008833BDE741F27073BAE71D484FF47A71DC
:10FB800001F03CFE00F5FA60D2E71A4BB0E7144BE7
:10FB90001B6803F55873ABE7114B1B6803F55B73E8
:10FBA000A6E71023A4E70E4B1B68A1E74FF08343A1
:10FBB00000939EE7104BFBE7104B99E740F21113BF
:10FBC000ADF8003095E7032392E790F901300C4A35
:10FBD000B9E70C4990F9010000F08CFFA8E700BFDD
:10FBE000A826002015700108057001080D70010895
:10FBF00018FCFFFF00EA06379A99094040F70937D9
:10FC0000407001082070010837B50B4B02781B6863
:10FC10000C2101FB02335B7A03EB4304074B1D68A5
:10FC200003690093C3684278816805EBC40000F063
:10FC3000DDFC03B030BD00BFA8260020A4260020B4
:10FC400070B586B0027B6423ADF80030012A4FF016
:10FC50000003CDE90133CDE903338DF802308DF88F
:10FC6000143030D0022A39D05ABB03684BB34368F2
:10FC70003BB31F4D80682B601E4B182269461860ED
:10FC800001F0D8FD1C4B2C6893E807000C3384E886
:10FC9000070093E8070004F10C06032386E8070039
:10FCA000A4F86C33012204F55B7104F5587000F080
:10FCB0008EFC2B684FF6B072A3F878230522C3F8A8
:10FCC0007C2306B070BD0A4908684360036100F5F3
:10FCD0005B7100F5587000F07AFCF2E7044B1B688A
:10FCE000B3F86023B3F86C130A43A3F86023E8E782
:10FCF000A8260020A4260020F86C010808B50346B9
:10FD00000A2924D8DFE801F006232323230B161B3E
:10FD100023212100BDE808400068FFF783BE90F969
:10FD200000009978052271B900F011FC003818BF65
:10FD3000012008BD052293F900000021F4E790F9A5
:10FD400000005978EEE70221EEE70722F3E70020F2
:10FD5000EFE7000008B502791AB1012A0BD00020A4
:10FD600008BD084B01681B68012203F5587000F0BC
:10FD70002EFC0120F4E7034B01681B6803F55B7060
:10FD8000F5E700BFA8260020F7B50528144D1C464E
:10FD9000A8BF052058700E462946174600F0AAFE57
:10FDA00094F90130A070072B13D1322000F0A2FD8E
:10FDB0000C4BDB6D0546984704F10C0208340346F2
:10FDC000019200943A463146284600F098FD03B06F
:10FDD000F0BD054A55F82310D05C00F083FDE7E73D
:10FDE000207001085C760108407001082DE9F04F91
:10FDF000344F90F901607B68D0F804908BB00446D2
:10FE0000884698470546002859D1E37C73B92E4AA5
:10FE10002378126803EB4303990002EB8303D3F8C2
:10FE20000490B9F1000F01D152F80190274B4846D8
:10FE300013F906B0FB689847A37C2289D7F818A06D
:10FE40000993072E28D100230121CDE90223204A5E
:10FE50000693CDE90431CDE907330521CDE9002131
:10FE60004FF47A7202FB0BF24CF250311846D04735
:10FE7000637C13B3174B995D7B6D0D31C9B2284676
:10FE80009847E07C3246494600F046FE88F800601C
:10FE900001200BB0BDE8F08F002101250823CDE93A
:10FEA0000013CDE90715CDE90511CDE90311029243
:10FEB000A1782B465A462846D9E7074BDBE70020B6
:10FEC000E7E700BF5C760108A82600204070010823
:10FED000854501000D700108157001082DE9F04FEE
:10FEE0008DB090F90130DFF8FCA0DFF8FC90CDE98F
:10FEF0000A123E4A12F903B00278DAF800300C25F3
:10FF000005FB02333A4A5B7A126803EB430302EBC8
:10FF1000C303044693F9021090F9020000F0E5FDD6
:10FF20003449064694F9010000F0E4FDA2686168D6
:10FF30008046304600F00BFD2178DAF80020D9F831
:10FF40000C306943074650589847D9F81C309C46F6
:10FF500094F901300025072B4FF47A63CDE907535C
:10FF6000CDE905552DD10123CDE903530523CDE975
:10FF700001534FF47A7303FB0BF300933946434666
:10FF800046F2A81228466746B8472378DAF80020D8
:10FF90000C214B4394F90110D05800F0DFFDA189EA
:10FFA00094F90100FFF752FD0B9B217B1860D9F8F3
:10FFB0005430284698470A9B01201E700DB0BDE8BA
:10FFC000F08F01200823CDE90350CDE901032A4633
:10FFD000CDF800B0654643463946A847012005469E
:10FFE000D3E700BFA82600205C7601084070010816
:10FFF000A4260020207001082DE9F04F8FB00024C6
:020000040801F1
:1000000005468A46914698460494ADF81440ADF8EA
:10001000024007264FF0010B2B7AA34206D96868ED
:1000200004A9204400F0F6FB00285ED102238DF8DD
:10003000083002A86B7A8DF80A30FFF731FDAB7AF1
:100040008DF81D309DF811308DF81E309DF812305E
:100050008DF81F309DF810308DF82030EB7A8DF838
:1000600021302B7B8DF822306B7B8DF823301023D1
:100070008DF81C608DF824303A4E8DF82C000DF16F
:1000800002030A9305238DF82D3033680C93072360
:10009000ADF834302B6806930DF1120204AB0DF16C
:1000A000110106A800F0D0FB072805460BD13068E7
:1000B0000C22002100F5587001F0D0FB3368BDF828
:1000C0000220A3F860239DF811308AF800309DF8D3
:1000D000123089F800309DF8103088F80030189BF5
:1000E00028461C700FB0BDE8F08F9DF81330BDF8A6
:1000F0001470ADF802702044C4B2F3B917B3194AB2
:1001000000201168072602464FF00C0C062B1BD16D
:100110000CFB00FE51F80EE0BEF1000F04D00BFA0C
:1001200000F23A4397B2012201301028EED1002AA2
:100130003FF472AFADF802706EE75A1E042A01D97F
:10014000062BDCD0062667E747FA00FE1EF0010FFB
:10015000EAD00CFB00FE51F80EE0BEF1000F08BF24
:100160000626E1E7A826002038B505464068FFF7D7
:1001700059FC0522841D002195F90000E4B200F02D
:10018000E6F908B904F0FD0495F901000722002101
:1001900000F0DDF908B904F0FB04204638BD00206A
:1001A0007047000010B503780F2B044618D840683C
:1001B000FFF738FC22780B4902EB42020968831CE6
:1001C00001EB820051F82220DBB21AB903F0FD03E3
:1001D00058B210BD032B06BF626842600223F7E7E6
:1001E0000020F6E7A8260020022070472DE9F04FF6
:1001F000DFF838810446D8F8000099B089461746E0
:1002000000211E460122032300F55870CDE9061196
:10021000CDE908118DF814108DF81510ADF81630D1
:1002200000F0B7F938B9D8F80020B2F8603343F0DD
:100230000303A2F86033D8F80020637A8DF82830E1
:1002400002F55871CDE90B12394A94F90830126859
:100250000D920DF116020F922268109262681192AF
:10026000D4E90301A27A8DF8482001228DF84920B3
:1002700013AA82E803001025227DE18A8DF8293037
:1002800018468DF85420ADF83850FFF7DFFB0AAB65
:1002900017930DF11503169000933146019705ABA6
:1002A00006AA10A800F0C2FB064698BB9DF81410E1
:1002B000204F013901F0A2FA1F4B1B690393C4B20E
:1002C0004FF00C0B04F160036B44D8F8000013F8F6
:1002D00048AC9DF814300BFB0AFC01343946B4FBE2
:1002E000F3F203FB1244D0F87C33B0F9782350F8D2
:1002F0000C00DDF80CC0E4B2E04728B189F800A09A
:10030000304619B0BDE8F08F013D15F0FF05D9D199
:100310000D26F5E70C2801BFD8F80020B2F86033AD
:1003200043F00303A2F86033EAE700BFA8260020E9
:10033000A4260020400D03005C760108F8B506797C
:10034000012E054648D90F2E48D80368187A40F385
:1003500003000522002140B200F0F9F82B680446A2
:10036000187A40F303100522002140B200F0EFF8A4
:10037000B8B1B4FA84F4640929680B7A086843F3C5
:10038000030243F303135BB252B29A42C8BF012483
:10039000FFF748FB80F00103DBB224B10533D8B28C
:1003A000F8BD0124E8E7DBB90E4F29683B6806EB8E
:1003B000460003EB80000C2201F03CFA3A680C2363
:1003C00003FB062320465C72B2F860130123B3409E
:1003D0000B43A2F86033E3E70620E1E70320DFE701
:1003E0000420DDE7A826002010B4017801290ED9E9
:1003F000084B18680C234B43C4180022C250C4E9B0
:10040000012200F5587010BC102200F0A9B800209D
:1004100010BC7047A82600202DE9F04186B050237B
:100420008DF81430037A102B074630D14368DD7BFA
:100430006DBB0224A8466426062C14D87A68535D46
:1004400003932A44517843EA01230393927843EAC1
:1004500002437343CDE9033863B968468DF8004021
:10046000FFF7C2FF0DE0CDF80C808DF81480CDF8B9
:100470001080F2E703AB01A801938DF80840FFF765
:100480005DFF0134E4B2102C05F10305D4D106B0B0
:10049000BDE8F0811FB502680379116849B901A868
:1004A0008DF80430FFF7A0FF78B1032005B05DF8A8
:1004B00004FB02A802928DF80C30FFF73FFF0428DE
:1004C00005D0052805D00028EFD00020EEE7022057
:1004D000ECE70120EAE70000C90020B9034B0B4418
:1004E0009856C0B27047024BF9E700BFC56F0108CC
:1004F000856F0108F0B59A42069D03DB9DF9143023
:100500009A4220DD0020F0BD03EB430331F814C014
:1005100005EB830300264CFA06F7FF0707D51F7A81
:1005200007F00F0E964502DCB2EB171F0DDD01360A
:10053000102E03F10C03EED10134E4B22301DBB23F
:100540009842E1D8DEE70024F8E70120DBE78842A3
:1005500004DB9042CCBF0020012070470020704790
:1005600010B51409B4EB111F03464FEA11100ED356
:1005700091420CD202B201F00F0133F81240012077
:1005800000FA01F124EA010123F8121010BD002045
:10059000FCE7F0B528B100EB4105012700209142AE
:1005A00000D3F0BD002435F802CB234607FA04F649
:1005B00036EA0C0608BF013304F1010408BFDBB2C0
:1005C000102CF3D118440131C0B2C9B2E7E710B51D
:1005D00000B149B910BD31F8134020F81340013380
:1005E000DCB2A242F7D8F5E70023F9E782B030B5D4
:1005F00004880493D2B9B3F5616F15D349F6AF25DA
:1006000042F21072AB4298BF4FF47A72944238BFF4
:1006100014466143BDE83040C3688B428CBF5B1A0F
:100620000023C36002B070476422EFE7012C38BF9B
:100630000124EEE72DE9F04F8FB01546199F039383
:100640009DF8603007930C46804603F0C7FB6A4A6A
:100650000590A7F5F633303BB3FBF2F3534303F5B4
:10066000F63B0493182313FB05430BF1300B069361
:1006700000254FF0FF3A069B9C4207D1002D14BF86
:1006800050464FF0FF300FB0BDE8F08FBDF9683035
:10069000ADF82430099919973846089703F02EFBD6
:1006A0002688B8F1000F5FD1B7F5616F5AD349F6CC
:1006B000AF2242F21073974298BF4FF47A739E4272
:1006C00038BF1E46642E59D1DFF83091A060A16872
:1006D0000CA803F035FB0D9B0093DDE908120C9B81
:1006E0000AA803F08CFA039A0A9B0AB9079A2AB15E
:1006F00022694A4502D1424A93420ED9414BC4F87D
:100700000C909F4209D90023ADF82C300B99CDF8FD
:1007100028B0584603F0F2FAA060606808B9C4F83F
:100720000C90C4F81090B8F1000F04D003F060FBF7
:10073000E3680344E360D4E903329342059B88BF36
:10074000E26063601B9BE1687343994204D20398A3
:10075000E8B9B8F1000F1AD001231D442375EDB29A
:10076000183488E76423AAE7039B0BB9234BE360A3
:10077000012EDFF8889038BF0126CEE7B6F57A7FE4
:100780000ABFDFF88490DFF88490A0609FE7002024
:100790009342207506D85B1A9A4505F1010528BFDA
:1007A0009A46EDB2B8F1000FDAD1642E184AADF8CE
:1007B0002C801DD049F6B023B6F57A7F18BF1346BA
:1007C000974281BF049A02F5A83202F5C0729B18C5
:1007D0000A931A9B00930AAE96E80600199B3046CE
:1007E00003F00DFA96E8030003F088FA8246B7E7B3
:1007F0004FF46163E4E700BF8051010040771B00C4
:100800007F5101002FEC010080A81201002E9302FD
:1008100030EC01000378032B14D1437803F00F026E
:100820001B098A704B7083788B80C27843EA02235D
:100830008B800379C3F3021203F00F03CA700B70AD
:1008400005207047002070472DE9F3479A46437909
:10085000057990F907609146044690F9062088468C
:10086000D3B190F90870002D37D00F2A1BD194F91D
:1008700009200F2E27D194F90A00072D02D1002F4D
:1008800008BF012788F8002089F8000028468AF868
:10089000007002B0BDE8F08790F90B7090F9092064
:1008A00090F90A60DFE7A369019394F9153000938A
:1008B00094F914302169207BFFF71CFE0028D8D161
:1008C00005F0FD05D5E794F91D00B042D5DC94F99B
:1008D0001C30B34203DA05F0FB053046D2E7304660
:1008E000CBE70000024B03FA00F0B0FBF1F07047D9
:1008F00040420F004FF4FA53B3FBF0F0704730B5AD
:100900004FF47A750C1F6A4300FB042252001EBF8D
:1009100000F1FF341219B2FBF0F2914238BF1146D8
:10092000039A1160820048431CBF013040084FF415
:100930007A71121A01FB1323002BCABF03F2E733AB
:1009400093FBF1F1B3FBF1F1049B196030BD38B5B5
:10095000400014460D46F1F7DDFA01462846F1F74E
:1009600027FA2146F1F724FAF0F7EEFE06F01CF91B
:10097000F1F7F2F940B238BD2DE9F74F01930023AA
:100980009C469E46048A1E01F6B2B44246D906EB46
:1009900046054FEA4309AD000024476837F809705F
:1009A0002741FF0729D5876807EB050A7F5927B339
:1009B000077837B9476927B137F809702741FF072A
:1009C0001BD59AF8087090F901B047F303084FFA65
:1009D00088F8D84511DC47F303177FB25F450CDB7D
:1009E0009AF8097007EB4708C76807EBC8073F7D0F
:1009F0005FB90CF1010C5FFA8CFC0134102C05F18D
:100A00000C05CAD10133DBB2BCE70EF1010706EBDE
:100A1000040801F80E805FFA87FEEEE7019B82F87A
:100A200000E083F800C003B0BDE8F08F2DE9FF4778
:100A300004464068DDE90C671D468A46914603F08E
:100A4000D7F923681B1A3B604FF00008012333706D
:100A500085F80080636813B12368834224D8D4F8F2
:100A60001CC0CAF80080A3699CF800E00393D4E995
:100A7000030101AB83E80300237D0093DCF80C1035
:100A8000237A627A7046FFF7D5FD334638602A46EE
:100A9000E0694946FFF770FF2B782BB1C7F800805B
:100AA000002004B0BDE8F0873378002B0CBF0C2089
:100AB0000B20F6E737B590F9002090F902509542E7
:100AC00004460FD0013A52B295420BD0A36801936D
:100AD00094F9013000936168E0782B46FFF70AFD36
:100AE0000028EFD0104603B030BD8842B8BF08469A
:100AF0007047000051F82000054B984205D0054B87
:100B0000C31A58425841400070470120704700BF47
:100B100090D0030020A1070005281FB50ED80C4B6C
:100B200053F820300093CDE901120A4B0122002135
:100B3000022002F06BFE05B05DF804FBCDE9001267
:100B4000054B01220021022002F060FEF3E700BF06
:100B5000B4700108487001086770010807B5054BBB
:100B6000CDE9000101220021022002F04FFE03B076
:100B70005DF804FB8370010810B5102204460021C3
:100B8000F13000F06BFE0021C4F814112046F02271
:100B9000BDE8104000F062BE02460846102100F099
:100BA000A5B92DE9F0430446D0F8140185B00E46EE
:100BB000154604F2011988B3C0F110089045474664
:100BC00028BF1746BAB2484400F034FED4F81431B6
:100BD0003B440F2BC4F814312DD9A8452BD204F176
:100BE000F00304F5807113F8012F187C8B4282EA20
:100BF00000021A70F7D104F1F1081022414668464C
:100C000000F018FE22466946684600F0F1F910220D
:100C10006946404600F00EFE3E44ED1B04F5807828
:100C200004F1F107102D09D8AAB23146484600F068
:100C300001FEC4F8145105B0BDE8F08304F1F003DF
:100C4000711E13F8012F11F8010F434582EA0002CB
:100C50001A70F6D110223946684600F0EBFD2246A4
:100C60006946684600F0C4F910226946384600F02B
:100C7000E1FD1036103DD5E7F0B589B00C461022E5
:100C800000210546684600F0E9FD224669466846AF
:100C900000F0AEF99DF90030002B6A464FF00001DC
:100CA00043DA137812F8010F01315B0043EAD013E5
:100CB0000F2902F8013CF4D19DF80F305B0083F05E
:100CC0008703D4F81401DBB210288DF80F303BD124
:100CD00004F58073694604F5887013F8016F11F804
:100CE000012B984282EA06021A70F6D104F1F00351
:100CF00004F5807113F8012F187C8B4282EA000200
:100D00001A70F7D110220DEB020004F1F10100F08E
:100D100091FD2246294604A800F06AF9102200211C
:100D2000684600F09BFD09B0F0BD137812F8010F82
:100D300001315B0043EAD0130F2902F8013CF4D1E2
:100D40009DF80F305B00BCE79DF90030002B6A4630
:100D50004FF0000137DA137812F8016F01315B00B0
:100D600043EAD6130F2902F8013CF4D19DF80F3065
:100D70005B0083F08703471CDBB28DF80F30102F28
:100D800004EB0003C0F10F064FF0800288BF00267D
:100D900000F5817083F801210021324620443E4451
:100DA00003F0D3FFC4F8146104F58073694604F5B9
:100DB000887013F8016F11F8012B984282EA06023D
:100DC0001A70F6D192E7137812F8016F01315B00C7
:100DD00043EAD6130F2902F8013CF4D19DF80F30F5
:100DE0005B00C8E70A780378534003704A78437879
:100DF000534043708A78837853408370CA78C378AD
:100E00005340C3700A790379534003714A79437997
:100E1000534043718A79837953408371CA79C37986
:100E20005340C3710A7A037A534003724A7A437A71
:100E3000534043728A7A837A53408372CA7AC37A60
:100E40005340C3720A7B037B534003734A7B437B4B
:100E5000534043738A7B837B53408373CA7BC37B3A
:100E60005340C373704710B50B7814786340037018
:100E700054784B786340437094788B7863408370E8
:100E8000D478CB786340C37014790B7963400371D5
:100E900054794B796340437194798B7963408371C2
:100EA000D479CB796340C371147A0B7A63400372AF
:100EB000547A4B7A634043728B7A947A634083729C
:100EC000D47ACB7A6340C372147B0B7B6340037389
:100ED000547B4B7B63404373947B8B7B6340837376
:100EE000CB7BD27B5340C37310BD0000A1F1100334
:100EF000DBB2102B2DE9F047044604D83A4820FA1B
:100F000003F3DB0705D4002382F8F030FF20BDE8AF
:100F1000F087561E254615F8013B06F8013F631B76
:100F20000B4413F0FF00F6D101F11C039B005FFAA4
:100F300083FCC3F30313013BDFF8B09082F8F03079
:100F4000884653184FF0010EB8FBF1FA01FB1A8ADC
:100F50001AF0FF0A13F8047C13F8036C13F8025C10
:100F600013F8014C30D119F806A019F8056019F8EA
:100F7000045019F807404FEADE1707EB47078EEADF
:100F80000A0A07EBC7074FEA4E0EFFB25FFA8EFE62
:100F900087EA0E0E574692F800A087EA0A071F70EC
:100FA00057787E405E70967875409D70D57808F1D0
:100FB00004085FFA88F86C40C445DC7002F1040252
:100FC00003F10403C0D8A2E71829E4D9BAF1100F3D
:100FD000E1D1DFF818A01AF807701AF806601AF8BD
:100FE00005501AF80440D6E701010100CC7201084F
:100FF0002DE9F04FA3B092F8F0301D911B920193B0
:10100000002B00F0538101461EA8FFF72CFF1B9B0D
:10101000A74CA84DA84E10330293002303939DF8CC
:101020007C0004909DF886000590205C06909DF859
:101030007B000790205C089004989DF881C0205C9C
:10104000099014F80C000A909DF880000B909DF810
:1010500085009DF878809DF87DE09DF882A09DF840
:1010600087900C909DF87A00029B1C9314F80A203C
:1010700014F8093014F8081014F80E700D90205C64
:101080000E909DF87F000F90205C10900B98205CD4
:1010900011900C98205C12909DF8840013909DF89C
:1010A000790014909DF87E001590205C16909DF8B4
:1010B00083001790205C18901398205C1990149866
:1010C000205C1A900398013003900298DDF804B078
:1010D000103002909DF80C00834536D88DF87810BA
:1010E0008DF87A2009990E9A8DF87C108DF882205F
:1010F0001199069A8DF880108DF87E201999169A0C
:101100008DF884108DF886200A99189A8DF87D1034
:101110008DF887201299109A8DF87B301B9B8DF8E3
:1011200081108DF883201A99089A1D988DF88510E2
:101130008DF87F201EA903EB0B128DF87970FFF755
:1011400092FE002023B0BDE8F08F15F808B082EAC7
:1011500003008BEA000016F80EB080EA0B008DF851
:10116000780015F80E004B40434016F80A00434043
:101170008DF8793081EA070315F80A10594016F8FE
:101180000930594016F808308DF87A107A405340EB
:1011900015F8092053408DF87B30089A069B534080
:1011A000049AAA5C534016F80C2053408DF87C300A
:1011B000DDE908325A4015F80C305340059AB25C0C
:1011C00053408DF87D30DDE909325A40059BEB5CD8
:1011D0005340079AB25C53408DF87E30069B0A9AC2
:1011E0005340049AB25C5A40079BEB5C5A408DF81E
:1011F0007F200E9B109A53400B9AAA5C53400C9A86
:10120000B25C53408DF88030DDE910325A400C9BBF
:10121000EB5C53400D9AB25C53408DF88130DDE9B0
:1012200011325A400D9BEB5C53400F9AB25C534015
:101230008DF88230129A0E9B53400B9AB25C5A4042
:101240000F9BEB5C1C995A408DF88320169B189AD3
:101250005340139AAA5C5340149AB25C53408DF8E1
:101260008430DDE918325A40149BEB5C5340159AE8
:10127000B25C53408DF88530DDE919325A40159B38
:10128000EB5C5340179AB25C53408DF886301A9A43
:10129000169B5340139AB25C5340179AAA5C1EA83F
:1012A00053408DF88730FFF79DFDB8E6FF2049E7F2
:1012B000CC720108CC710108CC70010808B538B1B6
:1012C000044A05491060D82200F0B4FA002008BD95
:1012D0000220FCE7AC260020687B01080A4B1A6854
:1012E00070B5002302F1180503EB03142E5D86424E
:1012F00004D1183422440A60002070BD01330B2B46
:10130000F2D10320F9E700BFAC2600202DE9F0411F
:10131000CCB00646DDF8488117461C460D4631B371
:10132000B8F1000F23D006A8FFF726FC204601A93C
:10133000FFF7D4FF0446B0B9019906A80131FFF7C1
:101340002BFC26B11022314606A8FFF72AFC3A46AC
:10135000294606A8FFF725FC06A902A8FFF78CFC82
:10136000029BC8F8003020464CB0BDE8F081022452
:10137000F9E7000030B595B013A90446FFF7AEFFBA
:10138000002830D11B4B0C2101FB00F2D5189A5CD0
:10139000A2422AD1139B1A7C1092DA7B0F929A7B7D
:1013A0000E925A7B0D921A7B0C92DA7A0B929A7AF1
:1013B0000A925A7A09921A7A0892DA7907929A79F5
:1013C00006925A7905921A790492DA7803929A78F9
:1013D00002925B7801930022AB6800931146064BA2
:1013E000022002F013FA15B030BD01300B28CBD12A
:1013F000F9E700BF44750108CC73010810B40B2B4A
:10140000019C03D8019410BCFFF780BF032010BCDF
:10141000704730B50D4685B01446014668B103AA41
:10142000002000922A460390FFF770FF18B9039836
:10143000001B18BF012005B030BD0220FBE72DE9DD
:10144000F0430D46BFB014469946804620B31BB307
:1014500011F00F0122D1F02201A800F0FFF920467F
:101460006946FFF73BFF044648B9009801AA1021DE
:101470000130FFF73BFD2E46AF1BFFB21EB92046E1
:101480003FB0BDE8F08301AA09EB070108EB0700B4
:10149000FFF7AEFD103EEFE70224F0E70524EEE78C
:1014A000F0B5184E3468024685B00846002304F1B2
:1014B000180103EB03154F5D97421ED10D2A05F16C
:1014C000190513D10023CDE90033CDE902330C22F5
:1014D00010216B46FFF7B3FF0446306810226946BF
:1014E000284400F0A7F9204605B0F0BD01461022BF
:1014F000601900F09FF90024F5E701330B2BD8D1D8
:101500000324F0E7AC26002009B1FFF7C9BF022091
:1015100070471FB51446A0B10C2A01D10B2912D176
:101520000023CDE90033CDE902330A466B46102192
:10153000FFF785FF18B969462046FFF7B1FF04B0F1
:1015400010BD0220FBE70320F9E7F8B51E46DDE9F0
:1015500007479DF818505BB354B34FB3212D29D8DA
:1015600019462A46204600F065F90122631C691ECF
:10157000B018FFF764FFF8B9E37ADB093B70EBB909
:101580006319204613F8012C13F8021C120642EAD4
:10159000014213F8041C0A4313F8031C012342EA16
:1015A0000122291FFFF735FF003818BF0120F8BDC1
:1015B0000220FCE70520FAE70720F8E70420F6E719
:1015C00010B5044628B1044B5B69984720600020A1
:1015D00010BD0220FCE700BF5C76010808B501469B
:1015E00030B1044B0822186800F024F9002008BD2F
:1015F0000220FCE7AC26002008B530B1044B0822DD
:10160000196800F017F9002008BD0220FCE700BFB0
:10161000AC2600207FB5124E0023044602A8019399
:101620000D46FFF7E9FF33685B6901936CB102AACD
:10163000082312F8011B41B9013B13F0FF03F8D155
:1016400002A8A04702A8FFF7C9FF35B1019B23B943
:1016500001A8A8473368019A5A61002004B070BD00
:10166000AC26002008B5014638B1054B18680822A1
:10167000104400F0DFF8002008BD0220FCE700BFA6
:10168000AC26002008B538B1044B19680822114473
:1016900000F0D0F8002008BD0220FCE7AC260020B6
:1016A000034B1B6802280CBF196159610020704769
:1016B000AC26002049B1064B1B68D3E9042302285D
:1016C00008BF13460B60002070470220704700BF20
:1016D000AC26002030B58FB0002405460CA8099434
:1016E000FFF78AFF9DF8373007939DF83630069351
:1016F0009DF8353005939DF8343004939DF83330D0
:1017000003939DF8323002939DF8313001939DF898
:1017100030300093224621461E4B022002F076F81C
:101720000AA8FFF7AFFF9DF82F3007939DF82E30E2
:1017300006939DF82D3005939DF82C3004939DF869
:101740002B3003939DF82A3002939DF829300193A2
:101750009DF82830009322460F4B2146022002F0CC
:1017600055F809A92846FFF7A5FF9DF824300393F3
:101770009DF8253002939DF8263001939DF827307F
:1017800000932246054B2146022002F03FF80FB09D
:1017900030BD00BF2874010866740108A4740108F4
:1017A00008B50020FFF7E6FD0120FFF7E3FD092063
:1017B000FFF7E0FD0820FFF7DDFD0020FFF78AFFBF
:1017C000002008BD10B504460B20FFF7D3FD0C2008
:1017D000FFF7D0FD0920FFF7CDFD0820FFF7CAFD78
:1017E0000A20FFF7C7FD2046FFF774FF002010BD59
:1017F000014B1860704700BFAC0800200B4A30B5A1
:1018000014680B4D43F2390305FB04331360091AC6
:101810006FF00042B3FBF2F2C2EBC27201319B1ACD
:1018200093FBF1F201FB1233184430BDAC080020E9
:101830006D4EC64101380A44914200D1704711F8FB
:10184000013B00F8013FF7E710440A44914200D100
:10185000704711F8013B00F8013DF7E703F075BA56
:1018600030B530B10A4D01444FF0FF33814201D110
:10187000D84330BD10F8012B5340082243F3000435
:10188000013A2C4092B284EA5303002AF6D1EDE7E4
:101890002083B8ED01207047054B4FF400529A6247
:1018A000044B1B6813B15B6803B11847704700BF56
:1018B000000400483C270020054B4FF480529A62F8
:1018C000044B1B6813B1DB6803B11847704700BFB6
:1018D000000400483C270020012070470120704789
:1018E00001F03EB901F02CB910B501F00FFE0E2148
:1018F000044640F61F1001F023F92046012101F0B3
:10190000EFFDBDE8104001F0CDBA000070B50C4EFF
:1019100001EB40030D46B3654FF6FF71002304460B
:101920001A46084601F054FB96F85600002101F0D3
:10193000D7FD29462046BDE8704001F08BBA00BFB4
:10194000E026002010B5044601F0A0FE01281CD1BD
:1019500001F0A4FE34B11248214602F00BFB1048FE
:1019600002F0CEFA0F4C104B00214FF48052A165CB
:101970009A6194F8560001F0B3FD63786BB16FF093
:101980007F40BDE8104001F049BA002340F26221D7
:101990001A46084601F01CFBDCE7A0688001F0E76E
:1019A000B0260020E026002000040048002001F0BE
:1019B000B5B9000008B501F0BDF80438C0B203287D
:1019C00096BF024B0020185C08BD00BF26760108B8
:1019D00008B501F0B0FD033008BD01F03FB901F0DA
:1019E000FFB808B501F0F6FC08BD000038B50D469B
:1019F000144601F053FB284601F088FD0E210546F0
:101A000040F61F1001F09CF828460121074D01F017
:101A100067FD01F047FA4FF47A716143284602F0FE
:101A2000A9FA2846BDE8384002F06ABAC826002064
:101A300001F034BB08B5084B002193F8560001F0C3
:101A40004FFD00234FF4C0711A46084601F0C0FA5A
:101A5000BDE8084001F01ABAE026002010B504469F
:101A600001F014FE01281CD101F018FE34B1124817
:101A7000214602F07FFA104802F042FA0F4C104B58
:101A800000214FF48052A1659A6194F8560001F04C
:101A900027FD63786BB16FF07F40BDE8104001F027
:101AA00073B9002340F262211A46084601F090FA09
:101AB000DCE7A0688001F0E7B0260020E0260020E7
:101AC0000004004808B54FF0040001F00DF9BDE82E
:101AD00008400220F1F750BA08B500231A4619460B
:101AE000184601F075FABDE8084001F063B900003E
:101AF0001D4B73B51D4D186000241D486C70C5E961
:101B00000144AC6501F08EFAAC8101F0F9F921468F
:101B1000204601F041FC21460422012001F0F2FAA6
:101B2000144E154D4FF6FF7123462246084601F02C
:101B30004FFAFFF7C7FF2246104B00944FF0FF31DA
:101B4000304602F031F90E4B009422464FF0FF313F
:101B5000284602F029F9304602F084F9284602B0FE
:101B6000BDE8704002F07EB93C270020E02600204E
:101B7000252B0108C8260020B0260020991801084E
:101B8000B91801080128084805D1084BC177197018
:101B90000E3001F09DBB437D012B03D1034B8175BA
:101BA0001970F5E7704700BFE0260020B00800205C
:101BB0000D4B10B5044618735873012000F016F849
:101BC0005CB134214FF4E86000F0BAFF4421BDE875
:101BD000104040F2417000F0B3BF14214FF4E860B0
:101BE00000F0AEFF2421F2E7E026002038B5114CCA
:101BF0000546207001F057FD052D04D8DFE805F0FB
:101C0000090B03171709032001F066FA0023637319
